:100000000C94FE040C9444050C9444050C94440593
:100010000C9444050C9444050C9444050C9444053C
:100020000C9444050C9479190C9444050C944405E3
:100030000C94EE300C9444050C9444050C94440547
:100040000C9444050C9444050C9493150C944405AD
:100050000C94170C0C9444050C94E10B0C9444057F
:100060000C946A1B0C9444050C94082C0C944405C5
:100070000C94B5700C9444050C94146B8F1B941B5A
:10008000991BA21BB91BD01BE01BF01B341C0F1EBD
:10009000D01B0A1D1B1D2F1D4D1D6A1DB51D011EE8
:1000A000FF1FDB204B21CA2102229B222F23DE24AB
:1000B0005F259A251526432670260A0D3D3D3D3DB8
:1000C0003D3D3D3D3D3D3D3D3D3D3D3D3D3D3D3D60
:1000D0003D3D3D3D3D3D3D3D3D3D3D3D3D3D3D008D
:1000E0000A0D426174743A002025642043656C6CEB
:1000F000732000204C6F77207761726E696E673ACB
:100100002025642E2564560020204175746F2D43F0
:10011000483A2025642E2564560020204175746FCE
:100120006C616E64696E673A2025642E2564560002
:100130000A0D4F6C642046432048617264776172F7
:1001400065206E6F7420737570706F7274656420B3
:1001500062792074686973204669726D776172658F
:1001600021000A0D466F756E6420424C2D43747257
:100170006C3A20002564000A0D0A0D2121204D490A
:100180005353494E4720424C2D4354524C3A20255C
:1001900064202121000A0D43616C696272617469F7
:1001A0006E672070726573737572652073656E7308
:1001B0006F722E2E004F4B0A0D000A0D466C6967B8
:1001C00068742D74696D65202575206D696E2054E5
:1001D0006F74616C3A2575206D696E00416E676CB5
:1001E000654E69636B20202020202020416E676CC3
:1001F00065526F6C6C202020202020204163634ECC
:1002000069636B202020202020202020416363523E
:100210006F6C6C20202020202020202059617747FF
:1002200079726F202020202020202020416C7469CA
:1002300074756465205B302E316D5D204163635AB7
:1002400020202020202020202020202047617320F3
:10025000202020202020202020202020436F6D708F
:100260006173732056616C7565202020566F6C7425
:10027000616765205B302E31565D202052656365D5
:1002800069766572204C6576656C20204779726FBF
:1002900020436F6D70617373202020204D6F746F49
:1002A0007220312020202020202020204D6F746FCC
:1002B0007220322020202020202020204D6F746FBB
:1002C0007220332020202020202020204D6F746FAA
:1002D0007220342020202020202020203136202091
:1002E00020202020202020202020202031372020E6
:1002F00020202020202020202020202031382020D5
:1003000020202020202020202020202031392020C3
:1003100020202020202020202020202053657276BD
:100320006F2020202020202020202020486F76656C
:100330007267617320202020202020204375727274
:10034000656E74205B302E31415D20204361706109
:1003500063697479205B6D41685D20204865696739
:10036000687420536574706F696E74203235202074
:100370002020202020202020202020203236202055
:100380002020202020202020202020203237202044
:100390002020202020202020202020204932432DF2
:1003A0004572726F7220202020202020424C204C69
:1003B000696D697420202020202020204750535F41
:1003C0004E69636B20202020202020204750535F5F
:1003D000526F6C6C20202020202020202121212001
:1003E000494E434F4D50415449424C452021212113
:1003F000002E005B25695D005B25695D002B204DAB
:10040000696B726F4B6F70746572202B0048573A9E
:100410005625642E25642053573A25642E25303204
:1004200064256320005365743A25642025730042D7
:100430004F4154004D69786572204572726F722188
:10044000004861726477617265204572726F722034
:10045000313A2564202121004D697373696E67204C
:10046000424C2D4374726C3A2564202121002120D6
:100470004E432D4552523A20253264202120004916
:100480003243204552524F5221212100424C2D53DC
:10049000656C6674657374204572723A2532640027
:1004A0004865696768743A2020253569005365748A
:1004B000706F696E743A2535690050726573737593
:1004C00072653A253569004F66667365743A202077
:1004D000253569006163742E2062656172696E67FB
:1004E000004E69636B3A20202020202025356900CA
:1004F000526F6C6C3A202020202020253569004363
:100500006F6D706173733A202020253569004B258B
:10051000693A25346920204B25693A253469200041
:100520004E693A2534692020526F3A2534692000FB
:1005300047733A253469202047693A2534692000F9
:1005400050313A253469202050323A253469200050
:1005500050333A253469202050343A25346920003C
:100560004779726F202D2053656E736F72004E694C
:10057000636B2025346920282534692900526F6C6B
:100580006C20253469202825346929005961772099
:100590002025346920282534692900414343202D32
:1005A0002053656E736F72004E69636B202534694A
:1005B00020282533692900526F6C6C20253469206E
:1005C0002825336929005A20202020253469202835
:1005D000253369292863616C290043616C69627263
:1005E0006174696F6E3A004143433A2020204E3ACD
:1005F00025336920523A2533692000537469636BAF
:100600003A202825692F25692920212120006F6E95
:1006100020006C616E6420746F2073617665202009
:10062000202000757365206B65797320746F2074CA
:1006300072696D20414343006F66660053617665C1
:100640003F20202020202879657329286E6F2900FB
:10065000466C79207769746820475053206F66662E
:1006600000566F6C746167653A2020202533692E2F
:10067000253169560043757272656E743A202020E8
:100680002533692E2531694100506F7765723A2014
:100690002020202025346957004469736368617203
:1006A00067653A202535696D416800526563656963
:1006B0007665720052432D5175616C6974793A20E8
:1006C0002534690052432D4368616E6E656C733A40
:1006D00025346900556E646572766F6C7461676568
:1006E000732020005761726E3A202532642E2564F3
:1006F0005600486F6D653A202532642E25645600F9
:100700004C616E643A202532642E25645600506F89
:10071000746925693A202025336900506F74692572
:10072000693A202025336900466C696768742D5446
:10073000696D65202000546F74616C3A2535756DC4
:10074000696E004163743A20202535756D696E002D
:1007500028726573657429000A0D47656E657261BC
:1007600074696E672064656661756C74205061728F
:10077000616D6574657220536574202564000A0DEF
:100780005573696E6720506172616D657465722082
:10079000536574202564000A0D47656E65726174A7
:1007A000696E672064656661756C74204D69786553
:1007B00072205461626C65000A0D4D697865722D76
:1007C000436F6E6669673A202725732720282575B1
:1007D000204D6F746F727329000A0D414343206EE0
:1007E0006F742063616C69627261746564210D0AC3
:1007F000000A0D4779726F2063616C6962726174DF
:10080000696F6E2064617461206E6F742076616C14
:1008100069640D0A0000008F001E01AD013B02CA91
:10082000025803E603740402058F051B06A706336E
:1008300007BE074808D2085B09E3096B0AF20A7889
:100840000BFD0B810C040D860D070E870E060F8421
:100850000F00107B10F5106E11E5115B12CF1242E4
:1008600013B31323149214FE146A15D3153B16A167
:100870001605176717C81727188318DE1837198E3B
:1008800019E319361A871AD61A231B6E1BB61BFDDD
:100890001B411C831CC31C001D3C1D751DAB1DE0B2
:1008A0001D121E421E6F1E9A1EC31EE91E0D1F2E14
:1008B0001F4D1F691F841F9B1FB01FC31FD31FE144
:1008C0001FEC1FF51FFB1FFF1F00200A0D77777716
:1008D0002E4D696B726F4B6F707465722E6465205C
:1008E00028632920486953797374656D7320476DB7
:1008F0006248000A0D74686520757365206F662074
:100900007468697320736F667477617265206973A8
:10091000206F6E6C79207065726D697474656420E7
:100920000A0D6F6E206F726967696E616C204D6988
:100930006B726F4B6F707465722D48617264776172
:100940007265005573657200486F54542056340028
:100950004143542044534C004A6574690053706508
:100960006B7472756D0050504D000A0D52656365D1
:10097000697665723A2000756E6B6E6F776E2E2009
:100980005573696E672050504D2E2E2E006E6F7479
:1009900020737570706F727465642062792068616D
:1009A00072647761726521000A0D202D204C494246
:1009B000204E4F5420434F4D50415449424C452006
:1009C00021212121000A0D466C69676874436F6E0E
:1009D00074726F6C0A0D48617264776172653A25B2
:1009E000642E25640A0D536F6674776172653A56FA
:1009F00025642E25303264256320000011241FBE9B
:100A0000CFEFD0E1DEBFCDBF11E0A0E0B1E0E4E088
:100A1000F7EE02C005900D92A03BB107D9F71AE09E
:100A2000A0EBB1E001C01D92A431B107E1F74AEAA1
:100A3000E2E0F0E081E280935700549120EF37EF3D
:100A4000A2E8B3E09FE0F9012F5F3F4F84918D93BF
:100A5000915097FFF8CF573911F40000FECFE2E82C
:100A6000F3E09EE0819148274095915097FFFACF9F
:100A700080919103481721F0573911F40000FECFFF
:100A80000E9486060C9481730C9400008AEB90E01F
:100A90009F938F938BE992E19F938F93E0919503BE
:100AA000F091960309950F900F900F900F90089575
:100AB0000E94AD4180915F08909160082FEF8D3EBC
:100AC000920714F0109204018A5B9F4FCCF480913E
:100AD00004018823A9F481E0809304018091D0036C
:100AE0008F5F8093D003853038F088EE93E0909349
:100AF000E9018093E801089566E970E00E94F2320E
:100B000008951F93CF93DF93182F882311F180EE60
:100B100090E09F938F938BE992E19F938F93E09165
:100B20009503F091960309958091230190912401FA
:100B30006BE270E00E94F472CB018F5F8093000142
:100B40000F900F900F900F90873018F086E08093F1
:100B5000000180915906823318F590910001989F09
:100B6000E00111241123F1F068EC70E0892F0E945C
:100B7000F2328091000199279F938F9388EE90E045
:100B80009F938F938BE992E19F938F93E0919503CD
:100B9000F091960309958DB79EB706968DBF02C05A
:100BA000C82FDD27CF3FD10519F010F0CFEFD0E0EF
:100BB000C09302019091AE06923330F4809100010F
:100BC000899FE001112402C0C92FDD27CF3FD10545
:100BD00019F010F0CFEFD0E0C093B9013091AF061B
:100BE000323330F480910001839FE001112402C070
:100BF000C32FDD27CF3FD10519F010F0CFEFD0E0A4
:100C0000C093B8018091B90190910201981720F426
:100C100091509093B9019F5FC91720F09150909324
:100C2000B8019F5F8091B9012091B801821728F027
:100C3000332319F021502093B901112309F462C024
:100C4000892F6AE00E94D472892F99279F938F93EE
:100C5000809102010E94D47299279F938F9383EF12
:100C600090E09F938F93CBE9D2E1DF93CF93E09114
:100C70009503F091960309958DB79EB708968DBFA1
:100C80008091B8018823E9F06AE00E94D472892F2C
:100C900099279F938F938091B8010E94D4729927CE
:100CA0009F938F9388E091E09F938F93DF93CF93EF
:100CB000E0919503F091960309958DB79EB708963C
:100CC0008DBF8091B9018823E9F06AE00E94D47257
:100CD000892F99279F938F938091B9010E94D47295
:100CE00099279F938F938AE191E09F938F93DF934E
:100CF000CF93E0919503F091960309958DB79EB738
:100D000008968DBFDF91CF911F910895CFEFD0E16D
:100D1000DEBFCDBF88249924C1E07C2E14B815B85D
:100D20008AE08AB98FE58BB9B7EECB2EB3E0DB2E24
:100D30002EEC3FEFC20ED31ED7FEFACF189B06C093
:100D4000199B02C08DE005C08BE003C0199B04C055
:100D500084E18093030107C08AE0809303018EE35E
:100D60008AB987E48BB981E887B93E9A8FEF88B951
:100D70008BE184B981E085B9469A84B7877F84BFC7
:100D8000809160008861809360001092600084EC24
:100D900099E09093E9018093E8011092A0021092EB
:100DA0009F021092A2021092A1021092A40210922D
:100DB000A30220910301243128F084EC94E0A0E008
:100DC000B0E004C08BE095E0A0E0B0E0809341018A
:100DD00090934201A0934301B09344012898293194
:100DE00011F4299A01C029980E94E4160E94B516B0
:100DF0000E94A3120E94B5300E94CA1A81E00E948C
:100E0000B52B0E94735E0E94946887E00E945E6F1B
:100E100080910301893111F4299A01C029987894AD
:100E20000E94D12A809103018431E8F488E190E0A6
:100E30002CE00FB6F894A895809360000FBE209325
:100E4000600080E391E09F938F938BE992E19F9301
:100E50008F93E0919503F091960309950F900F9071
:100E60000F900F90EECF80913E02826080933E0201
:100E700010924102C0E0D0E00E94003E85E090E088
:100E80000E947B166C0180913E0280FD05C0C60168
:100E90000E9484168823B9F3219631E0C43FD3071A
:100EA00058F382E691E09F938F93ABE9AA2EA2E1DB
:100EB000BA2EBF92AF92E0919503F09196030995F7
:100EC000C0E0D0E00F900F900F900F900AE617E06F
:100ED000F1EDEF2EF6E0FF2EF701808124E030E007
:100EE000E20EF31E181684F406C080913E0280FFC5
:100EF00002C00E94003EC6010E948416882321F48D
:100F0000F801838188238CF7F801838187FF2CC047
:100F1000CE0101966AE070E00E94E0729F938F9389
:100F200084E791E09F938F93BF92AF92E0919503F6
:100F3000F091960309958091B1018F5F8093B10183
:100F4000F801948584E6989FC00111242585280F17
:100F50008DB79EB706968DBF222331F08091B803DE
:100F6000281710F42093B8032196015F1F4FC0315A
:100F7000D10508F4B1CFC0E0D0E00AE617E0E1ED1A
:100F8000EE2EE6E0FE2EF801838187FD1DC0F701FD
:100F900080811816CCF42196DF93CF93219787E7B1
:100FA00091E09F938F938BE992E19F938F93E091D0
:100FB0009503F0919603099582E08093E6012DB7A1
:100FC0003EB72A5F3F4F2DBFF8018381807883832E
:100FD000219624E030E0E20EF31E015F1F4FC03186
:100FE000D10588F20E944605909134068091B101A6
:100FF000981728F48091B60380618093B6039930E6
:1010000020F088E080933B0102C090933B0185E98A
:1010100091E09F938F93CBE9D2E1DF93CF93E0915F
:101020009503F0919603099588EE93E00E947B1654
:101030006C010E94081B0F900F900F900F90C6013B
:101040000E9484168823D9F385EB91E09F938F93B8
:10105000DF93CF93E0919503F0919603099580E09B
:101060000E94E833289880ED97E09093E9018093FF
:10107000E8018EE090E00E94EF289927182F0027C2
:101080008FE090E00E94EF28080F111D1093B70128
:101090000093B6018AE090E00E94EF289927182F6C
:1010A00000278BE090E00E94EF28080F111D10939D
:1010B000B5010093B4010F900F900F900F900F5F48
:1010C0001F4F39F08091B6019091B7018F5F9F4F0C
:1010D00041F41092B7011092B6011092B50110922E
:1010E000B4018091B4019091B5019F938F93809149
:1010F000B6019091B7019F938F938AEB91E09F93F4
:101100008F93DF93CF93E0919503F0919603099528
:101110000E947C1F88E893E190933A018093390103
:10112000C1E0C093D1038C2F0E94810580915C06A1
:101130000E94B16E0E94460580ED97E00E947B16EA
:101140006C018AEF90E00E947B1693E090938E05ED
:101150001092B0018091B5062DB73EB7285F3F4F82
:101160002DBF84FF02C0C093BA0190933C0112BC12
:1011700011BC8091BC01882311F04798FECF80916B
:10118000EC01882309F4FAC280911501882309F43F
:10119000F5C2F8948091EC0181508093EC01789431
:1011A0008091D003882319F00E94580502C00E9444
:1011B0007C420E94003E289880919302882331F05F
:1011C0008091930281508093930252C080916F006E
:1011D000806280936F001092620810926108809183
:1011E000B60388608093B60380913606A82FBB278C
:1011F000AA0FBB1FFD01E755F74F118210828091A6
:101200003706E82FFF27EE0FFF1FCF018755974FB7
:10121000EC0119821882AF59B74F11961C921E9299
:10122000EF59F74F1182108280913906E82FFF277E
:10123000EE0FFF1FEF59F74F118210828091380691
:10124000E82FFF27EE0FFF1FEF59F74F1182108293
:101250001092600810925F0810925D0810925C086E
:1012600010925B0810925A081092A8081092A708D2
:101270008091390190913A01019790933A018093BE
:1012800039018091390190913A01892B21F08091A7
:101290003F028823C9F18091390190913A01892B4D
:1012A000D9F40E94E62B85E090E090933A01809378
:1012B00039018091C8059091C90501969093C9059F
:1012C0008093C8058091B60381608093B6038091B6
:1012D0008F05826080938F0580910B0190910C01A6
:1012E0008F5F9F4F91F480919202882371F088EA7A
:1012F00091E69093E9018093E80180E890E0909373
:101300000C0180930B0101C028980E942D708091E0
:10131000EC01882309F030C28091E701882311F4A1
:101320000E94945E80911101882311F00E943E1763
:101330000E94F0120E946C0EC6010E94841688233F
:1013400009F416C224E130E0C20ED31E0E94FC163E
:1013500020918D0130918E018FEF2F3F3807C9F119
:1013600080917D02882369F5E091AB02F091AC0297
:10137000E217F30731F180916702882321F480910D
:1013800045038823F1F0CF01821B930B845E9D4FB0
:1013900068E671E00E94F472845B904083309105AE
:1013A0001CF082E090E006C0CFEF8E3F9C0714F463
:1013B0008EEF9FEFE81BF90BF093AC02E093AB02CA
:1013C00008C08FEF9FEF90938E0180938D01109254
:1013D000450380913F02882329F48091E6098E31EC
:1013E00050F405C08091B60382608093B60380916B
:1013F0008F0582600FC08091E8019091E901892BEF
:1014000059F48091390190913A01079728F0809121
:101410008F058D7F80938F058091BA01882361F0BD
:1014200080919302873940F01092BA0188E893E1E5
:101430009093E9018093E80180910601882321F0CF
:1014400081508093060120C0809193028823E1F4AB
:1014500080910B0190910C018F5F9F4FA9F4209117
:10146000BA01223089F088E99AE39093E9018093E8
:10147000E80180E09CE090930C0180930B01222313
:1014800019F082E08093BA018091A001893C70F04C
:1014900081508093A0018091B6038B7F8093B60327
:1014A0008091B90381608093B90353C0809168092A
:1014B0008823F9F08091B60384608093B60389E0B5
:1014C00080934A0380910B0190910C018F5F9F4F95
:1014D00081F480919202882361F088E99AE39093E5
:1014E000E9018093E80180E098EA90930C018093F1
:1014F0000B0110923C0310923B0310923A0310929E
:1015000039031092380310925B098FEF8093D00952
:1015100010929A091092990910929C0910929B09B5
:101520008FEF9FEF90939809809397091092820212
:101530001092830210928402109285021092860209
:101540008091B9038E7F8093B90310924603109265
:10155000A00160910201262F3327809123019091F1
:10156000240128173907F4F080916002806280938B
:10157000600280910B0190910C018F5F9F4F91F45D
:1015800080912301909124010B9764F080E797E10B
:101590009093E9018093E80180E093E090930C013F
:1015A00080930B018091C501882359F0815080936D
:1015B000C501813031F480ED97E09093E90180938B
:1015C000E8018091BB018F5F8093BB01813309F0FB
:1015D00086C01092BB018091460383FF02C08AE05F
:1015E00005C080915002882319F0815080935002E9
:1015F0008091600281FF0AC08091B2019091B30195
:1016000001969093B3018093B20104C05AEA852EEB
:1016100055E0952E80916102909162028050944035
:1016200008F04EC02091D7053091D8054091D905DA
:101630005091DA0580911B0190911C01A0911D0130
:10164000B0911E01281739074A075B0764F480919F
:10165000D7059091D805A091D905B091DA050596E6
:10166000A11DB11D20C02091D7053091D805409112
:10167000D9055091DA0580911B0190911C01A09130
:101680001D01B0911E0182179307A407B5079CF4B2
:101690008091D7059091D805A091D905B091DA0530
:1016A0000597A109B1098093D7059093D805A09318
:1016B000D905B093DA0580915E028B7F80935E023C
:1016C000862F9927019620912301309124018217BA
:1016D00093072CF4809160028F7D809360020894C0
:1016E000811C911C82E788168BE0980609F040C0A7
:1016F000882499242091B6013091B7012F5F3F4F84
:101700003093B7012093B6018091B4019091B50157
:1017100001969093B5018093B401832F9927682F88
:101720008EE090E00E94F7288091B6019091B70179
:101730009070682F8FE090E00E94F7288091B401AC
:101740009091B501892F9927682F8AE090E00E9437
:10175000F7288091B4019091B5019070682F8BE0CB
:1017600090E00E94F72884E190E00E947B166C01D3
:101770000E9406640E94CE6871107A94772039F432
:101780000E94CA63882319F08CE0782EF0CC8091F7
:10179000E701882309F0EBCC0E94945EE8CC40E09E
:1017A00020E030E0F901E452FE4F85919491480F1A
:1017B0002F5F3F4F82E020303807A0F3842F992716
:1017C00008951F920F920FB60F9211248F939F933B
:1017D000EF93FF93809108018823E1F48091D70172
:1017E0009091D80101969093D8018093D701FC0184
:1017F000EE54FB4FE081ED3019F08C3D910539F44A
:101800001092D8011092D70181E080930801E093F3
:10181000C60004C01092D8011092D701FF91EF9139
:101820009F918F910F900FBE0F901F9018951F9250
:101830000F920FB60F9211242F933F934F935F9304
:101840006F937F938F939F93AF93BF93CF93EF93B8
:10185000FF9390E08091BC01813029F48091C60013
:101860008093CE00D1C08091BC01823029F4809158
:10187000C6008093D403C8C08091C6008093CF0176
:101880005091DD015C3D10F09093DE018091CF011D
:101890008D3009F06AC08091DE01823009F065C0A8
:1018A0009093DE01852F99278C529C4FFC01329733
:1018B00040812091D9013091DA01241B3109DC01EA
:1018C00011978C91281B3109C9019F709093DA01FF
:1018D0008093D90146E0969587954A95E1F7982F30
:1018E000935C9093DB012F733070235C2093DC01B9
:1018F0008081981729F48C91281711F491E006C083
:1019000090E08091CC018F5F8093CC018091CE01DB
:10191000882309F079C0992309F476C081E0809387
:10192000CE01580F5093CB015150E52FFF27EC52B9
:10193000FC4F8DE080838091D603823509F064C02E
:10194000C0919202CC2309F05FC00E947C1F88E105
:1019500090E02CE00FB6F894A895809360000FBE3D
:1019600020936000C093E6014FC02091DE01822FDA
:10197000992781309105F9F0823091051CF4892B6B
:1019800021F040C0029711F13DC08091CF01833218
:1019900039F48091CE01882319F481E08093DE012F
:1019A0008091CF018093D40381E08093DD01809109
:1019B000CF01992722C02F5F2093DE01E52FFF275B
:1019C000EC52FC4F8091CF01808309C0E52FFF27A7
:1019D000EC52FC4F8091CF0180835C3D20F45F5F2F
:1019E0005093DD0102C01092DE012091CF01809161
:1019F000D9019091DA01820F911D9093DA018093C1
:101A0000D90102C01092DE01FF91EF91CF91BF91F9
:101A1000AF919F918F917F916F915F914F913F9186
:101A20002F910F900FBE0F901F901895AC01A0E062
:101A3000B0E09D01A817B90748F4E2EBF4E081910A
:101A4000280F311D1196A417B507C8F33F70FD018B
:101A5000EE54FB4FC90156E0969587955A95E1F7EC
:101A6000835C80831196FD01EE54FB4F2F73307021
:101A7000822F835C8083AD54BB4F8DE08C9310929A
:101A800008018091B2048093C6000895A0E0B0E000
:101A9000ECE4FDE00C944D732C859D850E85BB24F4
:101AA00083E28093B2049F599093B3042093B404CB
:101AB00033E0E32EF12C002309F49EC0CF84D888B4
:101AC000BE016D5E7F4FA989BA890150109709F454
:101AD00093C01097B9F0F601EB0DF11DB39490810E
:101AE000119791F4002349F1FB016E5F7F4FDB01F9
:101AF000C080D1806E5F7F4F0D90BC91A02DBB2424
:101B0000015002C090E019C01097B9F0F601EB0D3A
:101B1000F11DB3944081119791F4002341F1FB0131
:101B20006E5F7F4FDB01C080D1806E5F7F4F0D9075
:101B3000BC91A02DBB24015002C040E018C01097FA
:101B4000B1F0F601EB0DF11DB3941081119781F402
:101B5000002371F0FB013296DB01CD90DC90BF01D8
:101B60006E5F7F4FA081B181BB24015001C010E0A6
:101B7000F701EE54FB4F892F86958695835C808311
:101B80000894E11CF11CF701EE54FB4F892F9927B3
:101B90008370907024E0880F991F2A95E1F75527EC
:101BA0009A0194E0369527959A95E1F7822B835C0C
:101BB00080830894E11CF11CF701EE54FB4F4F7039
:101BC0005070440F551F440F551F812F992726E051
:101BD000969587952A95E1F7842B835C80830894FA
:101BE000E11CF11CF701EE54FB4F1F73135C1083D3
:101BF0000894E11CF11C6ACFC7010E94160DE9E0B0
:101C00000C946973A3E07A2F4091CB014650442392
:101C100009F458C0E72FFF27EC52FC4F80818D5309
:101C20007F5FE72FFF27EC52FC4F20812D537F5F12
:101C3000E72FFF27EC52FC4F30813D537F5FE72FAA
:101C4000FF27EC52FC4F60816D537F5F9927880F0F
:101C5000991F880F991F522F52955F70582B822F12
:101C600099278F709070F4E0880F991FFA95E1F72B
:101C7000232F26952695282B832F992783709070E4
:101C8000E6E0880F991FEA95E1F7682B41504F3F36
:101C9000C9F0EA2FFF27EC52FC4F5083AF5F415051
:101CA0004F3F81F0EA2FFF27EC52FC4F2083AF5FBC
:101CB00041504F3F39F0EA2FFF27EC52FC4F608331
:101CC000AF5FA5CF87ED93E09093CA018093C901E0
:101CD000A350A093C8010895A2E0B0E0E2E7FEE0BF
:101CE0000C9453738091CE01882309F420C40E9480
:101CF000020E8091D503823609F0E4C28091D603AA
:101D000099278037910509F4AFC081379105C4F454
:101D10008A36910509F441C28B36910544F48B341F
:101D2000910571F18636910509F46AC1CBC28D36F1
:101D3000910509F469C08E36910509F44DC0C2C2FF
:101D40008437910541F1853791054CF48137910530
:101D500009F491C08337910509F4EAC0B3C287370B
:101D6000910509F4DCC1883791052CF4853791057C
:101D700009F498C1A7C28937910509F47DC1A2C2AF
:101D8000E091C901F091CA01808191819093900105
:101D900080938F0197C28091CB01A091C901B0912E
:101DA000CA01853140F080E1EAEBF3E00D90019249
:101DB0008A95E1F70DC08D919D910D90BC91A02D5C
:101DC0008093BA039093BB03A093BC03B093BD036D
:101DD00080EF8093C6014BC0809108018823E1F316
:101DE0008DE490E09F938F9384EC96E09F938F9384
:101DF00081E08F938F938EE48F930E94460D8DB771
:101E00009EB707968DBF5EC2A091C901B091CA016D
:101E10001C91113081F48DE4E4ECF6E00D90019218
:101E20008A95E1F70E940C2A19838091B6038F7E70
:101E30008093B60301C01982809108018823E1F3E1
:101E400081E090E09F938F93CE0101969F938F93B3
:101E500081E08F938F938DE48F930E94460DADB7F1
:101E6000BEB71796ADBF2EC281E08093D1018FEF30
:101E70008093060127C2809192028823E1F5E091C8
:101E8000C901F091CA01E0818E2F8A508A3058F43E
:101E90008983882311F481E003C0863010F085E047
:101EA000898361E00EC08E2F84518A3070F489835B
:101EB000882311F481E003C0863010F085E0898327
:101EC00060E089810E948E2A12C0E983EF3F19F4F5
:101ED0000E946F2A89838981882311F481E003C0DD
:101EE000863010F085E0898389810E940D2980E089
:101EF0000E94810503C00E946F2A89838091080196
:101F00008823E1F38EE890E09F938F9385E396E03A
:101F10009F938F9381E090E09F938F93CE010196E2
:101F20009F938F9382E08F9381E08F9381E52DC102
:101F30002091C9013091CA01D9018C91815085301D
:101F400008F045C0F9018181893609F040C08091CF
:101F500092028823E1F52F5F3F4F8EE8E5E3F6E03C
:101F6000D9010D9001928A95E1F7F90182910E94C1
:101F70007E29809176069927AA27BB27BC01CD012F
:101F800024EC39E040E050E00E94B572DC01CB0166
:101F90008093850190938601A0938701B093880177
:101FA000809177069927AA27BB27BC01CD010E9403
:101FB000B572DC01CB018093810190938201A093E3
:101FC0008301B09384010E946F2A898301C0198222
:101FD000809108018823E1F381E090E09F938F9343
:101FE000CE0101969F938F9381E08F938F9383E52A
:101FF0008F930E94460D8DB79EB707968DBF2BC05D
:1020000080919202882309F05DC1E091C901F091AD
:10201000CA01E0818E2F8150853018F48E2F0E94E6
:102020000D290E946F2A8983809108018823E1F39A
:1020300081E090E09F938F93CE0101969F938F93C1
:1020400081E08F938F9386E48F930E94460DADB706
:10205000BEB71796ADBF10919202112341F46EE600
:1020600070E089810E94F232812F0E948105809167
:102070005C060E94B16E26C119822981A091C90116
:10208000B091CA01E1E6F8E08D91992787FD90951E
:1020900093A382A3822F8F5F8983282F32968C305F
:1020A00098F310C1E091C901F091CA0180810E94AA
:1020B00025308A83882319F481E0898301C019823D
:1020C000809108018823E1F388E090E09F938F934B
:1020D00082E697E09F938F9321E030E03F932F9328
:1020E0008091C9019091CA019F938F933F932F9341
:1020F000CE0102969F938F933F932F93CE01820F31
:10210000931F9F938F9384E08F9381E08F9385E556
:102110008F930E94460DEDB7FEB773963CC0809139
:10212000C801893008F4CEC02091C9013091CA019C
:102130002F5F3F4F88E0A2E6B7E0F90101900D92D2
:102140008A95E1F7D9018E910E947F2F8A83882397
:1021500019F481E0898301C01982809108018823E4
:10216000E1F321E030E03F932F93CE0102969F935D
:102170008F933F932F93CE01820F931F9F938F9343
:1021800082E08F9381E08F9387E58F930E94460DC5
:10219000EDB7FEB73B96EDBF95C0809192028823C4
:1021A00009F090C00E94686E8983823019F08430F3
:1021B00009F088C020E430E0F8948091C1008F736A
:1021C0008093C1008091C9008F738093C900809172
:1021D000C100877E8093C1008091C900877E809373
:1021E000C9008091C80087FF03C08091CE00F9CF5D
:1021F0008091C00087FF03C08091C600F9CFE091B5
:10220000C901F091CA01E081E13021F482E08093BC
:10221000BC012EC0E43611F421E830E081E0809367
:10222000BC01832F99278093CD002093CC0080910F
:10223000CD008093C5008091CC008093C400809134
:10224000CA008F7D8093CA008091CA008F7E8093E0
:10225000CA008091C9008B7F8093C9008091CA0019
:1022600084608093CA008091CA0082608093CA0013
:102270008091CA00877F8093CA008091C200877FC7
:102280008093C2008091C9008E7F8093C9008091A5
:10229000C10088618093C1008091C90088618093EA
:1022A000C9008091C10080688093C1008091C900FD
:1022B00080688093C90010926E0010926F00109297
:1022C000700078948091D60399278436910509F49B
:1022D000C3C085369105ACF48136910509F46FC011
:1022E000823691052CF48B34910509F45DC017C139
:1022F0008236910509F473C08336910509F487C0CD
:102300000EC18C36910509F4F5C08D3691054CF45B
:102310008736910509F400C18836910509F4BAC0E1
:10232000FEC08437910529F08637910509F4F0C085
:10233000F6C08091CB01A091C901B091CA01803152
:1023400040F080E1EAEBF3E00D9001928A95E1F72D
:102350000DC08D919D910D90BC91A02D8093BA03DD
:102360009093BB03A093BC03B093BD03809108017D
:102370008823E1F31F92809105018F9384E58F9369
:102380000E94460D8AEF8093C6018FEF809306016D
:1023900080EA9FE00E947B169093BE018093BD016E
:1023A0000F900F900F90BBC0E091C901F091CA014E
:1023B000808191819093900180938F01B0C0E091D2
:1023C000C901F091CA01808180930701803218F021
:1023D0008FE1809307018FEF80930601A0C0809169
:1023E000CB01843108F09BC0A091C901B091CA0112
:1023F00087E0E9EAF3E00D9001928A95E1F7809198
:10240000AD038093D00584E68093C50188C0809198
:10241000C1019091C201892B89F4E091C901F09129
:10242000CA01E081EE2351F08AE0E89FC001112447
:102430000E947B169093A6038093A503E091C901A7
:10244000F091CA0190818AE0989FC0011124909375
:10245000C2018093C10115C08FEF80930601E09106
:10246000C901F091CA0190818AE0989FC0011124AE
:102470009093C4018093C301892B19F081E080936C
:10248000D30180EA9FE00E947B169093BE01809367
:10249000BD0145C08FEF80930601E091C901F09125
:1024A000CA01908197FD08C082E08093D00110920C
:1024B000C0011092BF011AC0909580913402892BFF
:1024C0008093340291818AE0989FC00111249093F7
:1024D000C0018093BF0184E08093D00180EA9FE037
:1024E0000E947B169093BE018093BD0181E0809392
:1024F000D40115C08FEF80930601E091C901F091DE
:10250000CA0180818093350281E08093D50107C0A4
:1025100081E08093D20103C081E08093D6011092C4
:10252000CE011092CA011092C9011092C801E3E0D5
:10253000CE5F0C946F73982F8091C00085FFFCCF05
:102540009093C60008950F931F9388E18093C10074
:102550008091C00082608093C0008091C10080683B
:102560008093C1008091C10080648093C10000E02D
:1025700010E00093C5008AE290E08093C40080914F
:10258000C3019091C4010E947B169093A80380938D
:10259000A7038CED90E00E947B169093D303809369
:1025A000D20392E09093B0038AE08093B1039093BA
:1025B000B4038BE08093B2038FEF8093B8038091D4
:1025C00003018093B7030E94CF0B8093B303109352
:1025D000CA010093C9011092C8011F910F9108957B
:1025E000A0E1B0E0E6EFF2E10C94527380910801B3
:1025F000882309F494C28091BD019091BE010E948C
:102600008416882361F01092C0011092BF011092CD
:10261000C4011092C3011092C2011092C1018091B5
:10262000BF019091C001892B41F08091B00490913D
:10263000B1040E948416882329F48091D401882350
:1026400009F460C080910801882309F45BC080917F
:10265000D00104EE15E08430A8F00E94921F80E5BE
:1026600090E09F938F931F930F9381E08F938F93AD
:1026700088E48F930E94460D2DB73EB7295F3F4FE8
:102680002DBF34C0109236028CED93E09F938F9350
:1026900085E89FE19F938F93E0919503F0919603D6
:1026A000099584E190E09F938F931F930F9381E0AE
:1026B00090E09F938F9380ED91E09F938F9382E0C2
:1026C0008F9381E08F9388E48F930E94460D8091D1
:1026D000D001982F8F5F8093D0012DB73EB7215F37
:1026E0003F4F2DBF943010F01092D0018091BF0168
:1026F0009091C0010E947B169093B1048093B00426
:102700001092D4018091D501882351F18091080164
:10271000882331F10E94921F80E590E09F938F9370
:1027200084EE95E09F938F9321E030E03F932F93C9
:1027300085E291E09F938F933F932F9385E392E0FF
:102740009F938F9383E08F9381E08F938CE48F939B
:102750000E94460D1092D5018DB79EB70F968DBF82
:102760008091D2018823D1F0809108018823B1F0B3
:102770008AE090E09F938F9380EB93E09F938F93F9
:1027800081E08F938F9386E58F930E94460D109280
:10279000D2012DB73EB7295F3F4F2DBF8091D601A3
:1027A0008823D9F0809108018823B9F087E090E070
:1027B0009F938F9389EA93E09F938F9381E08F9308
:1027C000809105018F9387E48F930E94460D1092AC
:1027D000D6018DB79EB707968DBF8091C3019091AA
:1027E000C401892B41F08091A7039091A8030E9416
:1027F0008416882321F48091D301882341F18091AC
:102800000801882321F10E94043282E490E09F9322
:102810008F938EE895E09F938F9381E08F938F93B2
:1028200084E48F930E94460D1092D3012DB73EB7DA
:10283000295F3F4F2DBF8091C3019091C401009744
:1028400031F00E947B169093A8038093A703809198
:10285000C1019091C201892B09F49FC08091A50309
:102860009091A6030E948416882309F496C0809153
:102870000801882309F491C080916E0990916F0935
:1028800090939803809397038091700990917109B8
:1028900090939A03809399032091500930915109A4
:1028A0004091520950915309DA01C90163E0880F40
:1028B000991FAA1FBB1F6A95D1F7820F931FA41FF0
:1028C000B51F820F931FA41FB51F209141013091A6
:1028D00042014091430150914401BC01CD010E944D
:1028E000297330939C0320939B038091B5029091B0
:1028F000B602A091B702B091B80249E0B595A7958C
:10290000979587954A95D1F780939D038091B10261
:102910009091B202A091B302B091B40239E0B595A2
:10292000A795979587953A95D1F780939E038091C7
:10293000BD029091BE02A091BF02B091C00229E0F9
:10294000B595A795979587952A95D1F780939F037D
:102950008091D5059091D6059093A1038093A00313
:102960008EE090E09F938F9387E993E09F938F93FE
:1029700081E08F938F9383E48F930E94460D809123
:10298000C1019091C2010E947B169093A60380938F
:10299000A5038DB79EB707968DBF809107018F3F26
:1029A00079F1992704E0880F991F0A95E1F784527D
:1029B0009E4F40E150E0BC01CE0101960E9408719B
:1029C00080E190E09F938F93CE0101969F938F9328
:1029D00081E090E09F938F9387E091E09F938F93A6
:1029E00082E08F9381E08F9381E48F930E94460D64
:1029F0008FEF809307012DB73EB7255F3F4F2DBF67
:102A00008091D0058823C9F0809108018823A9F01E
:102A100081E090E09F938F9380ED95E09F938F935B
:102A200081E08F938F9382E48F930E94460D1092E2
:102A3000D0058DB79EB707968DBF8091D1018823B1
:102A4000D1F0809108018823B1F086E490E09F9353
:102A50008F9381E698E09F938F9381E08F938F937C
:102A600080E58F930E94460D1092D1012DB73EB79D
:102A7000295F3F4F2DBF8091D2039091D3030E94D5
:102A80008416882309F44BC080910801882309F437
:102A900046C08091A001882361F580916E099091D4
:102AA0006F099093CB038093CA0380917009909132
:102AB00071099093CD038093CC0380916F02809332
:102AC000CE0380916E028093CF0388E090E09F93C5
:102AD0008F938AEC93E09F938F9381E08F9383E0B1
:102AE0008F938BE68F930E94460D8DB79EB7079606
:102AF0008DBF8091D003853018F086E08093D0039D
:102B00008091E501882319F083E690E002C087EE0A
:102B100093E00E947B169093D3038093D203E4E06A
:102B2000C05F0C946E731F920F920FB60F92112418
:102B30002F933F935F936F937F938F939F93AF9365
:102B4000BF93EF93FF938091E701882329F0809151
:102B5000E70181508093E70180916503882319F094
:102B60008150809365038091EF0181508093EF0144
:102B70008F3F09F051C089E08093EF018091ED0112
:102B80009091EE0101969093EE018093ED0180917A
:102B900012018F5F817080931201882349F4809124
:102BA000EC01843028F48091EC018F5F8093EC017C
:102BB000349903C081E08093E5018091E801909110
:102BC000E901892B11F18091E8019091E9010B97BE
:102BD00050F08091E8019091E9010A979093E90102
:102BE0008093E80104C01092E9011092E8018091FD
:102BF000E8019091E90120910B0130910C018223B1
:102C00009323892B41F0479A07C08FEF9FEF909352
:102C10000C0180930B0147988091E501882309F40A
:102C20005AC02091A001222309F055C080913E098D
:102C300083FF51C086B19927FC01E071F07084FFD9
:102C400013C08091EA019091EB0101969093EB0102
:102C50008093EA018091EA019091EB01895E9340B3
:102C6000D0F12093E50137C08091EA019091EB010A
:102C7000892B69F18091EA019091EB018A5691408C
:102C800030F58091EA019091EB0169E270E00E94D9
:102C9000E0728091EA019091EB01860F971F90936B
:102CA000EB018093EA018091EA019091EB010B978F
:102CB00050F08091EA019091EB010A979093900176
:102CC00080938F0104C0F0939001E0938F011092E4
:102CD000EB011092EA01FF91EF91BF91AF919F91AB
:102CE0008F917F916F915F913F912F910F900FBEC8
:102CF0000F901F9018952091ED013091EE01280F53
:102D0000391FC901019608952091ED013091EE011E
:102D1000821B930B892F9927869580749070089554
:102D2000CF93DF930E947B16EC01CE010E948416A4
:102D30008823D9F3DF91CF910895CF93DF930E9439
:102D40007B16EC0109C080911501882329F090932E
:102D500015018FEC80937A00CE010E948416982F83
:102D6000882389F3DF91CF9108959FB7F8945F98F6
:102D70003E9A469A8091B0008F708093B000809107
:102D8000B00083608093B0008091B1008B7380931A
:102D9000B1008091B1008B608093B1001092B200BD
:102DA0008FEF8093B3008091B00080688093B00073
:102DB000809170008A7F80937000809170008260A3
:102DC000809370009FBF08958AE090E00E947B1678
:102DD0009093D2058093D10582E085BD83EB84BDBD
:102DE0008FEF88BD84EB87BD86E086BD80916E0045
:102DF000816080936E0008958091B40620916C01EB
:102E000082FF30C0909165068CE3989FB001112439
:102E10009091640680E5989FA0011124922F90580C
:102E200097FD9D5F9595959586E09802C0011124C8
:102E30002091090130910A01281B390B30930A01B6
:102E400020930901421753072CF050930A01409335
:102E5000090108952617370784F070930A016093DB
:102E600009010895822F992736E0880F991F3A9516
:102E7000E1F790930A01809309010895EF92FF9280
:102E80000F931F93CF93DF9380916C06E82FFF275A
:102E9000EB5BFE4F9681C081809111012091B606B7
:102EA000813009F01FC127FF05C0C0E0D0E0E0E09D
:102EB000F0E046C0892F992787FD9095A92FB92F5B
:102EC0002091D1023091D2024091D3025091D4028C
:102ED000BC01CD010E94B57297FF04C061587F4FBD
:102EE0008F4F9F4F7B018C0187E015950795F794D5
:102EF000E7948A95D1F78C2F992787FD9095A92F74
:102F0000B92F2091CD023091CE024091CF02509145
:102F1000D002BC01CD010E94B57297FF04C0615878
:102F20007F4F8F4F9F4FC7E0959587957795679512
:102F3000CA95D1F7F801E701C61BD70BE80BF90BCF
:102F40002091430330914403C901B3E0880F991FD6
:102F5000BA95E1F7821B930BAA2797FDA095BA2F8C
:102F6000C81BD90BEA0BFB0B80916A019927AA2792
:102F7000BB27BC01CD019E01AF010E94B57297FF36
:102F800004C061507E4F8F4F9F4FFC01EB01A9E0C1
:102F9000F595E795D795C795AA95D1F71091B40601
:102FA0006091090170910A0112FF05C07093100130
:102FB00060930F0118C040910F0150911001809152
:102FC0006B06282F3327CB01841B950BB9010E9478
:102FD000F47280910F0190911001860F971F9093CA
:102FE000100180930F0110FF14C080910F01909188
:102FF000100197FD0F9674E0959587957A95E1F706
:10300000AA2797FDA095BA2FC80FD91FEA1FFB1F4B
:1030100015C080910F019091100197FD0F9664E00B
:10302000959587956A95E1F7AA2797FDA095BA2F00
:103030008C1B9D0BAE0BBF0BFD01EC012091A0067C
:10304000222321F133278091E1019091E201829FB7
:10305000A001839F500D929F500D1124CA01AA27F1
:1030600097FDA095BA2F8C0F9D1FAE1FBF1F2F5F1E
:103070003F4F442737FD4095542FBC01CD010E949E
:1030800029733093E2012093E10104C0D093E2015F
:10309000C093E10180916406282F3327220F331F4C
:1030A000220F331F8091E1019091E2018217930773
:1030B0007CF080916506282F3327220F331F220FC3
:1030C000331F8091E1019091E2012817390724F420
:1030D0003093E2012093E101809111018F5F809391
:1030E000110102C127FF05C0C0E0D0E0E0E0F0E040
:1030F00046C0892F992787FD9095A92FB92F209138
:10310000CD023091CE024091CF025091D002BC014D
:10311000CD010E94B57297FF04C061587F4F8F4F59
:103120009F4F7B018C0197E015950795F794E794E5
:103130009A95D1F78C2F992787FD9095A92FB92FB4
:103140002091D1023091D2024091D3025091D40209
:10315000BC01CD010E94B57297FF04C061587F4F3A
:103160008F4F9F4FFC01EB0187E0F595E795D795D1
:10317000C7958A95D1F7CE0DDF1DE01FF11F809115
:1031800069019927AA27BB27BC01CD019E01AF0188
:103190000E94B57297FF04C061507E4F8F4F9F4FC2
:1031A000FC01EB01B9E0F595E795D795C795BA9580
:1031B000D1F780916B019927A6E0880F991FAA95F6
:1031C000E1F740910D0150910E0120916B063327DC
:1031D000841B950BB9010E94F47280910D019091AE
:1031E0000E01860F971F90930E0180930D01809121
:1031F000B40681FF14C080910D0190910E0197FDDE
:103200000F9674E0959587957A95E1F7AA2797FD33
:10321000A095BA2FC80FD91FEA1FFB1F15C08091B8
:103220000D0190910E0197FD0F9664E0959587959D
:103230006A95E1F7AA2797FDA095BA2F8C1B9D0BE5
:10324000AE0BBF0BFD01EC012091A106222321F161
:1032500033278091DF019091E001829FA001839F3D
:10326000500D929F500D1124CA01AA2797FDA095D9
:10327000BA2F8C0F9D1FAE1FBF1F2F5F3F4F4427DC
:1032800037FD4095542FBC01CD010E942973309326
:10329000E0012093DF0104C0D093E001C093DF017F
:1032A00080916806282F3327220F331F220F331FE8
:1032B0008091DF019091E001821793077CF080916B
:1032C0006906282F3327220F331F220F331F8091C7
:1032D000DF019091E0012817390724F43093E001D1
:1032E0002093DF0110921101E6E0CDB7DEB70C9418
:1032F0006C731F920F920FB60F9211242F933F936E
:103300004F935F938F939F93EF93FF938091F0017F
:10331000882309F0FEC08091B00086FFC4C0809170
:10332000B0008F7B8093B0003091F30120916A064A
:103330003323D9F433278DED96E0289FA001299FF0
:10334000500D389F500D1124CA012091F101309188
:10335000F201821B930B9093E4018093E30110929E
:10336000F2011092F101469AD1C0231738F48AE095
:1033700090E09093E4018093E301C8C089EA93E070
:103380009093E4018093E30180915002882389F0B7
:10339000363078F4E32FFF27EB55F94F80818823EF
:1033A00041F09927880F991F880F991F87559E4FC5
:1033B0004DC0832F99278330910529F184309105E1
:1033C00034F48130910549F0029781F02FC08430A8
:1033D0009105E1F00597E9F029C08091E301909112
:1033E000E4012091E1013091E20108C08091E30104
:1033F0009091E4012091DF013091E001820F931F51
:103400008050924023C08091120905C08091F3083A
:1034100002C080911B09282F3327220F331F220F50
:10342000331F8091E3019091E401E8CFE32FFF2760
:10343000EE0FFF1FEF59F74F20813181220F331F0D
:103440008091E3019091E401820F931F9093E40136
:103450008093E3018091E3019091E40155E08D3D7B
:10346000950718F08CED95E005C08757914030F432
:1034700087E791E09093E4018093E3012091E301D9
:103480003091E4012C5B30403093E4012093E30160
:103490008091F1019091F201820F931F9093F201BC
:1034A0008093F10133C08091B00080648093B000BC
:1034B0008CEB90E09093E4018093E3018091F10123
:1034C0009091F20184549F4F9093F2018093F10107
:1034D0008091E601882321F48091E601823011F485
:1034E000469801C0469A8091F3018F5F8093F30163
:1034F000282F332780916A06992701968217930710
:103500002CF481E0809311011092F30181E080930B
:10351000F0012091E3013091E40141E02F373407BD
:1035200030F08FEF8093B3002F5F30400FC02F3FFC
:103530003105C9F0C0F0A9014F5F50404F37510528
:1035400050F480E88093B300205830403093E40179
:103550002093E30112C08FEF8093B3005093E401F6
:103560004093E3010AC08091E3018093B30010927D
:10357000E4011092E3011092F001FF91EF919F910D
:103580008F915F914F913F912F910F900FBE0F90B0
:103590001F90189510927C008FEC80937A0008950C
:1035A00080915702609113017091140120910402DF
:1035B000882379F0CB01AA27BB27332727FD309535
:1035C000432F532FBC01CD010E94B572DC01CB010A
:1035D00016C084E0660F771F8A95E1F7CB01AA2712
:1035E000BB27332727FD3095432F532FBC01CD0137
:1035F0000E94B572DC01CB010497A109B109809347
:10360000FC019093FD01A093FE01B093FF0108958A
:10361000CF93DF93109204020E94D01A83E090E0CF
:103620000E94EF28C82FDD27C03FD10508F42A9655
:10363000C7BD8C2F809588BD86E990E00E949D16BD
:103640008091190190911A018152934010F0C0EFBE
:10365000D0E0C630D10510F1C7BD8C2F809588BD54
:1036600084E690E00E949D1681EF93E09F938F93F4
:103670008BE992E19F938F93E0919503F0919603EC
:1036800009958091190190911A010F900F900F9058
:103690000F908152934010F42197DBCFC093E10546
:1036A0006C2F83E090E00E94F7288091420680FF13
:1036B0000AC08091E1058A508C3D28F08091B503C5
:1036C00080648093B5038CE291E00E949D16DF91A7
:1036D000CF9108951F920F920FB60F9211242F933E
:1036E0003F934F935F936F937F938F939F93AF938A
:1036F000BF93CF93DF93EF93FF9380911C02282F0A
:103700003327442755278F5F80931C02F90122310C
:10371000310508F0CEC3E25CFF4F0C947B738091BF
:1037200078009091790046C080917800909179005E
:103730007BC18091780090917900909320028093D2
:103740001F028BC18091DB029091DC0220917800F6
:1037500030917900821B930B9093D4058093D3050D
:103760008091D3059091D40590932A0280932902E9
:1037700092C180917800909179002091DD02309182
:10378000DE02821B930B9093E0058093DF0580910E
:10379000DF059091E00590932C0280932B028BC360
:1037A0008091230290912402209178003091790039
:1037B000820F931F909324028093230281E07CC3A5
:1037C000809121029091220220917800309179001D
:1037D000820F931F909322028093210284E06CC396
:1037E0008091320290913302892B91F420917800DC
:1037F00030917900C901E3E0880F991FEA95E1F75C
:10380000820F931F820F931F909333028093320293
:103810002091780030917900C90173E0880F991FD9
:103820007A95E1F7820F931F820F931F2091320246
:10383000309133028217930718F02E5F3F4F02C07A
:103840002250304030933302209332028091320272
:10385000909133026FE170E00E94E0727093240156
:103860006093230185E028C38091780090917900CE
:103870009093D6058093D5058091D5059091D60576
:103880004091D7025091D802841B950B2091D6020B
:10389000332727FD3095821B930B90930A02809368
:1038A000090280915702882309F06DC080910902B6
:1038B00090910A0202977CF122E04E3E52070CF0F2
:1038C00062C020911D0230911E022B5F3F4F30934A
:1038D0001E0220931D02255030408091610290917C
:1038E0006202845F914030F4215F3F4F30931E02AB
:1038F00020931D0280911D0290911E028536910534
:103900000CF441C04F5F5F4F5093D8024093D702F1
:103910008456904034C08091090290910A028F5FD2
:103920009F4F8CF562E0473256076CF120911D02E3
:1039300030911E022550304030931E0220931D020C
:103940002B5F3F4F8091610290916202845F9140B2
:1039500030F42F50304030931E0220931D0280918E
:103960001D0290911E022FEF8C39920764F4415092
:1039700050405093D8024093D7028C599F4F909358
:103980001E0280931D028091090290910A029C01FF
:10399000442737FD4095542F8091AD029091AE029F
:1039A000A091AF02B091B002820F931FA41FB51F68
:1039B0008093AD029093AE02A093AF02B093B00299
:1039C0002091AD023091AE024091AF025091B00211
:1039D00057FF04C021503C4F4F4F5F4F6AE0559551
:1039E0004795379527956A95D1F78091AD029091CB
:1039F000AE02A091AF02B091B002821B930BA40B58
:103A0000B50B8093AD029093AE02A093AF02B0933A
:103A1000B002F5C08091210290912202209178009D
:103A200030917900820F931F90932202809321029C
:103A300010921B0243C2209178003091790080914E
:103A40001F0290912002280F391F8FEF97E0821BF1
:103A5000930B9093100280930F0286E02DC2809109
:103A6000DB029091DC022091780030917900821B7A
:103A7000930B9093D4058093D3058091D3059091B7
:103A8000D4052091290230912A02820F931F90932E
:103A90000E0280930D0287E00FC280917800909112
:103AA00079002091DD023091DE02821B930B90930E
:103AB000E0058093DF058091DF059091E00520917E
:103AC0002B0230912C02820F931F90930C02809353
:103AD0000B02F1C1209123023091240280917800E1
:103AE00090917900280F391F220F331F220F331FA7
:103AF0003093240220932302C90137FD079643E047
:103B0000959587954A95E1F7909314028093130257
:103B10008091250290912602820F931F97FD0196B6
:103B20009595879590932602809325022091ED022A
:103B30003091EE02821B930B90932201809321011E
:103B40002091190230911A02809121019091220155
:103B5000280F391F37FF02C02F5F3F4F359527953C
:103B600030931A022093190229CE2091210230911C
:103B700022028091780090917900280F391F220F3E
:103B8000331F220F331F3093220220932102C901D9
:103B900037FD0796F3E095958795FA95E1F79093B1
:103BA0001202809311028091270290912802820FC5
:103BB000931F97FD01969595879590932802809382
:103BC00027022091EB023091EC02821B930B909321
:103BD000200180931F0120911702309118028091DB
:103BE0001F0190912001280F391F37FF02C02F5F5E
:103BF0003F4F35952795309318022093170283E0A5
:103C00005BC110921C0281E080931501809100023B
:103C1000909101020196909301028093000280919D
:103C200078009091790090931A0180931901809106
:103C3000190190911A01AA27BB27C0912D02D0919A
:103C40002E02E0912F02F0913002C80FD91FEA1F17
:103C5000FB1FC0932D02D0932E02E0932F02F0930E
:103C60003002809131028F5F80933102803108F4FD
:103C700022C180911B0190911C01A0911D01B09166
:103C80001E019C01AD0163E0220F331F441F551F2D
:103C90006A95D1F7281B390B4A0B5B0B2C0F3D1F84
:103CA0004E1F5F1F8091FC019091FD01A091FE01CC
:103CB000B091FF01281B390B4A0B5B0B57FF04C067
:103CC000295F3F4F4F4F5F4F93E05595479537958D
:103CD00027959A95D1F720931B0130931C014093AF
:103CE0001D0150931E01C091D705D091D805E091D8
:103CF000D905F091DA0580911B0190911C01A091EA
:103D00001D01B0911E01C81BD90BEA0BFB0BC09320
:103D1000F401D093F501E093F601F093F7012091BF
:103D2000050230910602409107025091080257FFA8
:103D300004C0215F3F4F4F4F5F4F84E0559547953B
:103D4000379527958A95D1F78091050290910602C3
:103D5000A0910702B0910802821B930BA40BB50B34
:103D60008093050290930602A0930702B093080285
:103D70008091050290910602A0910702B09108027D
:103D80008C0F9D1FAE1FBF1F8093050290930602EC
:103D9000A0930702B0930802809105029091060259
:103DA000A0910702B0910802B7FF03C00F96A11DB2
:103DB000B11DC4E0B595A79597958795CA95D1F79C
:103DC0002091F4013091F501281B390B64E021307A
:103DD00036071CF020E034E006C08CEF20303807B6
:103DE00014F420E03CEF8091020290910302809154
:103DF00002029091030297FF03C0909581959F4F17
:103E0000A901F3E0440F551FFA95E1F78D5B92404D
:103E1000C4F080910202909103029C01E4E0220F21
:103E2000331FEA95E1F7281B390B240F351F37FFA5
:103E300002C0215F3F4F74E0359527957A95E1F7F1
:103E400017C080910202909103029C0165E0220F4D
:103E5000331F6A95E1F7281B390B240F351F37FFF5
:103E600002C0215E3F4F45E0359527954A95E1F721
:103E7000309303022093020280912D0290912E0232
:103E8000A0912F02B0913002B7FF03C00196A11D8F
:103E9000B11DB595A7959795879580932D02909321
:103EA0002E02A0932F02B093300288E0809331025B
:103EB00002C010921C0282E080931B0280911B02C0
:103EC00080937C0080911C02882319F08FEC8093F2
:103ED0007A00FF91EF91DF91CF91BF91AF919F91C8
:103EE0008F917F916F915F914F913F912F910F90A3
:103EF0000FBE0F901F90189590E2E4EEF5E08FE46E
:103F00009193815087FFFCCF0895909136029035B0
:103F100040F4E92FFF27EC51FA4F80839F5F909385
:103F200036020895CF92DF92FF920F931F93CF93A3
:103F3000DF9380913702882321F52091340220FFFE
:103F40000AC080913502882311F0815002C080910F
:103F500025018093350221FF0CC09091350280919C
:103F60002501981719F41092350203C09F5F9093B2
:103F70003502822F992780FF04C081FF02C0109272
:103F800035020E947C1F80913502282F332745E897
:103F90005FE1E0919503F09196038A3090F481E11E
:103FA000809336023F932F9383EF93E09F938F93F9
:103FB0005F934F9309952DB73EB72A5F3F4F2DBFB3
:103FC00010C080E1809336023F932F9388EF93E0F7
:103FD0009F938F935F934F9309958DB79EB70696E6
:103FE0008DBF20913502822F9927AA27BB27FC017C
:103FF0000D9708F0D9C6E05BFF4F0C947B731092CD
:1040000036028DEF93E09F938F93C5E8DFE1DF9356
:10401000CF93E0919503F0919603099584E1809305
:1040200036020F900F900F900F9083E690E09F93D1
:104030008F938AE090E09F938F9382E090E09F932C
:104040008F93809103016AE00E94D472892F99278F
:104050009F938F93809103010E94D47299279F931D
:104060008F938DE094E09F938F93DF93CF93E091B4
:104070009503F0919603099588E280933602EDB797
:10408000FEB73E96EDBF85EC96E09F938F938091AF
:10409000010199279F938F9385E294E09F938F93DB
:1040A000DF93CF93E0919503F0919603099580916A
:1040B0005E022DB73EB7285F3F4F2DBF81FF12C074
:1040C00088E3809336028FE294E09F938F93DF938F
:1040D000CF93E0919503F091960309950F900F907F
:1040E0000F900F908091B60384FF06C08CE38093FD
:1040F000360284E394E051C49091B503992351F0C2
:104100008CE380933602892F99279F938F9381E4C4
:1041100094E044C090913F02992351F08CE3809346
:104120003602892F99279F938F9388E594E028C1C1
:1041300090914A039923C1F08CE380933602892F32
:1041400099279F938F938EE694E09F938F93DF93AD
:10415000CF93E0919503F091960309952DB73EB763
:104160002A5F3F4F2DBF29C68091390190913A01B6
:10417000069730F48CE3809336028FE794E00DC409
:104180009091E6099E3108F018C68CE380933602C0
:10419000892F99279F938F938CE894E09F938F9317
:1041A000DF93CF93E0919503F091960309958DB736
:1041B0009EB7069638C51092360280918D02909176
:1041C0008E02A0918F02B0919002BC01CD0125E03A
:1041D00030E040E050E00E9429733F932F9380EA43
:1041E00094E09F938F9305E81FE11F930F93E09155
:1041F0009503F0919603099584E180933602EDB71B
:10420000FEB73696EDBF8091890290918A02A09107
:104210008B02B0918C02BC01CD0125E030E040E082
:1042200050E00E9429733F932F938DEA94E09F936F
:104230008F931F930F93E0919503F0919603099547
:1042400088E2809336022DB73EB72A5F3F4F2DBFDD
:104250008091190190911A019F938F938AEB94E0BA
:104260009F938F931F930F93E0919503F091960383
:1042700009958CE3809336028DB79EB706968DBF65
:1042800087B599279F938F9387EC94E09F938F93A3
:104290001F930F9379C01092360284ED94E09F93A0
:1042A0008F93C5E8DFE1DF93CF93E0919503F09121
:1042B0009603099584E1809336020F900F900F903A
:1042C0000F908091D1029091D202A091D302B0912F
:1042D000D402B7FF04C081509C4FAF4FBF4F1AE0CC
:1042E000B595A795979587951A95D1F7BF93AF93F5
:1042F0009F938F9381EE94E09F938F93DF93CF935F
:10430000E0919503F0919603099588E28093360237
:104310002DB73EB7285F3F4F2DBF8091CD029091C2
:10432000CE02A091CF02B091D002B7FF04C081505D
:104330009C4FAF4FBF4FFAE0B595A79597958795DE
:10434000FA95D1F7BF93AF939F938F9380EF94E04B
:104350009F938F93DF93CF93E0919503F091960312
:1043600009958CE3809336028DB79EB708968DBF72
:1043700080914709909148099F938F938FEF94E024
:104380009F938F93DF93CF93E0919503F0919603E2
:10439000099590C3E1E0FE2EC1E0D0E003E618E00D
:1043A0009F2D969584E1989FC00111248093360239
:1043B000F801828193819F938F932196DF93CF930E
:1043C0002197808191819F938F93DF93CF938EE08C
:1043D00095E09F938F9385E89FE19F938F93E09162
:1043E0009503F091960309952DB73EB7245F3F4F93
:1043F0002DBF32E0F30E22960C5F1F4F88E08F1521
:1044000078F6DBC41092360280915C0890915D08CA
:104410009F938F9380915F08909160089F938F93F3
:1044200080E295E09F938F9305E81FE11F930F9320
:10443000E0919503F0919603099584E1809336020B
:10444000EDB7FEB73896EDBF80915A0890915B08A2
:104450009F938F938091A7089091A80881589F4FB0
:104460009F938F9380E395E09F938F931F930F9378
:10447000E0919503F0919603099588E280933602C6
:104480002DB73EB7285F3F4F2DBF80913B06E82FE9
:10449000FF27EE0FFF1FEF59F74F80819181815861
:1044A0009F4F9F938F9380913A06E82FFF27EE0F3F
:1044B000FF1FEF59F74F8081918181589F4F9F9344
:1044C0008F9380E495E09F938F931F930F93E091D8
:1044D0009503F091960309958CE3809336028DB78E
:1044E0009EB708968DBF80913D06E82FFF27EE0FFF
:1044F000FF1FEF59F74F8081918181589F4F9F9304
:104500008F9380913C06E82FFF27EE0FFF1FEF5996
:10451000F74F8081918181589F4F9F938F9380E5C2
:1045200095E09F938F931F930F93E0919503F091E4
:104530009603099590C01092360280E695E09F930D
:104540008F93C5E8DFE1DF93CF93E0919503F0917E
:104550009603099584E1809336020F900F900F9097
:104560000F908091ED029091EE029F938F93209196
:10457000ED023091EE0237FF02C0295F3F4F73E03A
:10458000359527957A95E1F7809113029091140261
:10459000821B930B9F938F938EE695E09F938F934F
:1045A000DF93CF93E0919503F0919603099588E20C
:1045B000809336022DB73EB7285F3F4F2DBF8091C5
:1045C000EB029091EC029F938F932091EB0230913C
:1045D000EC0237FF02C0295F3F4F63E03595279516
:1045E0006A95E1F78091110290911202821B930B60
:1045F0009F938F938DE795E09F938F93DF93CF9356
:10460000E0919503F091960309958CE3809336022F
:104610008DB79EB708968DBF8091E9029091EA020E
:104620009F938F938091E9029091EA0220910F026B
:1046300030911002821B930B9F938F938CE895E02F
:104640009F938F93DF93CF93E0919503F09196031F
:10465000099510923802EDB7FEB738962EC28091B8
:1046600038029927009721F0019709F479C0A3C176
:10467000109236028BE995E09F938F9305E81FE136
:104680001F930F93E0919503F0919603099584E1B0
:10469000809336020F900F900F900F908091DD0263
:1046A0009091DE029F938F9380910B0290910C0268
:1046B0009F938F9388EA95E09F938F931F930F9317
:1046C000E0919503F0919603099588E28093360274
:1046D0002DB73EB7285F3F4F2DBF8091DB029091F1
:1046E000DC029F938F9380910D0290910E029F9315
:1046F0008F9387EB95E09F938F931F930F93E09198
:104700009503F091960309958CE3809336028DB75B
:104710009EB708968DBF8091D7029091D8029F9343
:104720008F938091090290910A029F938F9386EC58
:1047300095E09F938F931F930F93E0919503F091D2
:104740009603099580913402EDB7FEB73896EDBF18
:1047500083FF1BC1809138028F5F8093380215C19F
:10476000109236028AED95E09F938F93C5E8DFE1C2
:10477000DF93CF93E0919503F0919603099584E13F
:10478000809336020F900F900F900F908091DD0272
:104790009091DE029F938F938091DB029091DC02D7
:1047A0009F938F9387EE95E09F938F93DF93CF93A3
:1047B000E0919503F091960309952DB73EB7285FD8
:1047C0003F4F2DBF80915F0890916008892B31F495
:1047D00080915C0890915D08892BF1F088E28093CC
:1047E000360280915C0890915D089F938F93809131
:1047F0005F08909160089F938F938BEF95E09F9354
:104800008F93DF93CF93E0919503F09196030995F1
:104810008DB79EB708968DBF8091600280FF7BC0E8
:1048200080919201803229F08F3219F08D3209F097
:1048300072C041E04093370280917906882319F4D1
:1048400086E08093790680913402282F332720FF59
:104850000BC08091DB029091DC0201979093DC0207
:104860008093DB024093390221FF0BC08091DB0271
:104870009091DC0201969093DC028093DB024093DE
:10488000390222FF0BC08091DD029091DE02019778
:104890009093DE028093DD024093390223FF0BC028
:1048A0008091DD029091DE0201969093DE0280936A
:1048B000DD02409339028DE0809336028EE096E06F
:1048C0009F938F93DF93CF93E0919503F09196039D
:1048D00009950F900F900F900F9080913902E09101
:1048E0009503F0919603882351F08CE38093360270
:1048F00082E196E09F938F93DF93CF9356C08CE332
:104900008093360283E296E09F938F9385E89FE140
:104910009F938F934AC08DE08093360288E396E0A0
:104920009F938F93DF93CF93E0919503F09196033C
:10493000099510923702809160020F900F900F90AE
:104940000F9080FD25C080913902882309F18CE306
:10495000809336028CE396E09F938F93DF93CF93FF
:10496000E0919503F09196030995809134020F90A0
:104970000F900F900F9082FF04C00E94A7331092F7
:1049800038028091340283FF18C21092390215C296
:104990008CE38093360280E596E09F938F93DF93BC
:1049A000CF93E0919503F091960309950F900F90A6
:1049B0000F900F9002C210923802FFC1109236027F
:1049C00080912301909124016AE070E00E94F472CA
:1049D0009F938F9380912301909124016AE070E06E
:1049E0000E94F4727F936F9381E696E09F938F937A
:1049F00005E81FE11F930F93E0919503F091960353
:104A0000099584E180933602EDB7FEB73896EDBF85
:104A10008091E0099091E1096AE070E00E94E07203
:104A20009F938F938091E0099091E1096AE070E093
:104A30000E94E0727F936F9385E796E09F938F9338
:104A40001F930F93E0919503F0919603099588E2E7
:104A5000809336022DB73EB7285F3F4F2DBF809120
:104A6000E2099091E3099F938F9389E896E09F93E1
:104A70008F931F930F93E0919503F09196030995FF
:104A80008CE3809336028DB79EB706968DBF8091DA
:104A9000E4099091E5099F938F9389E996E09F93AC
:104AA0008F931F930F93E0919503F09196030995CF
:104AB00010923802EDB7FEB73696EDBF7EC1109268
:104AC00036028BEA96E09F938F9305E81FE11F93D0
:104AD0000F93E0919503F0919603099588E28093F6
:104AE00036020F900F900F900F90809193029927AC
:104AF0009F938F9384EB96E09F938F931F930F93D5
:104B0000E0919503F091960309958CE3809336022A
:104B10002DB73EB72A5F3F4F2DBF80915E08992782
:104B200001979F938F9384EC96E09F938F931F93AD
:104B30000F9338CB1092360284ED96E09F938F93BB
:104B400005E81FE11F930F93E0919503F091960301
:104B5000099584E1809336020F900F900F900F908B
:104B6000809102016AE00E94D472892F99279F9355
:104B70008F93809102010E94D47299279F938F9303
:104B800084EE96E09F938F931F930F93E09195038C
:104B9000F0919603099588E280933602EDB7FEB74F
:104BA0003896EDBF8091B8016AE00E94D472892FD7
:104BB00099279F938F938091B8010E94D47299276F
:104BC0009F938F9382EF96E09F938F931F930F9302
:104BD000E0919503F091960309958CE3809336025A
:104BE0002DB73EB7285F3F4F2DBF8091B9016AE0D6
:104BF0000E94D472892F99279F938F938091B90136
:104C00000E94D47299279F938F9380E097E09F939F
:104C10008F931F930F93E0919503F091960309955D
:104C20008DB79EB708968DBFC8C054E9C52E52E017
:104C3000D52E20E030E0E90143E0F42EC0933602A7
:104C4000F60181916F0199279F938F9389010F5FDF
:104C50001F4F1F930F938EE097E09F938F9385E8EC
:104C60009FE19F938F93E0919503F09196030995AF
:104C70002DB73EB7285F3F4F2DBFFA946496980139
:104C8000F7FEDCCF9AC098E9C92E92E0D92EC0E099
:104C9000D0E08E0183E0F82E00933602F601819178
:104CA0006F0199279F938F932596DF93CF938BE185
:104CB00097E09F938F9385E89FE19F938F93E09177
:104CC0009503F091960309952DB73EB7285F3F4FA6
:104CD0002DBFFA940C5E1F4F2497F7FEDDCF6DC0F9
:104CE0001092360288E297E09F938F9305E81FE1C8
:104CF0001F930F93E0919503F0919603099584E13A
:104D0000809336020F900F900F900F908091B40116
:104D10009091B5019F938F9386E397E09F938F9334
:104D20001F930F93E0919503F0919603099588E204
:104D3000809336028DB79EB706968DBF8091B601DF
:104D40009091B7019F938F9383E497E09F938F9304
:104D50001F930F93E0919503F0919603099589E4D1
:104D600080933602EDB7FEB73696EDBF80E597E04B
:104D70009F938F931F930F93E0919503F091960368
:104D80000995809134020F900F900F900F9083FF40
:104D900014C01092B7011092B60160E070E08EE08E
:104DA00090E00E94082909C080912501281719F474
:104DB0002150209325011092350210923402DF9188
:104DC000CF911F910F91FF90DF90CF900895F999A7
:104DD000FECF92BD81BDF89A80B599270895F999C3
:104DE000FECF1FBA92BD81BD60BD0FB6F894FA9A8E
:104DF000F99A0FBE08954AEA20E030E026173707F7
:104E000040F4FC018191480F2F5F3F4F2617370771
:104E1000C8F3842F99270895EAEA40E050E0461746
:104E2000570778F49C01F999FECF32BD21BDF89A5D
:104E300080B5E80F4F5F5F4F2F5F3F4F4617570713
:104E400090F38E2F9927089581E08093380682E0B1
:104E50008093370683E08093360684E0809339069A
:104E600085E080933A0686E080933B0687E0809356
:104E70003C0688E080933D0689E080933E068AE008
:104E800080933F068BE0809340068CE08093410640
:104E9000089589E6809335069CE0E7EBF6E0892FDC
:104EA00011928A95E9F78AE0809355061092790667
:104EB0008BE1809351068EE480937606809377068B
:104EC000B0E2B09378061092B3068AE68093420669
:104ED00082E78093B50680E58093B60684E08093F0
:104EE0005C0610929A061092970678E070934F062F
:104EF00026EE2093500680E48093520685E080934E
:104F00004506FEE1F09343068EE680934A068FE065
:104F100080934606F0934406109248067093490623
:104F200010924B0610929D06809347061092AB0696
:104F30009093AC0610925E0610925F061092600687
:104F40001092610610927B0610927C0610927D06EC
:104F500010927E0690E89093620642E340936306C7
:104F6000A2E0A093B40688E18093640620936506CE
:104F700083E080936A065DE750936D0650936E065A
:104F800050936F0690936606E5E5E093670666E446
:104F9000609368068CED809369068CE380936B06C2
:104FA00010926C069AEA90937F068CEC80938106AF
:104FB000109283069093840698E2909380069093D3
:104FC0008206109285061092B0064093B106409377
:104FD00070062AE5209371064093720636E03093FE
:104FE000860684E680938706809388062093890648
:104FF00088E780938A0690938E068BE480938B06D5
:10500000E0938C0680938D0630938F067093900604
:10501000409391068AE28093920610929306109232
:1050200096069CE890939406A09395061092980695
:105030001092990681E480935A0620935B061092A1
:105040009B0610929C0686E980939E0650937306F9
:1050500084E38093740610929F061092A00610922B
:10506000A1069093A2066093A3069093A406609372
:10507000A5061092A6061092A7061092A8061092F6
:10508000A9061092AA061092AD06B09359068FE1B8
:105090008093AF06F093AE0680EF8093B20608953A
:1050A0000E9449278AE080934C0680E180934D0658
:1050B00026E020934E069AE59093530688E7809366
:1050C000540690935606809357062093580680E224
:1050D00080935D068CE3809375068BE480937A065B
:1050E00086E491E6A3E7B4E78093B7069093B80609
:1050F000A093B906B093BA066EE870E085E396E037
:105100000E94FB268093C3060895CF93DF930E94ED
:10511000492788E080934C0630E130934D0626E025
:1051200020934E0694E69093530688E780935406A6
:1051300090935606809357062093580630935D0649
:1051400086E48093750680937A06A7EBB6E085E047
:10515000E6E2F1E0ED01019009928A95E1F76EE84F
:1051600070E0CD01825890400E94FB268093C306D8
:10517000DF91CF9108950E94492726E020934C06A5
:105180008AE080934D0684E080934E0694E69093E7
:10519000530688E7809354069093560680935706EB
:1051A0002093580680E180935D0686E4809375061F
:1051B00080937A0685E491E6A3E7B9E78093B70682
:1051C0009093B806A093B906B093BA066EE870E063
:1051D00085E396E00E94FB268093C3060895F99923
:1051E000FECF92BD81BDF89A80B599270895F999AF
:1051F000FECF1FBA92BD81BD60BD0FB6F894FA9A7A
:10520000F99A0FBE089567EE76E20E944371089501
:105210004FEE56E20E947D710895EF92FF920F9338
:105220001F93CF93C82F8150853008F0C3E08FE8DB
:10523000C89F8001112485EDE82E8FEFF82EE00E37
:10524000F11E6EE870E0C7010E940C27682F9801DC
:105250002D593F4F8FB39927AC014270507081FD9B
:10526000F9CF32BD21BDF89A80B5861711F0CA0179
:1052700027C08FB399279C012270307081FDF9CF30
:10528000F2BCE1BCF89A80B5893611F0C90118C0AA
:105290008FE8C89FC00111248B9727EE36E24FE8B4
:1052A00050E0BC0185E396E00E941E710E94F76306
:1052B0008091B2068E3B10F41092B20681E090E02D
:1052C000CF911F910F91FF90EF900895282F863076
:1052D00010F025E003C0882309F421E020930101A8
:1052E000F999FECF1FBA82E090E092BD81BD20BD4A
:1052F0000FB6F894FA9AF99A0FBE0895CF93C82F73
:1053000080913506893609F04FC0C63010F0C5E0EF
:1053100003C0CC2309F448C00E9417708091B606E0
:1053200082FF07C080915A06843618F080E580938A
:105330005A066EE870E085E396E00E94FB268093B3
:10534000C3068FE8C89FC00111242FEE36E24FE854
:1053500050E065E376E08B970E945B712FEE36E2BA
:105360004CE050E066E376E080E590E00E945B71FF
:105370006CE070E086E396E00E94FB26282FF99906
:10538000FECF1FBA8CE590E092BD81BD20BD0FB667
:10539000F894FA9AF99A0FBE8C2F0E9466290E94FF
:1053A000F76381E090E002C080E090E0CF91089543
:1053B0006DE470E088EE93E00E940C27482F8FB3D5
:1053C00099279C012270307081FDF9CF85E394E02C
:1053D00092BD81BDF89A80B5841779F48FB399276F
:1053E0009C012270307081FDF9CF88EE93E092BD70
:1053F00081BDF89A80B5813011F0C901089527EE7A
:1054000036E24EE450E068EE73E084EC96E00E94F1
:105410001E7181E090E008958091C4068130A9F466
:105420006DE470E084EC96E00E94FB268093110707
:105430002FEE36E24EE450E064EC76E088EE93E046
:105440000E945B7181E090E0089580E090E0089513
:10545000CF93DF9381E08093C406E4ECF6E08FE025
:10546000158616861786108A8150349687FFF8CFE6
:1054700080E48093D1068093D2061092D306809365
:10548000D4068093D50690EC9093D6061092D7065A
:105490008093D8068093D9061092DA069093DB06A3
:1054A0009093DC068093DD061092DE068093DF0683
:1054B0009093E006A5ECB6E08CE0ECE2F1E0ED01C3
:1054C000019009928A95E1F76DE470E0CD010197B2
:1054D0000E94FB2680931107DF91CF910895F999DF
:1054E000FECF82E090E092BD81BDF89A80B5282F72
:1054F000863078F023E0322FF999FECF1FBA82E090
:1055000090E092BD81BD30BD0FB6F894FA9AF99A39
:105510000FBE20930101822F992708951F93CF93E7
:10552000C82F162F863010F0C5E003C0882309F479
:10553000C1E08C2F99278230910541F0833091058D
:1055400044F4019731F40E94502805C00E94852838
:1055500002C00E94BB281123E1F06CE070E080E5FE
:1055600090E00E940C27282FF999FECF8CE590E05F
:1055700092BD81BDF89A80B5821759F427EE36E2C4
:105580004CE050E060E570E086E396E00E941E711A
:1055900002C00E9424278C2F0E947E29CF911F9148
:1055A0000895DF92EF92FF920F931F93CF93FF2402
:1055B000DF2CEF2C81E090E00E94EF28893611F07B
:1055C00031E0E32E6CE070E080E590E00E940C2773
:1055D000C82FF999FECF8CE590E092BD81BDF89A75
:1055E00080B58C1711F421E0D22EC1E001E010E06B
:1055F000EE2029F48C2F0E940D298823B9F591E023
:10560000F92E1F930F9388E597E09F938F938BE973
:1056100092E19F938F93E0919503F0919603099502
:105620002DB73EB72A5F3F4F2DBF0130110521F046
:105630000230110521F006C00E94502805C00E94CA
:10564000852802C00E94BB28DD2059F027EE36E2F3
:105650004CE050E060E570E086E396E00E941E7149
:1056600002C00E9424278C2F0E947E29CF5F0F5FEB
:105670001F4FC63008F4BCCFFF2019F083E00E9412
:1056800066290E946F2AC82F0E940D298C2F992706
:105690009F938F938EE797E09F938F930BE912E18F
:1056A0001F930F93E0919503F0919603099581E084
:1056B00090E00E94EF282DB73EB72A5F3F4F2DBFE5
:1056C0008F3F21F00E94D829882399F487E997E039
:1056D0009F938F931F930F93E0919503F0919603FF
:1056E00009950E94282A0E940C2A0F900F900F9073
:1056F0000F90EE2029F069E681E090E00E94F72803
:105700001092340690E0E4ECF6E0CFE085851816C0
:1057100014F49F5F04C0158616861786108AC15040
:105720003496C7FFF3CF90933406892F99279F9320
:105730008F9385EC96E09F938F9388EB97E09F93F0
:105740008F931F930F93E0919503F0919603099522
:105750000E9446058DB79EB708968DBFCF911F91C9
:105760000F91FF90EF90DF900895982F2FB7F89446
:105770003998389A88B1836088B98091B9008C7F54
:105780008093B9008AE28093B8001092440210928C
:105790004202109241029923B1F0EAE6F7E08FE06D
:1057A000108211821282138214821582168217824D
:1057B00016861086118612861386148615868150E9
:1057C0003F9687FFEDCF78942FBF08951092440243
:1057D00084E98093BC0080E88093BC001092BD00F7
:1057E0001092BA001092BB001092B9001092B8004B
:1057F0001092400280E00E94B52B1092BB0085E819
:105800008093BC0080913E02826080933E020895A6
:105810001F920F920FB60F9211242F933F938F93E5
:105820009F93EF93FF9380914402282F33278F5F3C
:10583000809344022330310509F41CC12430310522
:105840005CF42130310509F452C0223031050CF0EE
:1058500097C0232B71F032C32530310509F470C194
:10586000253031050CF41EC12630310509F436C24D
:1058700025C381E08093400209C0809142028031BB
:1058800090F4809142028F5F8093420280914202A5
:10589000E82FFF27EE0FFF1FEE0FFF1FEC53F94F0E
:1058A0008585181654F7809142028F7080934202CA
:1058B00080914A028F5F80934A0290913B01981732
:1058C00070F410924A0210923D0210923C0285E060
:1058D0008093440280914102880F8D5A04C08091C8
:1058E0004202880F8E5A8093BB0085E826C18091C2
:1058F00042029927FC0124E0EE0FFF1F2A95E1F7F1
:10590000E81BF90BE659F84F81818093BB0085E8CD
:105910008093BC00809142029927FC01E295F295A8
:10592000F07FFE27E07FFE27E81BF90BE659F84FD2
:10593000808180FF9DC0809142029927FC01E29501
:10594000F295F07FFE27E07FFE27E81BF90BE65972
:10595000F84F8281882329F080913406873008F43B
:10596000C3C280913C0290913D02892B09F0BCC2D8
:1059700080913A0290913B02892B09F0B5C278C020
:105980008091420221E030E002C0220F331F8A954D
:10599000E2F780913A0290913B0228233923232B8E
:1059A00089F0809142029927FC01E295F295F07FFF
:1059B000FE27E07FFE27E81BF90BE659F84F80E150
:1059C00084830FC0809142029927FC01E295F295F1
:1059D000F07FFE27E07FFE27E81BF90BE659F84F22
:1059E0001482809142029927FC01E295F295F07FA2
:1059F000FE27E07FFE27E81BF90BE659F84F84816C
:105A0000282F3327220F331F220F331F220F331F5C
:105A1000809142029927FC0134E0EE0FFF1F3A9576
:105A2000E1F7E81BF90BE659F84F82818770822B6A
:105A30008093BB0085E88093BC002091420281E006
:105A400090E002C0880F991F2A95E2F720913C024E
:105A500030913D0282239323892B51F082E697E017
:105A6000909348028093470288E0809349023CC2A9
:105A700084E021C2E0914702F09148028191809335
:105A8000BB0085E88093BC00F0934802E093470296
:105A900080914902815080934902882309F424C2ED
:105AA00083E009C28091B900803379F58091450285
:105AB000882329F4809142028F5F80934502809170
:105AC00042029927FC01E295F295F07FFE27E07FE4
:105AD000FE27E81BF90BE659F84F838199278F774A
:105AE00090708F3791058CF4809142029927FC01C8
:105AF000E295F295F07FFE27E07FFE27E81BF90B89
:105B0000E659F84F83818F5F83831092440284E9C2
:105B10008093BC008AE090E090933A018093390131
:105B2000809142028F5F80934202109244028091E2
:105B30003E028E7F80933E0285EA8093BC00D4C1F2
:105B40008091B9008034D9F1809141029927FC01FC
:105B5000E295F295F07FFE27E07FFE27E81BF90B28
:105B6000E659F84F83818F778383809141028F5F5D
:105B700080934102809141028031A0F01092410255
:105B800010923B0210923A02809146028F5F8093FE
:105B90004602803138F01092460280913E028D7F9D
:105BA00080933E0280913E02816080933E0210927B
:105BB000440284E98093BC001092400288C0809126
:105BC00041029927FC01E295F295F07FFE27E07FE4
:105BD000FE27E81BF90BE659F84F83818068838321
:105BE000809141029927FC01E295F295F07FFE2712
:105BF000E07FFE27E81BF90BE659F84F808180FF14
:105C000042C0809141029927FC01E295F295F07F14
:105C1000FE27E07FFE27E81BF90BE659F84F848149
:105C200099270097D9F0409709F048C082E697E09D
:105C3000909348028093470288E0809349028091C4
:105C400041029927FC0134E0EE0FFF1F3A95E1F77E
:105C5000E81BF90BE659F84F148230C090914102CD
:105C60008FE0989FC00111248159984F909348026A
:105C70008093470290914102809146029817D9F48F
:105C800080913C0119C0909141028FE0989FC00122
:105C900011248159984F9093480280934702809134
:105CA0003E0281FD06C09091410280914602981704
:105CB00011F482E001C081E08093490280914902A1
:105CC000813011F485E801C085EC8093BC0080919F
:105CD000450280933F021092450206C1E0914702BF
:105CE000F09148028091BB0080838091470290919F
:105CF000480201969093480280934702809149029E
:105D0000815080934902823010F085ECD1C08130FF
:105D100011F485E8CDC080913E0281FF7DC0809165
:105D2000600280FD79C0809141029927FC0124E046
:105D3000EE0FFF1F2A95E1F7E81BF90BE659F84F24
:105D4000868199278C7F9070883F910591F480918E
:105D500041029927FC01E295F295F07FFE27E07F52
:105D6000FE27E81BF90BE659F84F8081816080839C
:105D70000FC0809141029927FC01E295F295F07FD6
:105D8000FE27E07FFE27E81BF90BE659F84F10824B
:105D9000809141029927FC01E295F295F07FFE2760
:105DA000E07FFE27E81BF90BE659F84F8681883F14
:105DB00089F4809141029927FC01E295F295F07FE8
:105DC000FE27E07FFE27E81BF90BE659F84F80819C
:105DD000866021C0809141029927FC01E295F295ED
:105DE000F07FFE27E07FFE27E81BF90BE659F84F0E
:105DF0008681893F89F4809141029927FC01E295CF
:105E0000F295F07FFE27E07FFE27E81BF90BE659AD
:105E1000F84F8081846080838091600281FF20C080
:105E2000809141029927FC0134E0EE0FFF1F3A9563
:105E3000E1F7E81BF90BE659F84F86818E3F80F4B5
:105E4000809141029927FC0124E0EE0FFF1F2A9563
:105E5000E1F7E81BF90BE659F84F86858F5F8687D7
:105E6000809141028F5F8093410280914102803195
:105E7000A0F01092410210923B0210923A028091DF
:105E800046028F5F80934602803138F010924602BE
:105E900080913E028D7F80933E021092440284E9FD
:105EA0008093BC0080913E02816080933E021AC0C4
:105EB0008093BC0086E08093440216C01092440296
:105EC00084E98093BC0080913E02816080933E0211
:105ED0008AE090E090933A01809339011092420257
:105EE0001092410210924002FF91EF919F918F9189
:105EF0003F912F910F900FBE0F901F9018950F9309
:105F00001F93CF93DF93182F80919202882321F45F
:105F10008091C601882319F081E090E091C0113191
:105F200008F08CC01123C9F0812F9927FC0144E0AF
:105F3000EE0FFF1F4A95E1F7E81BF90BE659F84F02
:105F40003C9780813C9688230CF078C03F978081F5
:105F500080FD03C083E090E073C0809162079927C1
:105F60008B709070029719F084E090E069C067E050
:105F700070E082E697E00E94FB26909169078917FE
:105F800019F085E090E05CC000913B0180E18093D6
:105F90003B0184E690E090933A01809339010E949E
:105FA0007B16EC0180913E0280FD05C0CE010E946F
:105FB00084168823B9F3112319F48FEF9FE00BC0E7
:105FC000212F33272150304081E090E002C0880F1C
:105FD000991F2A95E2F790933D0280933C0210921C
:105FE00042021092410288EE93E00E947B16EC017F
:105FF0001092440280913E028E7F80933E0285EA99
:106000008093BC0080913E0280FD05C0CE010E94BD
:1060100084168823B9F380913C0290913D02892B2C
:1060200029F0CE010E948416882311F300933B01CE
:1060300080913C0290913D02009711F082E090E047
:10604000DF91CF911F910F9108950F931F93CF93DD
:10605000DF93982F80919202882321F48091C601CA
:10606000882319F081E090E07BC09131B0F499234E
:1060700019F486E090E074C0C92FDD27FE0154E0DA
:10608000EE0FFF1F5A95E1F7EC1BFD0BE659F84F99
:106090003C9780813C9687FD03C082E090E060C021
:1060A0003F97808180FD03C083E090E059C088EE77
:1060B00093E00E947B168C0180913E0280FD05C01A
:1060C000C8010E9484168823B9F3219781E090E0EB
:1060D00002C0880F991FCA95E2F790933B02809304
:1060E0003A021092420210924102109262071092FC
:1060F00069071092440280913E028E7F80933E0297
:1061000085EA8093BC0080913E0280FD05C0C801F5
:106110000E9484168823B9F380913A0290913B0241
:10612000892B29F0C8010E948416882311F38091DD
:10613000620799278B709070029719F084E090E0C5
:106140000FC067E070E082E697E00E94FB26909126
:106150006907891719F085E090E002C080E090E0BF
:10616000DF91CF911F910F910895CF93DF9380E03E
:1061700021E83FEFC9EAD8E0E1E6F8E0DF01853049
:1061800020F411961C921E9202C031832083198242
:10619000188222968F5F12963296833280F38FE7B1
:1061A00090E09093A00880939F0881E89FEF9093E0
:1061B0009E0880939D081092A2081092A108109248
:1061C000EA021092E9021092EC021092EB02109295
:1061D000EE021092ED02DF91CF9108951F920F927F
:1061E0000FB60F9211240F931F932F933F934F934A
:1061F0005F936F937F938F939F93AF93BF93CF934F
:10620000DF93EF93FF934091860050918700809138
:106210004C0290914D02481B590B80918600909141
:10622000870090934D0280934C02CA018D54944094
:10623000A0914E02B0914F02835F9A4158F4809131
:106240004E0280935E08149714F010923F0181E093
:1062500090E0C1C0A131B1050CF0C1C0CA018B5F93
:106260009040845B914008F0B1C080913D019091D5
:106270003E01481B590BE0919F06EE2351F0FF278A
:10628000EE0FFF1FEF59F74F808191818436910502
:10629000ECF4FD01EA0FFB1FEF59F74F808191816C
:1062A000FA01E81BF90BCF01F7FF03C09095819528
:1062B0009F4F06975CF480919302883C20F4809174
:1062C0009302865F01C088EC80939302FD01EA0F80
:1062D000FB1FEF59F74F808191819C01220F331FE3
:1062E000280F391F240F351F37FF02C02D5F3F4F86
:1062F000E901D595C795D595C795CA0101968C1723
:106300009D0714F4219706C041505040C417D5078B
:106310000CF4219680919302833CD8F08D010A0FF2
:106320001B1FF801EF59F74F808191819E01281BB7
:10633000390BC90163E070E00E94F472CB01880F51
:10634000991F860F971F0755174FF8019183808378
:1063500007C0AA0FBB1FA755B74F11961C921E92DC
:10636000E0914E02F0914F02EE0FFF1FEF59F74FF1
:10637000D183C08380919302823340F580913606A9
:10638000E82FFF27EE0FFF1FEF59F74F1182108202
:1063900080913706E82FFF27EE0FFF1FEF59F74FC9
:1063A0001182108280913906E82FFF27EE0FFF1F20
:1063B000EF59F74F1182108280913806E82FFF279E
:1063C000EE0FFF1FEF59F74F1182108280914E029E
:1063D00090914F02019690934F0280934E02FF914D
:1063E000EF91DF91CF91BF91AF919F918F917F916D
:1063F0006F915F914F913F912F911F910F910F904E
:106400000FBE0F901F90189580916E0990916F09A3
:1064100090939105809390058091700990917109F6
:10642000909393058093920580914209909143093E
:1064300097FD0396959587959595879590939505E6
:1064400080939405809154099091550997FD039686
:106450009595879595958795909397058093960543
:106460008091E9029091EA0220910F02309110028E
:10647000821B930B909399058093980580918D02D0
:1064800090918E02A0918F02B0919002BC01CD013B
:106490002AE030E040E050E00E94297330939B05F1
:1064A00020939A058091D5059091D60590939D05EE
:1064B00080939C0580918F01909190019093A1050C
:1064C0008093A00580912301909124019093A305CE
:1064D0008093A2058091930299279093A5058093BC
:1064E000A4058091FB089091FC089093A7058093E8
:1064F000A60580916B0799279093A9058093A8051D
:1065000080917A0799279093AB058093AA05809193
:10651000890799279093AD058093AC0580919807E2
:1065200099279093AF058093AE058091E1019091FA
:10653000E2019093B9058093B8058091770290911C
:1065400078029093BB058093BA058091E009909101
:10655000E1099093BD058093BC058091E409909179
:10656000E5099093BF058093BE05809189029091C3
:106570008A02A0918B02B0918C02BC01CD012AE06D
:1065800030E040E050E00E9429733093C105209331
:10659000C0058091E60999279093CB058093CA05A1
:1065A00080913B0390913C039093CD058093CC0563
:1065B0008091390390913A039093CF058093CE0553
:1065C0008091B503882321F48091B603882321F0BC
:1065D00080918F05816003C080918F058E7F8093AD
:1065E0008F050895EF92FF921F93CF93DF93182F9B
:1065F0007B0180919202882371F58091030189319A
:1066000011F4299801C0299A11501F3FE9F0F09226
:10661000E901E092E801E7018091E8019091E90148
:10662000892B11F4209781F38091EC018823A1F349
:106630001092EC018091E8019091E901892B09F415
:1066400021970E942D70E8CF80910301893111F4C8
:10665000299A01C02998DF91CF911F91FF90EF9067
:106660000895EF92FF920F931F9310927A008091FA
:106670001302909114029093020980930109809172
:106680001102909112029093F7088093F60880917E
:106690000F029091100290934A098093490920912A
:1066A0000B0230910C02C901880F991F880F991FA6
:1066B000820F931F820F931F909343098093420987
:1066C00020910D0230910E02C901880F991F880F89
:1066D000991F820F931F820F931F909355098093E8
:1066E00054098FEC80937A00809176069927AA2727
:1066F000BB2744ECE42E49E0F42E012D112DBC0102
:10670000CD01A80197010E94B572DC01CB018093F5
:10671000850190938601A0938701B09388018091B1
:1067200077069927AA27BB27BC01CD010E94B57225
:10673000DC01CB018093810190938201A0938301BE
:10674000B09384011F910F91FF90EF900895809175
:10675000ED029091EE029093E4028093E302809127
:10676000EB029091EC029093E2028093E10280911F
:10677000E9029091EA029093E0028093DF02609137
:10678000DD027091DE0284E090E00E9408296091B1
:10679000DB027091DC0286E090E00E9408296091A3
:1067A000E3027091E40282E190E00E940829609186
:1067B000E1027091E20284E190E00E940829609178
:1067C000DF027091E00286E190E00E9408290895BE
:1067D000A0E0B0E0EEEEF3E30C944873782E91E085
:1067E000692EEE24FF245701470187011092B5035B
:1067F000F092DE02E092DD02F092DC02E092DB0237
:10680000F092D802E092D7021092D602F092EE02F5
:10681000E092ED02F092EC02E092EB02F092EA02DA
:10682000E092E90210926701109266011092040250
:1068300023E0821729F480915E02826080935E02D9
:106840000E94313384E690E00E949D160E9431330D
:106850008091420680FF14C08091190190911A0125
:10686000875B934058F48091190190911A018E5ED4
:10687000924020F080910402882311F00E94081BAE
:10688000C0911901D0911A0187B5865F87BD87B580
:10689000809588BD8FE1C82E8AE090E00E949D1609
:1068A00080910F0290911002E80EF91E8091130260
:1068B00090911402A80EB91E8091110290911202BB
:1068C000880E991E8091D5059091D605080F191F45
:1068D000CA94C7FEE1CF8091190190911A01825F9D
:1068E000934080F48091190190911A01459750F0DE
:1068F0008091190190911A01C81BD90BD0931401F2
:10690000C093130187B58A5087BD87B5809588BD30
:106910009501205F3F4F3695279536952795309303
:10692000EE022093ED02C4014096969587959695C8
:1069300087959093EC028093EB0240E150E0E40EE7
:10694000F51EA5E0F694E794AA95E1F7F092EA0225
:10695000E092E902040F151FF5E016950795FA95E8
:10696000E1F71093D8020093D7029093E802809346
:10697000E7023093E6022093E50252E0751629F50E
:10698000809142099091430997FF03C090958195AA
:106990009F4F6CE070E00E94F4727093DE0260938F
:1069A000DD02809154099091550997FF03C090959D
:1069B00081959F4F6CE070E00E94F4727093DC024E
:1069C0006093DB020E94A733AEC084E090E00E9497
:1069D00003299093DE028093DD0286E090E00E941E
:1069E00003299C019093DC028093DB028091DD02FD
:1069F0009091DE028150984018F421503840A0F167
:106A000089ED97E09F938F938BE992E19F938F930A
:106A1000E0919503F0919603099580914209909138
:106A2000430997FF03C0909581959F4F6CE070E0FC
:106A30000E94F4727093DE026093DD02809154092B
:106A40009091550997FF03C0909581959F4F6CE0F9
:106A500070E00E94F4727093DC026093DB026624A3
:106A60000F900F900F900F9082E190E00E94032909
:106A70009093E4028093E30284E190E00E94032972
:106A80009093E2028093E10286E190E00E94032964
:106A90009C019093E0028093DF0280915E0281FF6F
:106AA00042C04091E3025091E402CA0180509941F2
:106AB00081589C40A0F48091E1029091E20265E24D
:106AC0008138960760F469E18030960740F064E011
:106AD000213B360720F463E020323607C0F481EF13
:106AE00097E09F938F938BE992E19F938F93E0912F
:106AF0009503F09196030995662480915E028D7F3F
:106B000080935E020F900F900F900F900CC05093E7
:106B1000EE024093ED029093EC028093EB023093EF
:106B2000EA022093E90212BC11BC109202091092F1
:106B300001091092F7081092F60810924A09109273
:106B4000490988EC90E00E949D1680910B0290917B
:106B50000C029C01220F331F220F331F280F391FF5
:106B6000280F391F309343092093420980910D0269
:106B700090910E028C01000F111F000F111F080FC2
:106B8000191F080F191F109355090093540980917C
:106B90005106C82EDD24EE24FF24442737FD4095FE
:106BA000542FC701B6010E94B5724B015C0160937E
:106BB000D1027093D2028093D3029093D4029801B1
:106BC000442737FD4095542FC701B6010E94B57286
:106BD000DC01CB018093CD029093CE02A093CF0233
:106BE000B093D0028092C5029092C602A092C702D2
:106BF000B092C8028093C1029093C202A093C302D4
:106C0000B093C4021092BD021092BE021092BF0255
:106C10001092C00200918F01109190011093AC026C
:106C20000093AB028FEF9FEF90938E0180938D01C5
:106C300084E690E090938A018093890180917606A2
:106C40009927AA27BB27BC01CD0124EC39E040E0FD
:106C500050E00E94B572DC01CB018856954CAF4FD5
:106C6000BF4F8093850190938601A0938701B093D5
:106C70008801809177069927AA27BB27BC01CD01FF
:106C80000E94B572DC01CB018856954CAF4FBF4FC7
:106C90008093810190938201A0938301B09384013A
:106CA000C801AA2797FDA095BA2F209141013091E4
:106CB00042014091430150914401BC01CD010E9429
:106CC000B572DC01CB018093500990935109A093D8
:106CD0005209B09353091092A8021092A7020E9481
:106CE000F763772029F080916002846080936002CE
:106CF0008FEF8093D0091092D10980E28093D2095E
:106D000084E6809393028091E601882311F0579ADC
:106D100017C08091B406992780FF05C082FF03C089
:106D200080EE9EE202C080E091E190930A018093A0
:106D3000090181E0809311010E943E170E943E17D5
:106D400088E090E00E9403299093D8028093D702B4
:106D500012BC11BC8091ED029091EE0280569940D8
:106D6000815C9B4228F08091B50381608093B503DC
:106D70008091EB029091EC0280569940815C9B429D
:106D800028F08091B50382608093B5038091E90279
:106D90009091EA028C5291408957954028F0809159
:106DA000B50384608093B5038091DD029091DE028B
:106DB0008C529140835C914028F08091B5038860AB
:106DC0008093B5038091DB029091DC028C5291405C
:106DD000835C914028F08091B50380618093B50376
:106DE0008091D7029091D802805092408355914073
:106DF00028F08091B50380628093B5038091B5033C
:106E00008111662486E480937C0180911B0190911E
:106E10001C01A0911D01B0911E018093D705909394
:106E2000D805A093D905B093DA0510920302109209
:106E300002021092050210920602109207021092AE
:106E400008021092AD021092AE021092AF021092A0
:106E5000B0021092C9051092C8050E94D01A809104
:106E60005E0281FF07C080917906882319F484E0CF
:106E7000809379061092540310925303862D99271C
:106E8000EEE0CDB7DEB70C946473A3E1B0E0EBE4C1
:106E9000F7E30C9444738091E9029091EA02209107
:106EA0000F0230911002821B930B90934A0980933A
:106EB00049098091190290911A0297FD07969C0149
:106EC00083E0359527958A95E1F730930209209361
:106ED0000109809117029091180297FD079603E02F
:106EE000959587950A95E1F79093F7088093F608B2
:106EF00030930A09209309099093050980930409A6
:106F00008091420990914309AC01440F551F480FED
:106F1000591F20910B0230910C02C901880F991F53
:106F2000880F991F820F931F820F931F480F591FBD
:106F300057FF02C04D5F5F4F559547955595479553
:106F40005093430940934209809154099091550907
:106F5000AC01440F551F480F591F20910D0230916D
:106F60000E02C901880F991F880F991F820F931F66
:106F7000820F931F480F591F57FF02C04D5F5F4F8D
:106F80005595479555954795509355094093540904
:106F9000809113099091140920910B0230910C02F9
:106FA000820F931F909314098093130980914C09C9
:106FB00090914D0920910D0230910E02820F931F86
:106FC00090934D0980934C098091D9029091DA02F7
:106FD00001969093DA028093D9028091F401909106
:106FE000F501A091F601B091F70180938D02909385
:106FF0008E02A0938F02B09390028093F801909339
:10700000F901A093FA01B093FB018FEC80937A0011
:10701000109215012091C1023091C2024091C30229
:107020005091C40229873A874B875C8729543B4695
:10703000414050402CF028E43BE641E050E00DC0D8
:1070400089859A85AB85BC85885B9449AE4FBF4FD7
:107050004CF428EB34E94EEF5FEF2D833E834F83F2
:10706000588708C089859A85AB85BC858D839E83AA
:10707000AF83B8872091C5023091C6024091C70204
:107080005091C8022D873E874F87588B29543B4625
:10709000414050402CF028E43BE641E050E00DC078
:1070A0008D859E85AF85B889885B9449AE4FBF4F6B
:1070B0004CF428EB34E94EEF5FEF29833A834B839E
:1070C0005C8308C08D859E85AF85B88989839A8346
:1070D000AB83BC83A0914909B0914A09BB8BAA8BB1
:1070E000FD01CF01AA2797FDA095BA2FA090BD0260
:1070F000B090BE02C090BF02D090C002A80EB91ED0
:10710000CA1EDB1EA092BD02B092BE02C092BF0298
:10711000D092C002E0905009F090510900915209BC
:1071200010915309E80EF91E0A1F1B1FE092500927
:10713000F09251090093520910935309F09176028D
:10714000F98BFF2309F098C180917502882309F01B
:1071500093C180913E0986FF8FC18091F60890917E
:10716000F708AA2797FDA095BA2FBC01CD01298168
:107170003A814B815C810E94B5729B01AC0197FF03
:1071800004C02150384F4F4F5F4F6BE055954795E6
:10719000379527956A95D1F780916601682E7724F7
:1071A00088249924CA01B901A40193010E94B572EF
:1071B000DC01CB018093F9029093FA02A093FB02C9
:1071C000B093FC02B7FF04C08150904FAF4FBF4F48
:1071D0001C012D013CE055944794379427943A952F
:1071E000D1F72092F9023092FA024092FB025092BB
:1071F000FC028091010990910209AA2797FDA095B0
:10720000BA2FBC01CD012D813E814F8158850E944E
:10721000B57297FF04C06150784F8F4F9F4F2BE09E
:1072200095958795779567952A95D1F7A401930150
:107230000E94B572DC01CB018093FD029093FE02A7
:10724000A093FF02B0930003B7FF04C08150904F9A
:10725000AF4FBF4F9C01AD018CE0559547953795D9
:1072600027958A95D1F72093FD023093FE02409333
:10727000FF02509300038091F9029091FA029093DB
:10728000F0088093EF088091FD029091FE029093A8
:10729000F2088093F1082219330944095509209313
:1072A000FD023093FE024093FF0250930003E20E72
:1072B000F31E041F151FE0925009F092510900932C
:1072C000520910935309809165018823B1F457FF47
:1072D00004C02F5F3F4F4F4F5F4F559547953795F0
:1072E0002795A21AB30AC40AD50AA092BD02B09289
:1072F000BE02C092BF02D092C0022A893B897901A6
:107300000027F7FC0095102F8091FD029091FE025E
:10731000A091FF02B0910003E80EF91E0A1F1B1F87
:10732000C801B70129813A814B815C810E94B57205
:107330009B01AC0197FF04C02150384F4F4F5F4F66
:10734000BBE05595479537952795BA95D1F780912C
:107350006701A82EBB24CC24DD24CA01B901A601F3
:1073600095010E94B572DC01CB018093F1029093EC
:10737000F202A093F302B093F402B7FF04C081506D
:10738000904FAF4FBF4F3C014D01ACE095948794B7
:1073900077946794AA95D1F76092F1027092F20205
:1073A0008092F3029092F402C801B7012D813E81D0
:1073B0004F8158850E94B57297FF04C06150784F85
:1073C0008F4F9F4FFBE09595879577956795FA9539
:1073D000D1F7A60195010E94B572DC01CB01809323
:1073E000F5029093F602A093F702B093F802B7FF6C
:1073F00004C08150904FAF4FBF4FAC01BD01ECE0D6
:107400007595679557954795EA95D1F74093F5029D
:107410005093F6026093F7027093F8022A893B8931
:1074200037FF03C0309521953F4F21343105E4F1FA
:10743000D401C30197FE07C0B095A09590958195A2
:107440009F4FAF4FBF4F81389105A105B10584F41F
:10745000DB01CA0177FF07C0B095A0959095819593
:107460009F4FAF4FBF4F81389105A105B105E4F0A3
:1074700081E08093A90218C01092F2081092F108DE
:107480001092F0081092EF081092F5021092F60296
:107490001092F7021092F8021092F1021092F2028A
:1074A0001092F3021092F4028091F5029091F6028C
:1074B000A091F702B091F802BC01CD0124E630E0C2
:1074C00040E050E00E942973E090F102F090F20257
:1074D000E21AF30AF0920009E092FF088091F102AB
:1074E0009091F202A091F302B091F402BC01CD019F
:1074F00024E630E040E050E00E942973DA01C9013F
:107500002091F5023091F6028C01021B130B1093AF
:10751000F9080093F8088091410190914201A091EF
:107520004301B0914401BC01CD0128E631E040E0C7
:1075300050E00E94B572209150093091510940915C
:10754000520950915309261737074807590764F025
:10755000261B370B480B590B2093500930935109C8
:107560004093520950935309209150093091510989
:10757000409152095091530957FF0CC0260F371FF5
:10758000481F591F209350093093510940935209C5
:10759000509353098091F6089091F7088E0D9F1D26
:1075A00020917B0230917C02821B930BAA2797FDCE
:1075B000A095BA2F29853A854B855C85820F931F4C
:1075C000A41FB51F8093C1029093C202A093C3026F
:1075D000B093C402C0908101D0908201E0908301F9
:1075E000F0908401C816D906EA06FB0684F488EAFE
:1075F00091E6A0E0B0E08C199D09AE09BF09809327
:10760000C1029093C202A093C302B093C402222786
:107610003327A9012C193D094E095F098091C10248
:107620009091C202A091C302B091C4028217930745
:10763000A407B50784F488E59EE9AFEFBFEFC80E55
:10764000D91EEA1EFB1EC092C102D092C202E09275
:10765000C302F092C4028091010990910209800F47
:10766000911F2091790230917A02821B930BAA27F5
:1076700097FDA095BA2F2D853E854F855889820F9D
:10768000931FA41FB51F8093C5029093C602A093B9
:10769000C702B093C802E0908501F0908601009186
:1076A000870110918801E816F9060A071B0784F480
:1076B00088EA91E6A0E0B0E08E199F09A00BB10B1B
:1076C0008093C5029093C602A093C702B093C802EC
:1076D00022273327A9012E193F09400B510B809116
:1076E000C5029091C602A091C702B091C80282174C
:1076F0009307A407B50784F488E59EE9AFEFBFEFD1
:10770000E80EF91E0A1F1B1FE092C502F092C60286
:107710000093C7021093C8028091BD029091BE02EF
:10772000A091BF02B091C0028093C9029093CA0297
:10773000A093CB02B093CC028091C5029091C60277
:10774000A091C702B091C8028093D1029093D20257
:10775000A093D302B093D4028091C1029091C2024F
:10776000A091C302B091C4028093CD029093CE0247
:10777000A093CF02B093D002809121019091220179
:1077800097FD079633E0959587953A95E1F79093A5
:1077900002098093010980911F019091200197FDBA
:1077A000079623E0959587952A95E1F79093F7083A
:1077B0008093F60880911302909114020F9734F48D
:1077C00088E19CEF90930209809301098091130254
:1077D00090911402079734F480E398EF9093020994
:1077E000809301098091130290911402815D97406A
:1077F00034F088EE93E09093020980930109809120
:10780000130290911402805E974034F080ED97E06F
:1078100090930209809301098091110290911202C4
:107820000F9734F488E19CEF9093F7088093F60863
:107830008091110290911202079734F480E398EF3F
:107840009093F7088093F6088091110290911202AC
:10785000815D974034F088EE93E09093F708809331
:10786000F6088091110290911202805E974034F0E8
:1078700080ED97E09093F7088093F608609174018B
:10788000662309F4AFC040912101509122018091FB
:10789000010390910203481B590B50930803409336
:1078A00007032091210130912201280F391F37FF52
:1078B00002C02F5F3F4F35952795309302032093E9
:1078C0000103413851051CF080E890E005C04058A4
:1078D0005F4F34F480E89FEF909308038093070391
:1078E00040911F0150912001809103039091040366
:1078F000481B590B509306034093050320911F0129
:1079000030912001280F391F37FF02C02F5F3F4FF2
:10791000359527953093040320930303413851058F
:107920001CF080E890E005C040585F4F34F480E8D8
:107930009FEF9093060380930503462F5527809170
:10794000070390910803849FB001859F700D949F59
:10795000700D11249B0177FF02C0215F3F4FB4E0FF
:1079600035952795BA95E1F7809101099091020923
:10797000820F931F90930209809301098091050360
:1079800090910603849FD001859FB00D949FB00D08
:107990001124AD019D01B7FF02C0215F3F4FA4E05C
:1079A00035952795AA95E1F78091F6089091F7080B
:1079B000820F931F9093F7088093F608809121011E
:1079C00090912201860F971F9093220180932101AD
:1079D00080911F0190912001840F951F90932001A9
:1079E00080931F0100910409109105098091EF080F
:1079F0009091F008101611065CF59C0197FF04C0E9
:107A000022273327281B390BC901AA2797FDA095E8
:107A1000BA2F20916501332744275527BC01CD019A
:107A20000E94B5729B01AC0197FF04C0215C3F4FDF
:107A30004F4F5F4FF6E05595479537952795FA9547
:107A4000D1F78091FF0890910009820F931F27C002
:107A500097FF03C0909581959F4FAA2797FDA0950A
:107A6000BA2F20916501332744275527BC01CD014A
:107A70000E94B5729B01AC0197FF04C0215C3F4F8F
:107A80004F4F5F4FE6E05595479537952795EA9517
:107A9000D1F78091FF0890910009821B930B90937E
:107AA00000098093FF08E0900909F0900A0980918D
:107AB000F1089091F2081E141F045CF59C0197FFD9
:107AC00004C022273327281B390BC901AA2797FD99
:107AD000A095BA2F20916501332744275527BC0173
:107AE000CD010E94B5729B01AC0197FF04C0215CDF
:107AF0003F4F4F4F5F4F76E0559547953795279508
:107B00007A95D1F78091F8089091F908820F931F28
:107B100027C097FF03C0909581959F4FAA2797FD97
:107B2000A095BA2F20916501332744275527BC0122
:107B3000CD010E94B5729B01AC0197FF04C0215C8E
:107B40003F4F4F4F5F4F66E05595479537952795C7
:107B50006A95D1F78091F8089091F908821B930BF0
:107B60009093F9088093F80880913E0987FF44C0FC
:107B7000B989BB2309F040C0809175028823E1F5E3
:107B8000E1E0EE16E1E0FE064CF0809101099091F3
:107B900002098E0D9F1D805091400DC0F0E0EF1640
:107BA000FFEFFF0664F480910109909102098E0DA8
:107BB0009F1D80509F4F909302098093010921E0FF
:107BC000013012074CF08091F6089091F708800F71
:107BD000911F805091400CC03FEF0030130764F4B8
:107BE0008091F6089091F708800F911F80509F4F69
:107BF0009093F7088093F608E2E1CD5E0C946073F1
:107C000080919202882329F5809160028C7F809375
:107C1000600280915F028F7D80935F02AAEBB3E0E8
:107C2000EAE6F7E09FE08091C601882309F48C938F
:107C30008D918183128291503F9697FFF4CF80916E
:107C4000C601882359F08091C60181508093C601F6
:107C500005C0809160028160809360028091400243
:107C6000882319F010924002089580934402809175
:107C70003E028E7F80933E0285EA8093BC00089589
:107C8000882319F480E090E00895E82FFF27EE0F95
:107C9000FF1FEF59F74F8081918181589F4F8F3F90
:107CA000910521F01CF08FEF90E004C097FF02C017
:107CB00080E090E099270895CF93DF93A4E9B2E0A4
:107CC000CAE3D6E057E08991E82FFF27EE0FFF1FA8
:107CD000EF59F74F0190F081E02DE158FF4FEF3F52
:107CE000F10521F01CF0EFEFF0E004C0F7FF02C057
:107CF000E0E0F0E0893111F4EC931BC04C91242FAB
:107D00003327E217F307A9F0CF01821B930B97FDEE
:107D100003969595879595958795242F280F2C93F5
:107D2000822F9927E817F90714F4215001C02F5F1B
:107D30002C935150119657FFC6CF80914406883F2F
:107D400038F0EFEFF0E0E81BF109EC56FD4F8081D1
:107D50008093790180917901882329F0843618F085
:107D600084E68093790180914606883F38F0EFEFF2
:107D7000F0E0E81BF109EC56FD4F8081809378011B
:107D800080917801882329F0843618F084E6809366
:107D9000780180915306883F38F0EFEFF0E0E81B60
:107DA000F109EC56FD4F808180937301809173013E
:107DB0008B3010F48AE002C08F3F11F4809373017E
:107DC00080918006883F38F0EFEFF0E0E81BF10982
:107DD000EC56FD4F808180931509809115098630FE
:107DE00010F485E002C08F3F11F480931509809153
:107DF0008206883F38F0EFEFF0E0E81BF109EC561F
:107E0000FD4F80818093450980914509863010F4AB
:107E100085E002C08F3F11F48093450980916D0683
:107E2000873F19F4429905C007C0863F41F4439B40
:107E300003C08091A20616C08091A30613C0883F9C
:107E400038F0EFEFF0E0E81BF109EC56FD4F8081D0
:107E50008093120980911209893110F488E102C0DF
:107E60008F3F11F48093120980916E06873F19F4B9
:107E7000429905C007C0863F41F4439B03C08091EF
:107E8000A40616C08091A50613C0883F38F0EFEF16
:107E9000F0E0E81BF109EC56FD4F80818093F30878
:107EA0008091F308893110F488E102C08F3F11F40A
:107EB0008093F30880916F06883F38F0EFEFF0E091
:107EC000E81BF109EC56FD4F808180931B098091DE
:107ED0001B09893110F488E102C08F3F11F48093AF
:107EE0001B09809145060E94403E8093700280915C
:107EF0004806883F38F0EFEFF0E0E81BF109EC5658
:107F0000FD4F80818093770180914A06883F38F049
:107F1000EFEFF0E0E81BF109EC56FD4F8081809314
:107F2000750180915206883F38F0EFEFF0E0E81BD2
:107F3000F109EC56FD4F80818093760180915406C3
:107F4000883F38F0EFEFF0E0E81BF109EC56FD4F09
:107F500080818093720180915506883F38F0EFEF61
:107F6000F0E0E81BF109EC56FD4F8081809374012D
:107F700080915606883F38F0EFEFF0E0E81BF109FA
:107F8000EC56FD4F80818093710180915706883FA8
:107F900038F0EFEFF0E0E81BF109EC56FD4F80817F
:107FA0008093700180915D06883F38F0EFEFF0E03C
:107FB000E81BF109EC56FD4F808180936E018091A2
:107FC0005E06883F38F0EFEFF0E0E81BF109EC5671
:107FD000FD4F808180936F0280915F06883F38F06B
:107FE000EFEFF0E0E81BF109EC56FD4F8081809344
:107FF0006E0280916006883F38F0EFEFF0E0E81BFA
:10800000F109EC56FD4F808180936D0280916106ED
:10801000883F38F0EFEFF0E0E81BF109EC56FD4F38
:10802000808180936C0280917B06883F38F0EFEF6F
:10803000F0E0E81BF109EC56FD4F808180936B0264
:1080400080917C06883F38F0EFEFF0E0E81BF10903
:10805000EC56FD4F808180936A0280917D06883FB7
:1080600038F0EFEFF0E0E81BF109EC56FD4F8081AE
:108070008093690280917E06883F38F0EFEFF0E050
:10808000E81BF109EC56FD4F8081809368028091D6
:108090006206883F38F0EFEFF0E0E81BF109EC569C
:1080A000FD4F808180936C0180916606883F38F097
:1080B000EFEFF0E0E81BF109EC56FD4F8081809373
:1080C0006B0180916306883F38F0EFEFF0E0E81B2A
:1080D000F109EC56FD4F808180936A01809167061B
:1080E000883F38F0EFEFF0E0E81BF109EC56FD4F68
:1080F00080818093690180917006883F38F0EFEFAE
:10810000F0E0E81BF109EC56FD4F80818093680197
:1081100080917306883F38F0EFEFF0E0E81BF1093B
:10812000EC56FD4F80818093670180917406883FF3
:1081300038F0EFEFF0E0E81BF109EC56FD4F8081DD
:108140008093660180917506883F38F0EFEFF0E08C
:10815000E81BF109EC56FD4F808180936501809109
:108160009E06883F38F0EFEFF0E0E81BF109EC568F
:10817000FD4F80818093FE088091420680933E09E6
:108180008091B50680931A0980917A06883F38F06D
:10819000EFEFF0E0E81BF109EC56FD4F8081809392
:1081A000640180919706883F38F0EFEFF0E0E81B1C
:1081B000F109EC56FD4F80818093570980916E0143
:1081C000282F33272F5F3F4F8CE398E2B9010E949D
:1081D000F47270937B0160937A01809150068093D2
:1081E000460980914F0680930609E0919906EE2397
:1081F000D9F181E080936702FF27EE0FFF1FEF594F
:10820000F74F80819181805C9F4F14F41092670238
:1082100080917C01209167028217B1F0833088F44D
:10822000222319F08CED95E002C088EC90E0909349
:10823000E9018093E80185E080937D0220937C0131
:1082400003C0815080937C01809197099091980997
:1082500097FF0FC080916702882359F08091B50382
:1082600080688093B50305C0E09367028AE080933D
:108270007C01809197099091980997FF1DC080918A
:1082800092028823C9F0809167028823A9F0809127
:108290000B0190910C018F5F9F4F61F488E99AE385
:1082A0009093E9018093E80180E094EA90930C01B7
:1082B00080930B011092670280916702882321F05E
:1082C00080915F02816003C080915F028E7F809306
:1082D0005F02DF91CF91089580914B06882301F5CD
:1082E000609177027091780277FF02C06D5F7F4FD7
:1082F0007595679575956795409123015091240177
:1083000080910201282F3327649FC001659F900D43
:10831000749F900D1124B9010E94E072CB0101C03D
:1083200099279093800180937F0180917F019091A4
:1083300080018734910538F486E490E090938001C1
:1083400080937F0108958F3A910530F08FEA90E095
:108350009093800180937F010895F8948091360670
:10836000E82FFF27EE0FFF1FEF59F74F6081718154
:108370007093600860935F0880913706E82FFF27AD
:10838000EE0FFF1FEF59F74F4081518150935D0869
:1083900040935C0880913906E82FFF27EE0FFF1FFE
:1083A000EF59F74F2081318130935B0820935A08B1
:1083B00080913806E82FFF27EE0FFF1FEF59F74F88
:1083C0000190F081E02DF093A808E093A708809138
:1083D000AE03A82FBB27A0FF3DC08091570981386D
:1083E000C8F18091A903992787FD9095680F791F9F
:1083F0007093600860935F088091AA03992787FDB6
:108400009095480F591F50935D0840935C088091E8
:10841000AB03992787FD9095280F391F30935B0890
:1084200020935A088091AC03A1FF0AC0992787FDC9
:108430009095E80FF91FF093A808E093A7080AC0E9
:10844000992787FD90958E179F0724F49093A8088D
:108450008093A708789480915F0890916008803895
:1084600091051CF08FE790E005C081589F4F34F4D0
:1084700081E89FEF9093600880935F0880915C088B
:1084800090915D08803891051CF08FE790E005C061
:1084900081589F4F34F481E89FEF90935D0880935B
:1084A0005C0880915A0890915B08803891051CF017
:1084B0008FE790E005C081589F4F34F481E89FEF2B
:1084C00090935B0880935A088091A7089091A80820
:1084D000803891053CF08FE790E09093A808809356
:1084E000A708089581589F4F34F481E89FEF909337
:1084F000A8088093A7080895ABE0B0E0E2E8F2E4B2
:108500000C9444730E9445378091600299278471CE
:108510009070892B91F58091B60682FF27C08091DB
:108520007702909178020097F1F022E08835920767
:10853000D4F49C0197FF02C02D5F3F4F35952795DE
:108540003595279580915A069927289FA001299F44
:10855000500D389F500D1124CA0164E670E00E944E
:10856000F472CB0106C08DE290E003C080915A0600
:10857000992790935D0280935C0220915A0230917A
:108580005B0255E72033350759F410929E02109292
:108590009D0280910609992790935D0280935C0269
:1085A00060919D0270919E027A8369838091060991
:1085B00099270A966817790714F49A83898380911A
:1085C00093028436C8F580915F0282FD35C08AE04F
:1085D000809350028091150390911603009731F01B
:1085E000019790931603809315030BC0109292028B
:1085F0009093620280936102809160028D7E8093ED
:108600006002289A8091610290916202895E934093
:1086100080F08091E609853660F080915C0290914F
:108620005D029A83898380916002806180936002F9
:10863000E9C310929202E6C3809193028D3808F448
:10864000B7C3809160028F7E8093600290915B0639
:1086500082E3989FC0011124909316038093150321
:10866000A981BA8199978CF080919202882369F050
:108670008091610290916202BFEF8F3F9B0729F0CA
:108680000196909362028093610220916102309181
:1086900062022F3F310509F030F51092B5021092B9
:1086A000B6021092B7021092B8021092B102109264
:1086B000B2021092B3021092B40210920903109207
:1086C0000A0310920B0310920C031092BD02109239
:1086D000BE021092BF021092C00280915F028062BF
:1086E00080935F024DC0809160028260809360023F
:1086F00080915F0285FF44C08091F8019091F9015B
:10870000A091FA01B091FB0187399105A105B1054E
:108710008CF480918D0290918E02A0918F02B09185
:108720009002825A9E4FAF4FBF4F24F080913E0976
:1087300080FD05C080915F028F7180935F0210926F
:10874000B5021092B6021092B7021092B8021092BF
:10875000B1021092B2021092B3021092B4021092BF
:10876000BD021092BE021092BF021092C002295E9A
:10877000334030F088EE93E0909362028093610280
:108780008091A7089091A808813591050CF4F9C053
:1087900040919202442309F0F4C080914603992746
:1087A0009C012071307084FDECC080915A0890913A
:1087B0005B088C3491050CF4B4C0809119038F5F71
:1087C00080931903893C08F4DCC0142F40931903EB
:1087D000309362022093610220915F08309160081B
:1087E000273431056CF480915C0890915D0897FF07
:1087F00003C0909581959F4F873491050CF444C038
:1088000040915C0850915D08473451053CF0263496
:10881000310524F42B5B3F4F0CF011E04734510538
:1088200044F080915F0890916008873491050CF0C6
:1088300012E04634510544F480915F08909160083D
:10884000873491050CF013E07FEF4A3B570744F45F
:1088500080915F0890916008873491050CF014E0D6
:108860004A5B5F4F64F480915F08909160088634A2
:1088700091052CF48B5B9F4F14F015E002C011237F
:1088800019F0812F0E94662980915C0890915D0803
:108890004D96CB9798F480915F08909160088A5B21
:1088A0009F4F64F481E08093D00310927E0288EEA3
:1088B00093E09093E9018093E80163C08091010106
:1088C0000E940D2980E00E94810580915C060E9433
:1088D000B16E80913E0980FF10C080911901909186
:1088E0001A01875B934038F48091190190911A0125
:1088F0008E5E924010F40E94081B112381F4809137
:108900005C0890915D088A5B9F4F4CF480915F08F2
:10891000909160088634910514F483E01DC081E0D5
:108920001BC0855B9F4F3CF580915C0890915D0872
:108930000F964F9700F580911703909118030196B9
:108940009093180380931703855C9940D0F030937F
:1089500018032093170382E00E94E83380937E027D
:1089600081E08093E601579A68E770E08091010109
:108970000E94F23206C0109219031092180310924E
:1089800017038091A7089091A8088C599F4F0CF06D
:1089900008C2E0919A06AE2FBB27AF77B070AA0F3E
:1089A000BB1FA755B74F8D919C911197069714F057
:1089B00084E606C08D919C918B5F9F4F1CF48CE9DF
:1089C00080931C038091920220915A0830915B0899
:1089D000882309F04EC12C593F4F94F48091B6067C
:1089E00083FD0AC0FF27EE0FFF1FEF59F74F80816D
:1089F0009181855B9F4FDCF080919A068823B9F0C6
:108A00008091B60683FF32C180919A06E82FFF2736
:108A1000EE0FFF1FEF59F74F80819181875F9F4FC6
:108A20000CF424C180911C03843609F01FC180918D
:108A3000460384FD1BC180917E02882329F080912A
:108A4000600288608093600280911B0190911C01FC
:108A5000A0911D01B0911E018093D7059093D80578
:108A6000A093D905B093DA0510928D0210928E0270
:108A700010928F02109290021092F4011092F50160
:108A80001092F6011092F70188E592E090935B0254
:108A900080935A0210920502109206021092070269
:108AA0001092080280915F08909160088D599F4F45
:108AB0004CF480915C0890915D088D599F4F873CE4
:108AC000910530F480919A06882311F480931A035B
:108AD00080911A038F5F80931A038E3F08F444C17C
:108AE00080915E022091490930914A0981FF21C09D
:108AF000C90137FF04C088279927821B930B813453
:108B00009105ACF5809101099091020997FF03C08E
:108B1000909581959F4FCD9754F58091F60890914F
:108B2000F70897FF03C0909581959F4FCD970CF163
:108B30001EC0C90137FF03C0909581959F4F819753
:108B4000B4F4809101099091020997FF03C09095B8
:108B500081959F4F45975CF48091F6089091F708B6
:108B600097FF03C0909581959F4F459714F0109201
:108B70007E0210921A038091B503882309F073C016
:108B800080917E02882309F46EC080914A03882375
:108B900009F069C081E090E09093620280936102E5
:108BA00081E0809392021092090310920A031092BE
:108BB0000B0310920C031092BD021092BE02109291
:108BC000BF021092C0021092B9021092BA02109223
:108BD000BB021092BC0280915106E82EFF240027B0
:108BE000112780914209909143099C01442737FD48
:108BF0004095542FC801B7010E94B572DC01CB012A
:108C00008093C5029093C602A093C702B093C80296
:108C100080915409909155099C01442737FD409556
:108C2000542FC801B7010E94B572DC01CB018093BB
:108C3000C1029093C202A093C302B093C4021092E7
:108C4000B5021092B6021092B7021092B8021092BA
:108C5000B1021092B2021092B3021092B40284E6F2
:108C600080937D0281C08CED95E077C010921A034D
:108C70007BC02536310594F08091B60683FD0AC08D
:108C8000FF27EE0FFF1FEF59F74F80819181855B22
:108C90009F4FDCF080919A068823B9F08091B60648
:108CA00083FF60C080919A06E82FFF27EE0FFF1F19
:108CB000EF59F74F808191818E5C9F4F0CF052C02D
:108CC00080911C038C3909F04DC080915F08909110
:108CD00060088D599F4F4CF480915C0890915D081D
:108CE0008D599F4F873C910538F480919A068823CF
:108CF00019F480931B0318C01092B5021092B602AB
:108D00001092B7021092B8021092B1021092B20201
:108D10001092B3021092B4021092A4021092A30215
:108D20001092A2021092A10280911B038F5F809388
:108D30001B038B3F70F01092920210921B03109253
:108D400062021092610280915F028F7180935F02D4
:108D50000BC0843649F48CEA9DE09093E90180933E
:108D6000E80102C010921B0320915A0230915B026D
:108D700043E0283E340708F045C0809102029091FC
:108D800003028B569F4F1CF02F5F3F4F05C02115EC
:108D90003105C1F12150304030935B0220935A02DB
:108DA00031C010921C0310925B0210925A022AC02A
:108DB0002E5E324038F180915F09909160098059B0
:108DC000914000F580918D0290918E02A0918F02CA
:108DD000B09190028C5D9540A040B0409CF480E33F
:108DE00095E790935B0280935A0280916102909183
:108DF00062028A5E934030F089EE93E090936202C3
:108E00008093610280913F01815080933F01809166
:108E10003F018F3F21F08091600284FF80C30E9458
:108E20005C3E0E94AD4120914C0680911D039091C3
:108E30001E03AC01440F551F480F591F3327809163
:108E40005F0890916008829FB001839F700D929F90
:108E5000700D1124460F571F57FF02C04D5F5F4F23
:108E6000559547955595479550931E0340931D037F
:108E700080911F0390912003AC01440F551F480FB0
:108E8000591F80915C0890915D08829FD001839F5B
:108E9000B00D929FB00D11244A0F5B1F57FF02C007
:108EA0004D5F5F4F559547955595479550932003D6
:108EB00040931F03F89400913606E02FFF27EE0F32
:108EC000FF1FE755F74F80914D06482F55278081AA
:108ED0009181849F9001859F300D949F300D1124C6
:108EE00080911D0390911E03820F931F90931E0388
:108EF00080931D0310913706E12FFF27EE0FFF1F10
:108F0000E755F74F80819181849F9001859F300DB7
:108F1000949F300D112480911F0390912003820FA4
:108F2000931F9093200380931F0378948091A70848
:108F30009091A80881589F4F90939E0280939D0224
:108F40008091670240911D0350911E03882309F40C
:108F50004BC0CA0157FD0396DC01B595A795B595A1
:108F6000A79580911F039091200397FD0396FC0124
:108F7000F595E795F595E7958091A101682F7727FD
:108F800067FD70956A9F90016B9F300D7A9F300D41
:108F9000112480914D03482F552747FD50954E9F32
:108FA000C0014F9F900D5E9F900D1124280F391F17
:108FB00037FF02C0295F3F4F93E0359527959A957B
:108FC000E1F73093A4022093A3026E9F90016F9F5C
:108FD000300D7E9F300D11244A9FC0014B9F900D94
:108FE0005A9F900D112443C080919806E82FFF27C7
:108FF000EB5BFE4F86818093A101908190934D039E
:10900000A82FBB27A7FDB095A49F9001A59F300D69
:10901000B49F300D1124E92FFF27E7FDF0956091F3
:109020001F0370912003E69FC001E79F900DF69FFC
:10903000900D1124280F391F37FF02C0295F3F4FC1
:1090400083E0359527958A95E1F73093A402209324
:10905000A302A69F9001A79F300DB69F300D11244B
:10906000E49FC001E59F900DF49F900D1124281BF3
:10907000390B37FF02C0295F3F4FF3E03595279545
:10908000FA95E1F73093A2022093A10280915A0849
:1090900090915B08909581959F4F9093A00280934B
:1090A0009F028530910514F0049705C0BFEF8C3FF7
:1090B0009B0734F404969093A00280939F0204C00F
:1090C0001092A00210929F0280915A0290915B022E
:1090D0008150924078F18091A3029091A40297FD73
:1090E0000796E3E095958795EA95E1F79093A402BA
:1090F0008093A3028091A1029091A20297FD07960E
:1091000073E0959587957A95E1F79093A202809305
:10911000A1021092B5021092B6021092B7021092FC
:10912000B8021092B1021092B2021092B3021092E1
:10913000B40243C080913803882309F43EC0282F2D
:1091400033278091A3029091A40297FD079663E0D4
:10915000959587956A95E1F7289FA001299F500D65
:10916000389F500D1124CA0157FD0F9654E0959574
:1091700087955A95E1F79093A4028093A30280917A
:10918000A1029091A20297FD079643E095958795DD
:109190004A95E1F7289FB001299F700D389F700D07
:1091A0001124CB0177FD0F96B4E095958795BA957C
:1091B000E1F79093A2028093A102C090A302D09005
:1091C000A40280913B0390913C03C81AD90AD09223
:1091D000A402C092A3028091A1029091A2022091C8
:1091E000390330913A03821B930B9093A202809330
:1091F000A102809173019927AA2797FDA095BA2F04
:10920000BC01CD010E942972DC01CB0120E030E0DD
:1092100040E251E4BC01CD010E949771DC01CB0119
:10922000BC01CD010E94FB71DC01CB0180934E0992
:109230008091720180931C09809171019927AA275E
:1092400097FDA095BA2FBC01CD010E942972DC01C7
:10925000CB0120E030E040E251E4BC01CD010E94AE
:109260009771DC01CB01BC01CD010E94FB71DC01D7
:10927000CB018093FD088091700180930B09809150
:109280003E0982FF02C010921C09C601D7FC03965A
:109290009C01359527953595279537FF03C0309567
:1092A00021953F4F80916502909166028217930746
:1092B000B4F4C601D7FE03C0909581959F4F97FDEA
:1092C00003969595879595958795909366028093DB
:1092D00065028536910544F084E690E001C001976F
:1092E00090936602809365024091A1025091A20280
:1092F000CA0157FD03969C0135952795359527950D
:1093000037FF03C0309521953F4F809163029091C4
:10931000640282179307B4F4CA0157FF03C0909503
:1093200081959F4F97FD0396959587959595879580
:1093300090936402809363028536910544F084E63D
:1093400090E001C001979093640280936302809142
:10935000600284FF08C010926602109265021092AB
:10936000640210926302E12FFF27EE0FFF1FEF59F7
:10937000F74F40917106242F332780819181281760
:10938000390744F48091B30682FF04C081E08093E2
:10939000740213C0E12FFF27EE0FFF1FEF59F74FA5
:1093A000842F992720917206821B91092081318197
:1093B0002817390714F41092740240913706E42FED
:1093C000FF27EE0FFF1FEF59F74F50917106852FC2
:1093D000992722273327281B390B808191818217F7
:1093E000930744F48091B30683FF04C081E0809327
:1093F000730216C080917302882391F0E42FFF2737
:10940000EE0FFF1FEF59F74F809172069927851BCA
:109410009109208131818217930714F4109273020D
:10942000E02FFF27EE0FFF1FEF59F74F4091710616
:10943000242F3327808191812817390744F48091A4
:10944000B30680FF04C081E08093710217C0809151
:109450007102882399F0E02FFF27EE0FFF1FEF59CD
:10946000F74F842F992720917206821B9109208142
:1094700031812817390714F4109271024091360691
:10948000E42FFF27EE0FFF1FEF59F74F50917106A2
:10949000852F992722273327281B390B808191811B
:1094A0008217930744F48091B30681FF04C081E0E2
:1094B0008093720216C080917202882391F0E42F8B
:1094C000FF27EE0FFF1FEF59F74F80917206992784
:1094D000851B9109208131818217930714F4109222
:1094E000720280917402882319F4809173028111B1
:1094F00081E08093750280917102882321F480912C
:109500007202882351F081E08093760210927502F6
:10951000109274021092730202C0809376028091BE
:109520007502882321F480917602882369F0809166
:1095300070069927A981BA818A179B0714F49A8328
:10954000898381E08093A90280915F0299279C0121
:109550002470307082FF31C080913B0390913C03B6
:10956000909581959F4F9093A4028093A302809140
:10957000390390913A03909581959F4F9093A20261
:109580008093A10280917F019091800190939E022F
:1095900080939D021092A00210929F0280913E093A
:1095A0008B778B6680933E0980911A098C7B809320
:1095B0001A0988EC809370021EC08091600284FFBB
:1095C0001AC03093A00220939F023093A4022093EC
:1095D000A3023093A2022093A1029AE590934E0930
:1095E00088E780931C099093FD0880930B091092E3
:1095F00075021092760280910E0990910F09A09148
:109600001009B09111092091D1023091D2024091FC
:10961000D3025091D402820F931FA41FB51F8093D1
:109620000E0990930F09A0931009B093110980912E
:10963000160990911709A0911809B0911909209065
:10964000CD023090CE024090CF025090D002820DD9
:10965000931DA41DB51D8093160990931709A0931F
:109660001809B0931909B0917602BB83BB2321F48A
:1096700080917502882301F110920E0910920F0952
:1096800010921009109211091092160910921709E0
:1096900010921809109219091092010210920002FA
:1096A00010927A021092790210927C0210927B0240
:1096B000EB81EE2309F0E4C180917502882309F063
:1096C000DFC18091D5059091D605815092402CF450
:1096D00080919202882309F4D3C19090D009A09080
:1096E000510660914209709143097B876A87809196
:1096F0005409909155099987888719140CF0BEC0B8
:10970000BB24CC24DD24CA01B901A60195010E9425
:10971000297379018A018091990990919A09AA8502
:10972000BB85A81BB90BFD01CF01AA2797FDA0950A
:10973000BA2FE81AF90A0A0B1B0BC201B101A601E4
:1097400095010E94297359016A0180919B099091AA
:109750009C0928853985281B390BC901AA2797FD43
:10976000A095BA2FA81AB90ACA0ADB0A292C3324F1
:1097700027FC3094432C532CC801B701A20191015E
:109780000E94B57297FF04C061507E4F8F4F9F4F6C
:109790003B014C0169E095948794779467946A95AE
:1097A000D1F7C601B501A20191010E94B57297FFE0
:1097B00004C061507E4F8F4F9F4F5B016C0159E099
:1097C000D594C794B794A7945A95D1F78091650220
:1097D00090916602813491053CF4809163029091EE
:1097E000640281349105D4F0D401C30197FE03C013
:1097F0000196A11DB11D3C014D019594879477946C
:109800006794D601C501D7FE03C00196A11DB11D05
:109810005C016D01D594C794B794A7948091D20947
:10982000282F332727FD3095432F532F2615370533
:109830004805590514F439014A01992787FD909587
:10984000909581959F4FAA2797FDA095BA2F6816EE
:1098500079068A069B0614F43C014D012A153B0546
:109860004C055D0514F459016A01A816B906CA062B
:10987000DB060CF0C9C05C016D01C6C0EA2CFF24F8
:1098800000271127CA01B901A80197010E94297375
:1098900039014A014A855B85CA01AA2797FDA0952F
:1098A000BA2F681A790A8A0A9B0AC201B101A80173
:1098B00097010E94297359016A0168857985CB0156
:1098C000AA2797FDA095BA2FA81AB90ACA0ADB0AD7
:1098D000D401C30197FE03C00F96A11DB11D3C0129
:1098E0004D0124E095948794779467942A95D1F755
:1098F000D601C501D7FE03C00F96A11DB11D5C01A5
:109900006D0194E0D594C794B794A7949A95D1F734
:109910008091650290916602813491053CF48091BA
:1099200063029091640281349105A4F0C401B301F3
:1099300023E030E040E050E00E94297339014A0101
:10994000C601B50123E030E040E050E00E942973F9
:1099500059016A0180915A0890915B0897FF03C0F2
:10996000909581959F4F4A97A4F0C401B30123E0DD
:1099700030E040E050E00E94297339014A01C601FD
:10998000B50123E030E040E050E00E942973590126
:109990006A0189E180938B0171E267167104810489
:1099A00091042CF080E2682E712C812C912C80EE99
:1099B00068168FEF78068FEF88068FEF980644F4CD
:1099C00000EE602E0FEF702E0FEF802E0FEF902E17
:1099D00091E2A916B104C104D1042CF010E2A12E29
:1099E000B12CC12CD12CA0EEAA16AFEFBA06AFEF66
:1099F000CA06AFEFDA0644F4B0EEAB2EBFEFBB2ED3
:109A0000BFEFCB2EBFEFDB2E8091C5029091C60237
:109A1000A091C702B091C80286199709A809B9098F
:109A20008093C5029093C602A093C702B093C80268
:109A30008091C1029091C202A091C302B091C40270
:109A40008A199B09AC09BD098093C1029093C20297
:109A5000A093C302B093C402809153029091540228
:109A6000860D971D9093540280935302809151026A
:109A7000909152028A0D9B1D909352028093510245
:109A800080910002909101028F3F910509F008F446
:109A900052C1E0917906EE2309F4FFC0809142099A
:109AA00090914309815E9C4F8F53964008F0F5C01A
:109AB0008091540990915509815E9C4F8F53964037
:109AC00008F0EBC08091A902882309F0E6C08091DC
:109AD000490990914A094F96CF9708F0DEC0FF27B9
:109AE000A6E0EE0FFF1FAA95E1F7209153023091F7
:109AF0005402C901BF010E94E072261B370B30934C
:109B00005402209353022091510230915202C90114
:109B1000BF010E94E072261B370B30935202209344
:109B200051022091A7023091A802C901BF010E94F1
:109B3000E072261B370B3093A8022093A702809176
:109B40006502909166028134910594F480916302DC
:109B500090916402813491055CF480915A0890914F
:109B60005B0897FF03C0909581959F4F4A97E4F05B
:109B7000809153029091540297FD01969595879597
:109B8000909354028093530280915102909152021B
:109B900097FD019695958795909352028093510277
:109BA0001092A8021092A702809153029091540241
:109BB000895B9B406CF0109254021092530280918A
:109BC000ED029091EE0201969093EE028093ED02E9
:109BD00080915302909154028854944F6CF41092E7
:109BE0005402109253028091ED029091EE0201977F
:109BF0009093EE028093ED02809151029091520277
:109C0000895B9B406CF0109252021092510280913D
:109C1000EB029091EC0201969093EC028093EB02A0
:109C200080915102909152028854944F6CF410929A
:109C30005202109251028091EB029091EC02019736
:109C40009093EC028093EB028091A7029091A8027E
:109C50008D5A9D406CF01092A8021092A70280913C
:109C6000E9029091EA0201969093EA028093E90258
:109C70008091A7029091A8028455924FD4F410923B
:109C8000A8021092A7028091E9029091EA0201973E
:109C90009093EA028093E9020CC010925402109251
:109CA000530210925202109251021092A802109286
:109CB000A7021092A90280911C09882341F41092F6
:109CC0007C0210927B0210927A02109279028091AB
:109CD0000E0990910F09A0911009B091110980937C
:109CE000210390932203A0932303B0932403809134
:109CF000160990911709A0911809B091190980933C
:109D0000250390932603A0932703B0932803109272
:109D10000E0910920F091092100910921109109259
:109D20001609109217091092180910921909109229
:109D300001021092000280909F029090A002C40144
:109D400097FE04C0882799278819990904973CF041
:109D500080913E0984FD03C082E380937D021091CF
:109D60004E06A12EBB24CC24DD24B401882777FD28
:109D70008095982F940197FE04C022273327281935
:109D80003909442737FD4095542F0E94B5729B0135
:109D9000AC01C601B5010E94B57297FF04C06150C5
:109DA0007E4F8F4F9F4F59E0959587957795679593
:109DB0005A95D1F79B01812F9927889DD001899DC4
:109DC000B00D989DB00D1124CD01B7FD039695956A
:109DD000879595958795280F391F80915A02909104
:109DE0005B028150924010F020E030E080917F02D1
:109DF00090918002820F931F9C01442737FD40956C
:109E0000542F2093090330930A0340930B0350937C
:109E10000C038091BD029091BE02A091BF02B0914F
:109E2000C002821B930BA40BB50B8093BD029093D1
:109E3000BE02A093BF02B093C0028155934CA040D4
:109E4000B04064F080E593ECA0E0B0E08093BD0208
:109E50009093BE02A093BF02B093C0028091BD0256
:109E60009091BE02A091BF02B091C002805B9C4362
:109E7000AF4FBF4F64F480EB9CE3AFEFBFEF809335
:109E8000BD029093BE02A093BF02B093C002809027
:109E90008F019090900197FCFAC080913E0983FF5A
:109EA000F6C080918C01815080938C01882309F049
:109EB000F2C08DE080938C018091D1029091D2020A
:109EC000A091D302B091D402B7FF04C081509E4F3D
:109ED000AF4FBF4F39E0B595A795979587953A95C0
:109EE000D1F78C0197FF03C0109501951F4F80910A
:109EF000CD029091CE02A091CF02B091D002B7FFD7
:109F000004C081509E4FAF4FBF4F29E0B595A79534
:109F1000979587952A95D1F79C0197FF03C03095B7
:109F200021953F4F021713070CF48901B80117FF61
:109F300002C0695F7F4F3B01A3E075946794AA95C7
:109F4000E1F722E030E0620E731EA0905009B0905D
:109F50005109C0905209D09053092091410130918C
:109F600042014091430150914401C601B5010E9454
:109F7000297319012A013093FC082093FB08821AE7
:109F8000930AC401845E9D4F68E671E00E94F472FA
:109F9000AC01445B504020917D02222321F030929D
:109FA000AC022092AB028091890190918A010097C6
:109FB00031F0019790938A018093890112C0093191
:109FC00011057CF48091A7029091A802840F951F3F
:109FD0009093A8028093A702222319F02150209386
:109FE0007D028091890190918A01892BF9F48091F9
:109FF0008B019927489FB001499F700D589F700DA4
:10A000001124CB01B3010E94F472CB01AA2797FD62
:10A01000A095BA2FA80EB91ECA1EDB1EA092500929
:10A02000B0925109C0925209D092530980917D0299
:10A03000882369F58091AB029091AC022091FB08D6
:10A040003091FC08821B930B845E9D4F68E671E0A3
:10A050000E94F4729C01245B3040809176018695C9
:10A060009927289FD001299FB00D389FB00D11244A
:10A070009D01B7FF02C0215F3F4FF4E03595279562
:10A08000FA95E1F73093800220937F0204C010928A
:10A09000800210927F028091A902882381F01092A1
:10A0A000B1021092B2021092B3021092B402109256
:10A0B000B5021092B6021092B7021092B802BB819C
:10A0C000BB23F1F480911C09282F332744275527FF
:10A0D0008091D1029091D202A091D302B091D4028A
:10A0E000BC01CD010E94B572DC01CB01BC01CD01E8
:10A0F00028EF3AE240E050E00E942973390102C0A3
:10A1000066247724809175028823F1F480911C09DC
:10A11000282F3327442755278091CD029091CE02D6
:10A12000A091CF02B091D002BC01CD010E94B572C6
:10A13000DC01CB01BC01CD0128EF3AE240E050E068
:10A140000E942973290102C0442455248091F808F3
:10A150009091F908893C91051CF088EC90E005C0CD
:10A1600088539F4F34F488E39FEF9093F9088093CE
:10A17000F8088091FF0890910009893C91051CF036
:10A1800088EC90E005C088539F4F34F488E39FEF3C
:10A19000909300098093FF08809101099091020932
:10A1A000AA2797FDA095BA2F20914E09A22EBB2475
:10A1B000CC24DD24BC01CD01A60195010E94B5721D
:10A1C0009B01AC018091F8089091F908AA2797FDAE
:10A1D000A095BA2FE7E0880F991FAA1FBB1FEA9529
:10A1E000D1F7280F391F4A1F5B1F57FF04C0215C9E
:10A1F0003F4F4F4F5F4F76E05595479537952795E1
:10A200007A95D1F78301020F131F1093020900936F
:10A2100001098091F6089091F708AA2797FDA0956B
:10A22000BA2FBC01CD01A60195010E94B5729B0118
:10A23000AC018091FF0890910009AA2797FDA09595
:10A24000BA2F67E0880F991FAA1FBB1F6A95D1F725
:10A25000280F391F4A1F5B1F57FF04C0215C3F4F67
:10A260004F4F5F4FA6E05595479537952795AA958F
:10A27000D1F74201820E931E9092F7088092F60861
:10A280008091490990914A09880F991FAA2797FD43
:10A29000A095BA2F2091FD08332744275527BC01EC
:10A2A000CD010E94B5725B016C0197FF08C02FE3DE
:10A2B00030E040E050E0A20EB31EC41ED51EF6E012
:10A2C000D594C794B794A794FA95D1F780910B09C8
:10A2D000282F3327442755278091C9029091CA021D
:10A2E000A091CB02B091CC02BC01CD010E94B5720D
:10A2F000DC01CB01BC01CD0120EF35E540E050E0B1
:10A300000E942973B501620F731F70934A0960930D
:10A3100049090150104134F080E090E19093020926
:10A320008093010980910109909102098050904F1A
:10A3300034F480E090EF909302098093010951E09A
:10A34000851650E1950634F080E090E19093F7088F
:10A350008093F6088091F6089091F7088050904F0E
:10A3600034F480E090EF9093F7088093F608615002
:10A37000704134F080E090E190934A09809349095C
:10A380008091490990914A098050904F34F480E0BF
:10A3900090EF90934A09809349098091600285FD6E
:10A3A00016C0809102019927209123013091240148
:10A3B00069817A81689FA001699F500D789F500D37
:10A3C0001124CA01B9010E94E0727A8369838091E5
:10A3D00029038150809329038F3F09F062C0809147
:10A3E0002A0390912B03892B41F4809123019091B2
:10A3F000240190932B0380932A0380912301909151
:10A40000240120912A0330912B032817390718F4CF
:10A410002F5F3F4F09C08091230190912401821743
:10A42000930730F42150304030932B0320932A03BC
:10A4300084E6809329038091B901282F3327409126
:10A440002A0350912B034217530730F48AE080937C
:10A450005602809350020EC080910001280F311DDA
:10A460002417350738F480915602882319F081505B
:10A47000809356028091B801282F33274217530743
:10A4800010F489E10CC080910001280F311D2417C0
:10A49000350738F480915502882319F08150809354
:10A4A000550280915602882369F180918302909130
:10A4B0008402A0918502B0918602B7FD23C020914D
:10A4C000AC062093820280918D0290918E02A09121
:10A4D0008F02B09190028D5D9540A040B04034F065
:10A4E000822F9927880F991F8093820280EE91EB2B
:10A4F000AFEFBFEF8093830290938402A093850215
:10A50000B09386028091E701882311F40E94945E43
:10A5100089819A81880F991F880F991F9A8389834F
:10A5200080913E0980FFDAC780917502882309F087
:10A53000D5C740917602442309F0D0C78091B50376
:10A5400099278F779070009709F0C8C74C01209128
:10A55000EF023091F0022115310509F044C08091DD
:10A56000190190911A018959934058F087B5853F98
:10A5700020F480910402815011C081E08093370360
:10A5800055C08091190190911A018436910530F5DA
:10A5900087B58B30F8F0809104028F5F80930402BE
:10A5A0009AE08902900111248091E105821B87BD08
:10A5B00087B5809588BD8CE291E09093E901809306
:10A5C000E8018EE591E09093F0028093EF020E9403
:10A5D000D01A2CC081E08093360328C04093360304
:10A5E0004093370323C09093030280930202F894B0
:10A5F00080918D0290918E02A0918F02B091900275
:10A6000074E0880F991FAA1FBB1F7A95D1F780931A
:10A61000050290930602A0930702B0930802789473
:10A62000215030403093F0022093EF0280913E0998
:10A630009091700281FF25C09233E8F480919101DE
:10A640008150809391018F3F81F51092AA028091F1
:10A650008D0290918E02A0918F02B0919002809312
:10A66000890290938A02A0938B02B0938C0281E0BE
:10A67000809391011AC09734C0F088EC80939101C7
:10A6800011C080914706989FC0011124AA2797FD09
:10A69000A095BA2F8093890290938A02A0938B028F
:10A6A000B0938C0281E08093AA028091D1029091B4
:10A6B000D202A091D302B091D402E0904101F09077
:10A6C00042010091430110914401BC01CD01A80158
:10A6D00097010E94297359016A018091CD029091DE
:10A6E000CE02A091CF02B091D002BC01CD01A80151
:10A6F00097010E942973B901C5010E94106A209137
:10A7000075013327829FF001839FF00D929FF00D1A
:10A710001124CF0164E670E00E94F4729B016C3357
:10A72000710514F02CE330E0C9010E943968909360
:10A7300008098093070980E2809340011092880203
:10A74000109287028091AA02882309F46EC5809135
:10A75000600299279C012071307084FD66C580914C
:10A760005F02826080935F0270911A09872F992798
:10A7700061E0C62ED12CC822D92280FD04C0809170
:10A780003E0981FD10C009811A8130932D03209369
:10A790002C03309388022093870280916002806CA2
:10A7A00080936002CFC28091600281FF9EC20091BF
:10A7B0007F0110918001C8010F96A0909D02B0907A
:10A7C0009E028A159B0508F079C080913603882384
:10A7D00009F074C08091600287FF15C0809160020B
:10A7E0008F77809360028091F8019091F901A09198
:10A7F000FA01B091FB018093890290938A02A093A1
:10A800008B02B0938C02E090FE08EE20F9F080916C
:10A81000890290918A02A0918B02B0918C02BC01B6
:10A82000CD0124E630E040E050E00E9429738E2DF7
:10A830009927AA27BB2782179307A407B50734F4E3
:10A84000D0928802C09287028DE378C080912E0357
:10A8500090912F03459784F08091F8019091F90130
:10A86000A091FA01B091FB018093890290938A0232
:10A87000A0938B02B0938C028091600280648093DD
:10A8800060029501201B310B2F50304037FF03C071
:10A89000309521953F4F3093880220938702809115
:10A8A0005602882349F0C90163E070E00E94F47207
:10A8B00070938802609387028BE240C0C8010F97B3
:10A8C000A816B90608F03FC0809137038823D9F550
:10A8D0008091600286FD07C080912E0390912F0326
:10A8E000845D9E4FACF4809160028F7B8093600208
:10A8F0008091F8019091F901A091FA01B091FB01CA
:10A900008093890290938A02A0938B02B0938C0269
:10A9100080916002806880936002C501801B910B6A
:10A920000F9697FF03C0909581959F4F90958195C5
:10A930009F4F90938802809387028DE2809340011D
:10A9400010928102D9C08DE3809340016091820210
:10A95000662371F120918302309184024091850237
:10A96000509186028091890290918A02A0918B0277
:10A97000B0918C0282179307A407B507CCF480919D
:10A980006002806480936002862F992790938802EA
:10A99000809387028AE0809381028EE58093400154
:10A9A0008091600287FFA8C0809160028F7733C0DA
:10A9B000662309F443C020918302309184024091C0
:10A9C0008502509186028091890290918A02A0911D
:10A9D0008B02B0918C02281739074A075B0774F580
:10A9E00080916002806880936002862F99279095FD
:10A9F00081959F4F909388028093870286EF809382
:10AA0000810286E7809340018091600286FF74C0D6
:10AA1000809160028F7B809360028091F801909119
:10AA2000F901A091FA01B091FB0180938902909302
:10AA30008A02A0938B02B0938C025EC08091600268
:10AA4000807C09F459C080918102882379F5A09017
:10AA5000F801B090F901C090FA01D090FB01D60145
:10AA6000C501885C9040A040B0402091890230919F
:10AA70008A0240918B0250918C0282179307A4079F
:10AA8000B5075CF4D601C50188539F4FAF4FBF4F48
:10AA9000281739074A075B075CF080938902909377
:10AAA0008A02A0938B02B0938C0202C010928102A2
:10AAB000809160028F738093600210922D03109238
:10AAC0002C0371FF06C084EF91E09093E90180931D
:10AAD000E80180919102882379F480918D02909110
:10AAE0008E02A0918F02B0919002C397A105B1058B
:10AAF0001CF081E08093910260912C0370912D03F2
:10AB00008091870290918802680F791F70932D03BE
:10AB100060932C03CB0177FF04C088279927861BFD
:10AB2000970B855F91400CF4C9C04091810244238A
:10AB300089F1809183029091840220918902309161
:10AB40008A02821B930B0996439748F480918302F3
:10AB500090918402A0918502B091860212C0242FA8
:10AB6000332727FD3095432F532F809189029091F1
:10AB70008A02A0918B02B0918C02820F931FA41FB6
:10AB8000B51F8093890290938A02A0938B02B093A1
:10AB90008C0224C02091890230918A0240918B025C
:10ABA00050918C02809147061616170644F463E014
:10ABB0000E94D472280F311D411D511D07C063E052
:10ABC0000E94D472281B310941095109209389023E
:10ABD00030938A0240938B0250938C0210922D0383
:10ABE00010922C03A0908D02B0908E02C0908F0224
:10ABF000D0909002D601C50180509440A040B04052
:10AC00002091F8013091F9014091FA015091FB0136
:10AC100082179307A407B5075CF4D601C5018050DD
:10AC20009C4FAF4FBF4F281739074A075B0744F0C7
:10AC30008093F8019093F901A093FA01B093FB017E
:10AC4000A090F801B090F901C090FA01D090FB01FA
:10AC5000D601C50180509440A040B04020918902A7
:10AC600030918A0240918B0250918C028217930797
:10AC7000A407B5075CF4D601C50184529A4FAF4FC3
:10AC8000BF4F281739074A075B0744F080938902B2
:10AC900090938A02A0938B02B0938C0280911A0940
:10ACA00081FF06C084E690E09093E9018093E8017B
:10ACB00080918202882311F40E946C418091EF02FE
:10ACC0009091F002892BD1F18091F8019091F901D6
:10ACD000A091FA01B091FB018093890290938A02BE
:10ACE000A0938B02B0938C0229C08091F8019091BF
:10ACF000F901A091FA01B091FB01805D9740A0405D
:10AD0000B0408093890290938A02A0938B02B09303
:10AD10008C0280914B06882311F0992702C08FE79F
:10AD200090E09093800180937F0149815A815093F4
:10AD30007802409377028EE280934001009177027F
:10AD400010917802A090F801B090F901C090FA013A
:10AD5000D090FB012091890230918A0240918B02B0
:10AD600050918C022A153B054C055D0524F080911D
:10AD70001A0980FD6CC280915702882309F067C2CE
:10AD80008091EF029091F002892B49F000917702B7
:10AD90001091780210922F0310922E03DCC0D6017E
:10ADA000C501821B930BA40BB50B80930D039093ED
:10ADB0000E03A0930F03B0931003823050E8950761
:10ADC0005FEFA5075FEFB5072CF481E090E8AFEFE8
:10ADD000BFEF09C08F5F9F47A040B04064F08FEF86
:10ADE0009FE7A0E0B0E080930D0390930E03A09343
:10ADF0000F03B093100380910D0390910E03909375
:10AE00002F0380932E0380917801282F3327442726
:10AE1000552780910D0390910E03A0910F03B091DF
:10AE20001003BC01CD010E94B57297FF04C0615EA2
:10AE30007F4F8F4F9F4F55E09595879577956795F5
:10AE40005A95D1F760930D0370930E0380930F030F
:10AE5000909310036530AEEF7A07AFEF8A07AFEF3C
:10AE60009A072CF484E09EEFAFEFBFEF09C060506B
:10AE700074408040904064F080E094E0A0E0B0E056
:10AE800080930D0390930E03A0930F03B0931003D0
:10AE900080900D0390900E03609102027091030266
:10AEA00077FF02C0695F7F4F9B0143E0359527958F
:10AEB0004A95E1F7EFEF22383E071CF421E83FEF17
:10AEC00005C02038310514F020E830E0C901AA2778
:10AED00097FDA095BA2F2091790133274427552754
:10AEE000BC01CD010E94B57297FF04C06D5F7F4F1A
:10AEF0008F4F9F4F22E095958795779567952A9577
:10AF0000D1F79B01FFEF61307F071CF420E03FEF9A
:10AF100006C06F3F710519F014F020E031E0809118
:10AF20006002807C49F0C90137FD03969C0135958C
:10AF30002795359527950DC080911A0980FF09C086
:10AF4000C90137FD07969C01A3E035952795AA9581
:10AF5000E1F7820E931E20917701222309F454C059
:10AF60006091AD027091AE028091AF029091B002FB
:10AF700097FF04C061587F4F8F4F9F4FF7E0959523
:10AF8000879577956795FA95D1F733274427552705
:10AF90000E94B57297FF04C0615E7F4F8F4F9F4F35
:10AFA000E5E09595879577956795EA95D1F7609354
:10AFB0000D0370930E0380930F0390931003613879
:10AFC0002FEF72072FEF82072FEF92072CF480E804
:10AFD0009FEFAFEFBFEF0AC06F3F7105810591058D
:10AFE00069F064F080E091E0A0E0B0E080930D03B0
:10AFF00090930E03A0930F03B093100380910D0361
:10B0000090910E03880E991EC401AA2797FDA09562
:10B01000BA2FC0907702D09078029601442737FD6E
:10B020004095542FBC01CD010E94B57297FF04C01A
:10B0300061507E4F8F4F9F4F59E09595879577953B
:10B0400067955A95D1F7061B170B8091870290914F
:10B050008802892B09F064C01C141D040CF060C028
:10B0600020912E0330912F03C90137FF03C0309583
:10B0700021953F4F2D33310540F48091A5029091E9
:10B08000A6028017910774F526C02C53304045E086
:10B09000369527954A95E1F72031310510F02FE0DC
:10B0A00030E04091A5025091A60218161906E4F46A
:10B0B00080E190E0821B930B489F9001499F300DE7
:10B0C000589F300D112494E0369527959A95E1F715
:10B0D0002017310720F580917D0190917E0108179E
:10B0E0001907F4F08C011CC0205F3F4F80917D0157
:10B0F00090917E01829FB001839F700D929F700D91
:10B1000011249B0184E0369527958A95E1F7401735
:10B11000510714F08A0104C00217130708F08901CF
:10B12000C801AA2797FDA095BA2F1DE0880F991F87
:10B13000AA1FBB1F1A95D1F7209107093091080962
:10B14000442737FD4095542FBC01CD010E9429733F
:10B15000209311033093120340931303509314036D
:10B1600000911103109112038091300390913103EB
:10B170009C01220F331F280F391F200F311F37FF6B
:10B1800002C02D5F3F4FA9015595479555954795AD
:10B19000509331034093300380914306282F332787
:10B1A000220F331F220F331F241735076CF48091B1
:10B1B0004609282F3327220F331F220F331F205514
:10B1C00030404217530724F030933103209330036B
:10B1D00080911A0980FF14C080913003909131034F
:10B1E000A981BA818A179B0724F0B0933103A093F9
:10B1F0003003E0913003F0913103FA83E98327C0F3
:10B2000029813A812C193D0937FF02C02D5F3F4F3C
:10B210003595279535952795409130035091310309
:10B22000420F531F5A83498312C00E946C416981A7
:10B230007A81709331036093300380916002806C57
:10B240008093600280915F028D7F80935F02809186
:10B25000600299279C012270307081FF30C180917B
:10B26000320390913303A0913403B09135030097DA
:10B27000A105B10521F0809191028130B9F480914E
:10B28000770290917802AA2797FDA095BA2F2EE019
:10B29000880F991FAA1FBB1F2A95D1F780933203ED
:10B2A00090933303A0933403B093350380919102BC
:10B2B000813019F482E08093910289819A817C0126
:10B2C0000027F7FC0095102F80910709909108093D
:10B2D0009C01442737FD4095542FC801B7010E94B7
:10B2E000B572DC01CB018093110390931203A093FC
:10B2F0001303B0931403B7FF04C08150904EAF4FB7
:10B30000BF4F5C016D010DE0D594C794B794A7942D
:10B310000A95D1F7A0921103B0921203C0921303C1
:10B32000D092140360916102709162029FE0603AD2
:10B33000790750F58091320390913303A091340343
:10B34000B09135039C01AD011AE0569547953795AC
:10B3500027951A95D1F7821B930BA40BB50BA60169
:10B360009501F4E0220F331F441F551FFA95D1F7C2
:10B37000820F931FA41FB51F809332039093330352
:10B38000A0933403B093350360547F4118F5809146
:10B39000320390913303A0913403B09135039C01A3
:10B3A000AD01ECE05695479537952795EA95D1F78D
:10B3B000821B930BA40BB50BA601950172E0220F23
:10B3C000331F441F551F7A95D1F7820F931FA41F77
:10B3D000B51F38C080910202909103028091020251
:10B3E0009091030297FF03C0909581959F4F8436FB
:10B3F000910584F58091F8019091F90120918902DD
:10B4000030918A02821B930B81509F4F8F5F914036
:10B4100008F58091320390913303A0913403B091E9
:10B4200035039C01AD016EE05695479537952795FC
:10B430006A95D1F7821B930BA40BB50B8A0D9B1D4C
:10B44000AC1DBD1D8093320390933303A09334034E
:10B45000B09335038091320390913303A09134036C
:10B46000B09135033EE0B695A795979587953A95A7
:10B47000D1F7909378028093770240914906442354
:10B4800099F055279C01BA010E94F472C901861BEC
:10B49000970B9093A6028093A502260F371F309337
:10B4A0007E0120937D011FC01092A6021092A5027A
:10B4B0008FEF93E090937E0180937D0114C01092F2
:10B4C00091021092320310923303109234031092BF
:10B4D0003503309378022093770205C08091600293
:10B4E000806C809360028091460381FF37C0898120
:10B4F0009A8197FD039695958795959587952091C7
:10B500005C0230915D022817390760F48091770260
:10B5100090917802892B31F0220F331F220F331FB5
:10B520003A8329838091F8019091F901A091FA0161
:10B53000B091FB018093890290938A02A0938B02C1
:10B54000B0938C0288E99AE39093E9018093E80133
:10B5500080E09EE090930C0180930B0120910609FE
:10B56000822F9927880F991F880F991F8896E98144
:10B57000FA818E179F0714F09A8389838091460978
:10B580009927880F991F880F991F805590404981EE
:10B590005A818417950714F49A83898380913F0216
:10B5A000882341F48091E6098E3F20F080914A0380
:10B5B0008823D9F080916102909162020297C0972E
:10B5C000A0F469817A81161617067CF481E090E078
:10B5D0009093620280936102822F9927880F991FAE
:10B5E000880F991F88969A8389838091E701882321
:10B5F00011F40E94945EA981BA81B0939F05A09333
:10B600009E058091090390910A03A0910B03B091CC
:10B610000C03F2E0880F991FAA1FBB1FFA95D1F700
:10B620000091490910914A09081B190BE981FA8117
:10B63000E13AF1058CF0CF01F7FD019695958795DC
:10B64000801791070CF48C01909581959F4F0817F6
:10B6500019076CF48C010BC00135110514F000E5DD
:10B6600010E0FFEF003B1F0714F400EB1FEF809189
:10B670004609282F3327220F331F220F331FC901FA
:10B6800049815A81841B950B801791070CF48C011A
:10B6900069817A81621B730B061717070CF48B0103
:10B6A00080910109909102096091A3027091A40216
:10B6B000861B970B90930D0980930C09D0901C0961
:10B6C0002091B5023091B6024091B7025091B80274
:10B6D000DD2041F0661A770AC301AA2797FDA095DD
:10B6E000BA2F04C0AA2797FDA095BA2F280F391F9B
:10B6F0004A1F5B1F2093B5023093B6024093B702F6
:10B700005093B8028091B5029091B602A091B70211
:10B71000B091B80281509A4FA040B04064F080E0F0
:10B720009AEFA0E0B0E08093B5029093B602A093A8
:10B73000B702B093B8028091B5029091B602A09181
:10B74000B702B091B80280509640AF4FBF4F64F43B
:10B7500080E096E0AFEFBFEF8093B5029093B60222
:10B76000A093B702B093B802C090580620910C097C
:10B7700030910D0978E07C1598F08C2D9927829FE7
:10B78000D001839FB00D929FB00D1124CD01B7FD64
:10B7900007965C0163E0B594A7946A95E1F712C03F
:10B7A0008C2D86959927829FF001839FF00D929FA3
:10B7B000F00D1124CF01F7FD03965C01B594A79419
:10B7C000B594A79480907A0190907B0194014427CE
:10B7D00037FD4095542F8091B5029091B602A0910B
:10B7E000B702B091B802BC01CD010E942973A20E2C
:10B7F000B31EE09064016E2D772788279927980162
:10B8000017FF04C022273327201B310B37FF02C04C
:10B810002F5F3F4F3595279549815A81240F351F5A
:10B82000442737FD4095542F0E94B57297FF04C0FE
:10B83000615C7F4F8F4F9F4F26E095958795779559
:10B8400067952A95D1F79B016A157B050CF45B017E
:10B8500066277727621B730BA616B7060CF45B01ED
:10B860008091F6089091F7086091A1027091A20270
:10B87000861B970B9093F5088093F4082091B102F2
:10B880003091B2024091B3025091B402DD2041F0F8
:10B89000461A570AC201AA2797FDA095BA2F04C0DD
:10B8A000AA2797FDA095BA2F280F391F4A1F5B1FA3
:10B8B0002093B1023093B2024093B3025093B4028A
:10B8C0008091B1029091B202A091B302B091B40202
:10B8D00081509A4FA040B04064F080E09AEFA0E021
:10B8E000B0E08093B1029093B202A093B302B09300
:10B8F000B4028091B1029091B202A091B302B091D2
:10B90000B40280509640AF4FBF4F64F480E096E0A1
:10B91000AFEFBFEF8093B1029093B202A093B30256
:10B92000B093B4022091F4083091F50878E07C15CA
:10B9300098F08C2D9927829FD001839FB00D929F04
:10B94000B00D1124CD01B7FD07966C01B3E0D5947D
:10B95000C794BA95E1F712C0C6948C2D9927829F9F
:10B96000F001839FF00D929FF00D1124CF01F7FDA0
:10B9700003966C01D594C794D594C7949401442739
:10B9800037FD4095542F8091B1029091B202A09161
:10B99000B302B091B402BC01CD010E942973C20E62
:10B9A000D31E6E2D772788279927980117FF04C08B
:10B9B00022273327201B310B37FF02C02F5F3F4F59
:10B9C0003595279549815A81240F351F442737FD26
:10B9D0004095542F0E94B57297FF04C0615C7F4F61
:10B9E0008F4F9F4FE6E09595879577956795EA95F8
:10B9F000D1F79B016C157D050CF46B016627772749
:10BA0000621B730BC616D7060CF46B018091E7011D
:10BA1000882311F40E94945E80910609682F77278D
:10BA20007D836C8380914609A82FBB27BF83AE839B
:10BA3000E0909B066AE6862E67E0962E51ED652E15
:10BA400056E0752E4FE0342E3DE1432E39E0532E63
:10BA5000F301208112160CF030C1203429F4298121
:10BA60003A813B872A871FC049815A81CA01AA2788
:10BA700097FDA095BA2F332727FD3095432F532FDD
:10BA8000BC01CD010E94B57297FF04C0615C7F4F7D
:10BA90008F4F9F4F26E095958795779567952A95C7
:10BAA000D1F77B876A87F3012181203439F42A8515
:10BAB0003B852A0D3B1D3B872A872AC0203C39F451
:10BAC0004A855B854A195B095B874A8721C0C501A6
:10BAD000AA2797FDA095BA2F332727FD3095432F2E
:10BAE000532FBC01CD010E94B57297FF04C0615C69
:10BAF0007F4F8F4F9F4FB6E09595879577956795C8
:10BB0000BA95D1F7AA85BB85A60FB71FBB87AA87B1
:10BB1000F3012281203439F42A853B852C0D3D1D0B
:10BB20003B872A872AC0203C39F44A855B854C191B
:10BB30005D095B874A8721C0C601AA2797FDA095AA
:10BB4000BA2F332727FD3095432F532FBC01CD014A
:10BB50000E94B57297FF04C0615C7F4F8F4F9F4F6B
:10BB6000A6E09595879577956795AA95D1F7AA85CB
:10BB7000BB85A60FB71FBB87AA87F301238120349B
:10BB800039F42A853B85200F311F3B872A872AC03D
:10BB9000203C39F44A855B85401B510B5B874A8703
:10BBA00021C0C801AA2797FDA095BA2F332727FDEA
:10BBB0003095432F532FBC01CD010E94B57297FFE2
:10BBC00004C0615C7F4F8F4F9F4FF6E0959587953E
:10BBD00077956795FA95D1F7AA85BB85A60FB71F0C
:10BBE000BB87AA87F401808181FD08C0D2018D91B5
:10BBF0009C91EA85FB858E179F0774F4D2018D9185
:10BC00009C91EA85FB858E0F9F1F97FD0196959568
:10BC100087959B878A871EC0EE2049F42A853B853D
:10BC2000220F331F281B390B3B872A8713C031E0B3
:10BC30003E1580F42E2D33274A855B85841B950B9A
:10BC4000B9010E94F472CB016A857B85680F791F68
:10BC50007B876A878C819D81880F991F880F991F28
:10BC6000AA85BB858A179B075CF48E819F81880F0C
:10BC7000991F880F991FEA85FB85E817F90714F0CB
:10BC80009B878A878A859B8597FD039695958795DF
:10BC900095958795F4018183880F991F880F991FC7
:10BCA0002A853B85281B390BC901880F8283EA85C9
:10BCB000FB85D201ED93FC9303C0F4011182128243
:10BCC0003A9422E030E0420E531E44E050E0640E0D
:10BCD000751E6FE070E0860E971E37FEB9CEE2E16A
:10BCE000C55F0C94607384B1806A84B93D9A82E523
:10BCF0008CBD1DBC459A81E080935A098AEA8093E5
:10BD00006B0983E880936C098AE080936D09109237
:10BD10006F0910926E0910927109109270091092B9
:10BD2000D30910928F09089530915A09332309F0ED
:10BD300070C00DB407FE6DC085E08093E701459AA1
:10BD40002EB580914E0399278130910589F082307C
:10BD500091051CF4892B21F03EC00297B9F03BC03D
:10BD600030938E0920934F032138A9F581E008C054
:10BD7000253549F480914F03820F80934F0382E071
:10BD800080934E0328C030934E0325C080918E09C6
:10BD9000E82FFF27E055F64F20838F5F80938E09B1
:10BDA00090914F038032A0F0291769F480E2A0EB54
:10BDB000B9E0E0E9F9E00D9001928A95E1F781E0C0
:10BDC00080938F0902C030938F0910924E0303C0F5
:10BDD000920F90934F0320916A092232A0F4459864
:10BDE0000000000000000000E0916309F091640988
:10BDF000E20FF11D80818EBD80918C099081890FA9
:10BE000080938C0903C081E080935A092F5F2093AF
:10BE10006A090895EF92FF920F931F93CF93DF93D8
:10BE2000809151069927880F991F880F991F7C01CF
:10BE30000027F7FC0095102F8091D1029091D2023B
:10BE4000A091D302B091D402BC01CD01A801970109
:10BE50000E94297330936F0920936E098091CD025F
:10BE60009091CE02A091CF02B091D002BC01CD0141
:10BE7000A80197010E9429733093710920937009DA
:10BE80002091500930915109409152095091530924
:10BE9000DA01C90163E0880F991FAA1FBB1F6A95C9
:10BEA000D1F7820F931FA41FB51F820F931FA41FEA
:10BEB000B51F2091410130914201409143015091C1
:10BEC0004401BC01CD010E9429733093770920936E
:10BED0007609C091E902D091EA0280910F02909117
:10BEE00010029E01281B390B30937D0920937C0999
:10BEF000E091D902F091DA0280911309909114092E
:10BF0000BF010E94F4729B01220F331F220F331FC7
:10BF1000260F371F260F371F37FF02C02D5F3F4FF9
:10BF20003595279535952795309373092093720998
:10BF300080914C0990914D09BF010E94F4729B01C0
:10BF4000220F331F220F331F260F371F260F371FD5
:10BF500037FF02C02D5F3F4F3595279535952795C3
:10BF600030937509209374091092DA021092D90265
:10BF7000109214091092130910924D0910924C0955
:10BF800080916D0999278C30910509F436C28D3066
:10BF900091053CF48A30910599F00B9709F4FEC1A4
:10BFA0008FC28131910509F4BDC18231910524F41C
:10BFB000409709F442C084C2439709F4A6C080C2E6
:10BFC00080916F028093800980916E028093810935
:10BFD00080916D028093820980916C028093830925
:10BFE00080916B028093840980916A028093850915
:10BFF0008091690280938609809168028093870905
:10C00000809160028093880980915F028093890902
:10C0100080916002837F80936002809123019091E0
:10C02000240190938B0980938A09429949C2809197
:10C030005F02877F80935F0243C28091E009909105
:10C04000E109909381098093800980915003909138
:10C050005203892B809382098091E609809383099A
:10C06000809186060E94403E809384098091400121
:10C070008093850920915003822F9927FC01C4E009
:10C08000EE0FFF1FCA95E1F7E81BF90BE659F84FD1
:10C090008685809386098081809387098681809335
:10C0A0008809838180938909878180938A098581A2
:10C0B00080938B092F5F20935003E22FFF27EE0F11
:10C0C000FF1FEE0FFF1FEC53F94F85851816D4F0B4
:10C0D0002223C1F0822F992701966DE070E00E9423
:10C0E000F472AC01282FE82FFF27EE0FFF1FEE0F91
:10C0F000FF1FEC53F94F8585181614F0442351F7B0
:10C100004093500310925203DBC120915103822FC0
:10C11000992781309105E9F1823091051CF4892B32
:10C1200049F0CEC08230910509F465C0039709F447
:10C1300096C0C6C08EE080936D0992E0909380090E
:10C140008AE080938109909382098BE4809383092C
:10C1500080910301809384098091AC0680938509C6
:10C1600080919C06809386098091B0068093870910
:10C170008091B80380938809809101018093890997
:10C180008091B4019091B50190938B0980938A09B5
:10C1900093C08DE080936D098091020180938009A6
:10C1A0008091870680938109809188068093820917
:10C1B000809189068093830980918A0680938409FF
:10C1C00080918E068093850980918F0680938609E1
:10C1D00080919006809387098091930680938809C7
:10C1E00080919106809389098091920680938A09B3
:10C1F0008091940631C084E180936D098091E302BF
:10C200009091E40290938109809380098091E102EA
:10C210009091E20290938309809382098091DF02DA
:10C220009091E002909385098093840980916C0637
:10C23000809386098091AD068093870980913E099D
:10C240008093880980911A098093890980919806C2
:10C2500080938A098091B60680938B092DC08FE068
:10C2600080936D0980916C018093800980916B01AE
:10C270008093810980919606809382098091FE08BF
:10C28000809383098091B406809384098091000192
:10C29000809385098091530390915403909387096B
:10C2A00080938609809156028093880910928909AB
:10C2B00010928A0910928B092F5F2093510300C1BD
:10C2C00082E180936D098091ED029091EE0290934E
:10C2D0008109809380098091EB029091EC02909308
:10C2E000830980938209D0938509C0938409809142
:10C2F00079068093860980919506809387098091BD
:10C300005C068093880980918B06809389098091CF
:10C310008C0680938A0980918D0680938B091092F8
:10C320005103CEC0809185068093800910928109C7
:10C330008091E4099091E5099093830980938209A3
:10C3400080915502809384098091770380938509B9
:10C350008091750380938609809174038093870987
:10C3600010927703109275031092740380917601F6
:10C37000882329F08091AB029091AC0204C0809197
:10C38000FB089091FC08909389098093880980911B
:10C390005E0280938A098091B10690C08091A708BF
:10C3A0008093800980915A088093810980915C086C
:10C3B0008093820980915F08809383098091940221
:10C3C00080938409809195028093850980919602DB
:10C3D00080938609809197028093870980919802C3
:10C3E00080938809809199028093890980919A02AB
:10C3F00080938A0980919B0261C08091D00385302F
:10C4000018F01092D00385E0809380098091770224
:10C410009091780297FD03969595879595958795C8
:10C420008093810980918D0290918E02A0918F025C
:10C43000B0919002BC01CD0125E030E040E050E039
:10C440000E94297330938309209382098091890285
:10C4500090918A02A0918B02B0918C02BC01CD0117
:10C4600025E030E040E050E00E94297330938509D8
:10C47000209384098091B503809386099091B60337
:10C48000909387098F778093B50390719093B6034B
:10C490008091C805809388098091930280938909CF
:10C4A0008091550380938A0980919E0590919F0504
:10C4B00097FD0396959587959595879580938B091C
:10C4C00080918F09882309F458C160919009809167
:10C4D000A201681719F08AEF8093A0016093A2016E
:10C4E00081E080938C014091910950919209CA0199
:10C4F00081509E4F8F5F9340B0F42091930930910B
:10C500009409C90181509E4F8F5F934060F48091E0
:10C51000420685FF08C050933C0340933B03309391
:10C520003A0320933903809197099091980921E06B
:10C530008936920724F49093900180938F01209183
:10C54000A1093091A2098091E8019091E901821737
:10C55000930740F48091BA01882321F43093E901D4
:10C560002093E801862F99278836910509F452C057
:10C570008936910524F48736910551F006C1893634
:10C58000910509F47CC08B36910509F4D1C0FDC03A
:10C590008091A3098093D0098091A4098093D20946
:10C5A0008091A5098093D1098091A60980938B0180
:10C5B0008091A70980FF03C081E0809345038091AB
:10C5C000A8098093A1018091A90980934D038091CE
:10C5D000AA09809338038091AB099091AC0997FD2B
:10C5E00004C090938E0180938D012091430330917C
:10C5F00044038091AD099091AE09280F391F37FF90
:10C6000002C02F5F3F4F3595279530934403209309
:10C610004303BBC08091A309809365098091A4095D
:10C62000809366098091A509809367098091A60986
:10C63000809368098091A7098093690980918E058C
:10C640009091A809892B80938E0590918F05937006
:10C650008091A9098C70982B90938F058091AA09DD
:10C6600080934A038091AB09809392018091AC0939
:10C670008093D3098091AD098093460386C0809151
:10C68000A30980935B098091A40980935C09809140
:10C69000A50980935D098091A60980935E09809128
:10C6A000A7099091A8099093600980935F098091F0
:10C6B000A9099091AA0990936209809361098091D8
:10C6C0004C03882329F48091AB09815880934C0353
:10C6D0008091AB09992787FD909590939C08809352
:10C6E0009B088091AC09809382028091AD09909162
:10C6F000AE099C01442737FD4095542FDA01C9014A
:10C7000063E0880F991FAA1FBB1F6A95D1F7820F9C
:10C71000931FA41FB51F820F931FA41FB51F8093E3
:10C72000830290938402A0938502B09386022DC069
:10C730008091A309809349038091A40980934803C1
:10C740008091A509809347038091A70980937A037C
:10C750008091A809809379038091AB098093780335
:10C760008091AC09809376038091AD099091AE09D8
:10C77000909348098093470908C010923C03109297
:10C780003B0310923A0310923903E6E0CDB7DEB7CF
:10C790000C946C7380915A09882319F480E090E01E
:10C7A000089545988BE699E0909364098093630916
:10C7B00090914B03E92FFF27ED56FE4F9F5F90931B
:10C7C0004B03808180936D099D3010F010924B03D4
:10C7D00010925A090E940A5F81E080936A09809151
:10C7E0006B0980938C098EBD81E090E0089587B13C
:10C7F0008C6087B9429843981092570380E88093E1
:10C80000A401109256038093A301089580915503CB
:10C81000882339F480919B0890919C0881588093DB
:10C82000620380915C03815080935C038F3F09F029
:10C830006DC180917F0680935E0380918106809315
:10C840005F0389E080935C03809160029927807385
:10C850009070892B41F48091B60380FD04C08091D3
:10C8600093028823E9F480918306882351F0809114
:10C870006003882319F484E08093570381E0809358
:10C88000600380918406882379F080916103882376
:10C8900019F484E08093560381E08093610304C01F
:10C8A000109260031092610380916003882309F065
:10C8B00088C08091B306282F332724FF07C08091BA
:10C8C0009202882319F425FD95C096C090918006A8
:10C8D000983F48F0809115098D3D28F080915E03C6
:10C8E00088236CF00AC0983F78F080911509853054
:10C8F00059F480915E0387FF02C0429A01C04298BA
:10C9000081E08093A4015AC08091570381508093A5
:10C9100057038F3F09F071C08091B60685FF35C07F
:10C9200090916203892F869580935703992361F430
:10C930009093550380915E0387FF02C0429A01C025
:10C9400042981092A40159C081E0809355038091D0
:10C95000A40190915E03882359F480914C03809345
:10C96000620380E48093A40199230CF443C044C083
:10C97000982311F0429A01C0429886958093A401B1
:10C980008130D9F510924C0338C0809115098695F5
:10C99000809357038091A401813021F410926203A7
:10C9A00080E401C086958093A4018091A4019091B8
:10C9B0005E03892311F0429A01C0429810925503F8
:10C9C0001CC0809157038150809357038F3FA9F477
:10C9D00089E0809357038091A401813011F480E8AD
:10C9E00001C086958093A4018091A4019091830653
:10C9F000892311F0429A01C04298809161038823F3
:10CA000009F043C09091B30697FF07C0809192024E
:10CA1000882319F496FD52C053C090918206983F26
:10CA200048F0809145098D3D28F080915F0388236F
:10CA30006CF00AC0983F78F080914509853059F430
:10CA400080915F0387FF02C0439A01C0439881E051
:10CA50008093A30136C08091560381508093560382
:10CA60008F3F79F580914509869580935603809193
:10CA7000A301813011F480E401C086958093A30165
:10CA80008091A30190915F0317C08091560381505C
:10CA9000809356038F3FA9F489E0809356038091D9
:10CAA000A301813011F480E801C086958093A30131
:10CAB0008091A30190918406892311F0439A01C0CB
:10CAC0004398429B15C080915D0382FD0CC080E8B5
:10CAD0008093520380915303909154030196909355
:10CAE00054038093530380915F02886080935F02B8
:10CAF000439B04C080915F02806103C080915F020C
:10CB00008F7E80935F0288B180935D0308950F93B9
:10CB10001F93CF93DF93482FEB0180919302E42F73
:10CB2000FF27843BD8F08F010E0F1F1FF801EF592C
:10CB3000F74F808191819B01281B390BC90163E06C
:10CB400070E00E94F472CB01880F991F860F971F27
:10CB50000755174FF8019183808306C0EE0FFF1F22
:10CB6000E755F74F11821082E42FFF27EE0FFF1FCA
:10CB7000EF59F74FD183C083DF91CF911F910F9170
:10CB800008954FB724E130E0F8948091C9008F7781
:10CB90008093C9008091C9008F7B8093C9008091E8
:10CBA000C9008F7D8093C900832F99278093CD0082
:10CBB0002093CC008091C80082608093C80080E1FF
:10CBC0008093C9008091CA008F778093CA008091BA
:10CBD000CA008F7B8093CA008091CA008F7D8093AA
:10CBE000CA008091CA008F7E8093CA008091CA00DB
:10CBF000877F8093CA008091C9008B7F8093C90092
:10CC00008091CA0084608093CA008091CA008260CB
:10CC10008093CA008091C80087FF03C08091CE0036
:10CC2000F9CF8091C90080688093C9004FBF0895F3
:10CC3000EF92FF920F931F93CF93DF93482F00E063
:10CC400010E08091A501813061F41092A50184E487
:10CC50008093650310926703109266031092680335
:10CC600003C280916503882319F421E030E001C0FC
:10CC7000980190916603992371F4232B11F081E0C0
:10CC800010C084E4809365039093670390936603D8
:10CC900090936803D2C1913069F4232B09F0C3C18A
:10CCA00082E080936603809167038F5F80936703C0
:10CCB00083E0C1C19230D1F4232B09F0B4C183E0E9
:10CCC000809365034093680390916703923039F431
:10CCD0001092690347FF03C081E08093690383E0FA
:10CCE000809366039F5F90936703A7C1933009F019
:10CCF0009AC1232B09F097C19093650382E080933A
:10CD00006603809167038F5F8093670320916803B8
:10CD1000822F9927782F6627842F9927682B792BC4
:10CD200080915C06813051F47370CB018050924049
:10CD300063E070E00E94F472EB0119C0823069F484
:10CD40007770CB018050944066E070E00E94F472EE
:10CD5000EB012695269526950CC0EB01D370C8569D
:10CD6000D140CE01D7FD0196EC01D595C79526950A
:10CD70002695022F11270F7010700F5F1F4F0D3077
:10CD8000110508F049C10230110519F404E010E062
:10CD900005C00430110511F402E010E0D801A00F25
:10CDA000B11FFD01EF59F74F808191819E01281B32
:10CDB000390BC90137FF03C0909581959F4F0697A6
:10CDC00004F5E0919F06EE2351F0FF27EE0FFF1FC1
:10CDD000EF59F74F808191818436910594F48091C9
:10CDE0009302883C30F480919302865F8093930293
:10CDF00008C088EC8093930280916F008F7D8093B0
:10CE00006F00AF59B74F8D919C91BC01660F771F92
:10CE1000680F791F6C0F7D1F77FF02C06D5F7F4F1A
:10CE20007B01F594E794F594E794CE0101968E1575
:10CE30009F0524F40894E108F10808C0CE01019789
:10CE4000E816F9061CF40894E11CF11C06301105E3
:10CE500009F0CEC0C536D1050CF4A5C0909164038D
:10CE6000E92FFF27EB52F64FE081ED3729F480914F
:10CE70006303809580936303963061F4809163032C
:10CE8000882311F0E338B9F0882309F088C0ED3722
:10CE900091F085C0993009F082C0809163038823A6
:10CEA00029F48091DE09833831F079C08091DE0960
:10CEB0008D3709F074C08091D6098D3739F480918F
:10CEC000D709833899F463E87FEF0DC0833871F494
:10CED0008091D709833819F460E070E004C08D3781
:10CEE00029F46DE770E085E00E9487658091D8099C
:10CEF000992787FD9095BC0186E00E948765809107
:10CF0000D909992787FD9095BC018BE00E94876520
:10CF10008091DA09992787FD9095BC018CE00E94E9
:10CF20008765809164038930D1F58091DC098D3764
:10CF300049F480917108909172080596BC0188E0CF
:10CF40000E9487658091DD098D3749F480917108D1
:10CF5000909172080597BC0188E00E9487658091D6
:10CF600071089091720883589F4F1CF483E89FEFDB
:10CF700009C080917108909172088E37910534F044
:10CF80008DE790E090937208809371088091DB099F
:10CF9000992787FD9095BC018AE00E9487651092D1
:10CFA000640310926303CA30D1055CF4809164037A
:10CFB0008F5F80936403E82FFF27EB52F64F83E8DF
:10CFC0008083809164038A3011F4109264038FEFA0
:10CFD000CC39D8076CF480916403E82FFF27EB521B
:10CFE000F64F8DE780838091630380958093630380
:10CFF0000530110518F4B701802F0BC0053011055D
:10D0000019F4BE0187E005C007301105B1F4BE0177
:10D0100089E00E94876511C00231110570F081E03E
:10D020008093A5010AC081E08093A5011092670357
:10D030001092690384E480936503809167038031D3
:10D0400098F080916903882331F48091A5018823A9
:10D0500011F480933F0110926703109269031092BC
:10D06000660384E480936503E6E0CDB7DEB70C94F5
:10D070006C73CF93EAE5F0E0E81BF90BF7FF05C00E
:10D08000CFEFF095E195FF4F01C0C1E028E631E018
:10D09000CF01B9010E94F472FC018B35910554F067
:10D0A0008B5590408A35910538F484EB90E08E1BC7
:10D0B0009F0BFC0141E00DC0CF01855B90408A359C
:10D0C000910518F4E45BF04003C02E1B3F0BF901FF
:10D0D0004FEFEE0FFF1FEB5EF74F259134918C2F32
:10D0E000992787FD9095289FB001299F700D389F43
:10D0F000700D1124842F992787FD9095689FA001BA
:10D10000699F500D789F500D1124CA01CF91089549
:10D110000895089508950895089508950895089527
:10D12000089580E090E008951092E1091092E009DE
:10D130001092E5091092E4091092E3091092E209B5
:10D140001092E60982E390E00E947B1690936B03B5
:10D1500080936A0308959927FC0124E0EE0FFF1FD6
:10D160002A95E1F7E81BF90BE659F84F95819F3FA7
:10D1700019F480E090E00895993C18F4892F9927DC
:10D180000895808182FF07C08AE0989FC001112422
:10D19000885097400895892F99270895A0E0B0E01E
:10D1A000E4EDF8E60C944D7380916A0390916B0363
:10D1B0000E948416882309F4D6C080916A03909156
:10D1C0006B03C29690936B0380936A03C0E0D0E038
:10D1D0007E01BB247FEFC72E8091E6098E3F29F4A4
:10D1E00080915E02816080935E02DB2C0AE617E08C
:10D1F000F801838187FF1CC0B3948581893C30F09E
:10D200008D2D0E94AB68C80FD91F02C0C80FD11D59
:10D21000F8018181E80EF11C8681C81610F0C82E35
:10D2200007C08F3F29F480915E028E7F80935E025B
:10D23000D394015F1F4FFFE0FD15D0F6C092E609C1
:10D24000EF2869F5209170033091710340917203CA
:10D2500050917303BB27A52F942F832F90936F03B7
:10D2600080936E03AA27BB27281B390B4A0B5B0B45
:10D27000CE01AA27BB27280F391F4A1F5B1F209307
:10D280007003309371034093720350937303C5E0AE
:10D29000D0E080915E028E7F80935E0213C0809109
:10D2A0006E0390916F038C179D0718F4C81BD90B60
:10D2B00002C0C0E0D0E08B2D9927880F991FC80FBE
:10D2C000D91F2596D093E109C093E009CF3FD1053E
:10D2D00078F480912301909124018C9F90018D9F7F
:10D2E000300D9C9F300D1124C90164E670E013C01D
:10D2F000CE0196958795969587952091230130913B
:10D300002401289FA001299F500D389F500D112402
:10D31000CA0169E170E00E94E0727093E3096093D2
:10D32000E20980916C0390916D038C0F9D1F909387
:10D330006D0380936C0352E0813D9507A0F020912E
:10D34000E4093091E5092F5F3F4F805D9240E2E0B4
:10D35000813D9E07C0F790936D0380936C033093DB
:10D36000E5092093E409E9E0CDB7DEB70C946973D1
:10D3700008950895002422273327442751E0BB272E
:10D38000EE27FF27A0E1660F771F881F991F001C5B
:10D39000221F331F441F660F771F881F991F001C11
:10D3A000221F331F441F2AF4050E2B1F3E1F4F1F41
:10D3B00004C0051A2B0B3E0B4F0B550FBB1FEE1F66
:10D3C000587F556047FD5250AA95E9F6E695B79506
:10D3D0005795E695B7955795852F9B2F089522274A
:10D3E000332741E0552768E0880F991F221F331F1C
:10D3F000880F991F221F331F1AF4240F351F02C0F4
:10D40000241B350B440F551F487F456037FD4250A4
:10D410006A9551F75695479556954795842F0895E7
:10D42000AA2797FF04C0809590958A1F9A1F77FFBF
:10D4300004C0609570956A1F7A1F669F9001779F60
:10D44000A001679F300D411D5A1F300D411D5A1F0D
:10D45000889FF001999F2E0F3F1F401D511D899FEE
:10D46000300D411D5A1F300D411D5A1FCA01B9010F
:10D47000112480CF90917E03933240F4E92FFF274F
:10D48000EF50F64F80839F5F90937E030895833221
:10D4900018F48D5F80937E03089590E2E4EFF9E045
:10D4A0008FE19193815087FFFCCF0895CF93CFB741
:10D4B00023E031E0F8948091C9008F778093C90010
:10D4C0008091C9008F7B8093C9008091C9008F7DB6
:10D4D0008093C900832F99278093CD002093CC009F
:10D4E0008091C80082608093C80088E18093C90061
:10D4F0008091CA008F778093CA008091CA008F7B89
:10D500008093CA008091CA0080628093CA00809193
:10D51000CA0080618093CA008091CA0088608093AD
:10D52000CA008091C90084608093C9008091CA00BC
:10D5300084608093CA008091CA0082608093CA0090
:10D540008091C80087FF03C08091CE00F9CF809101
:10D55000C90080688093C9008091C900806480936D
:10D56000C9000E944D6ACFBFCF910895282F9927F7
:10D570008F709070892B31F4209580917D03822BE0
:10D5800080937D0308958091AD01882309F44BC0F9
:10D590008091600285FD04C08091B001882381F0F4
:10D5A00082E98093F10983E28093F2098091B001CE
:10D5B000882309F485E58093F3091092B00102C035
:10D5C0008093F1098091AE018F3071F480917D03D9
:10D5D0000E949168882341F081E98093F10980934A
:10D5E000F20981E38093F3091092AD018091C800A4
:10D5F00085FFFCCF8091C9008F7E8093C900809108
:10D60000C9008E7F8093C9008091F109882311F4AD
:10D610008EEF01C08EE78093CE0080917D038093D2
:10D62000AE0110927D0308951F920F920FB60F92D4
:10D6300011248F939F93EF93FF939091AD019923C2
:10D6400009F040C080917F03882361F48091F10943
:10D65000882311F483E003C0813999F481E0809339
:10D660007F030FC0833099F48091F109882349F03A
:10D670009093F1098091C9008E7F8093C9008EEF4D
:10D680001EC08091C90081608093C9000EC08332A2
:10D6900061F48091C9008E7F8093C9008FEF8093E1
:10D6A000CE0081E08093AD0118C080917F03E82F08
:10D6B000FF27EF50F64F8F5F80937F038081809329
:10D6C000CE000BC010927F03109280031092810352
:10D6D0008091C90080618093C900FF91EF919F9173
:10D6E0008F910F900FBE0F901F901895EF92FF92A1
:10D6F0000F931F93CF93DF937C018B01EA01452B9E
:10D7000039F0F80181918F01F70109952197C9F747
:10D71000E6E0CDB7DEB70C946C73EF92FF920F93F7
:10D720001F93CF93DF937C018B01EA01452B41F0DE
:10D73000F8010F5F1F4F8491F70109952197C1F7F9
:10D74000E6E0CDB7DEB70C946C730F931F93CF93C5
:10D750008C01C62F161634F480E2F8010995C150E9
:10D760001C16D4F3CF911F910F9108950F931F931F
:10D77000CF938C01C62F161634F480E3F801099577
:10D78000C1501C16D4F3CF911F910F910895A5E3BA
:10D79000B0E0EDECFBE60C9444732E96EEADFFADDD
:10D7A0002E9788249924540180917C03882321F4A6
:10D7B0002C961FAE1EAE2C97AEE44A2E512C4C0E6A
:10D7C0005D1E6F01B60105C0153239F00894C11C09
:10D7D000D11CF60114911123B9F7A601461B570B72
:10D7E00031F02C968EAD9FAD2C970E948D6B11233E
:10D7F00009F46AC20894C11CD11CFF24FDA6FCA632
:10D800007FEFE72EF9A6F6010894C11CD11C1491F4
:10D81000153721F0812F80628837B1F4F0FE0AC0FD
:10D82000F20124E030E0420E531E80809180A280FD
:10D83000B3800AC0F20142E050E0440E551E8081E0
:10D8400091814C01AA24BB24103221F489A588239C
:10D85000D1F61DC0133219F458E0F52AD4CF1A328C
:10D8600011F01D3291F41A3259F4F20182E090E085
:10D87000480E591EE081ECA7EE232CF6E195ECA7AB
:10D8800090E1F92AAFEDFA22BECF1B3211F419A7AD
:10D89000BACF1E32C1F5F6010894C11CD11C1491F7
:10D8A0001A3279F4F20122E030E0420E531E408138
:10D8B00051813FEF4F3F530714F44FEF5FEFE42EDA
:10D8C000A2CF40E050E0812F80538A30A0F4CA01FB
:10D8D00063E0880F991F6A95E1F7840F951F480F41
:10D8E000591F410F511D40535040F6010894C11C6F
:10D8F000D11C1491E8CF8FEF4F3F580714F44FEF2E
:10D900005FEFE42E85CF103329F4F4FC7CCF90E256
:10D91000F92A79CF812F81538930D8F440E050E043
:10D92000CA0133E0880F991F3A95E1F7840F951FDC
:10D93000480F591F410F511D40535040F6010894A4
:10D94000C11CD11C1491812F80538A3048F34CA7FD
:10D950005FCF183619F4A4E0FA2A55CF1C3619F413
:10D96000B1E0FB2A50CF133661F43E010894611CEC
:10D97000711CF20122E030E0420E531E8081898347
:10D980003CC1143421F0143611F0193651F5143419
:10D9900011F431E0F32AF0FE0AC0F20144E050E055
:10D9A000440E551E80809180A280B3800CC0F2018D
:10D9B00082E090E0480E591E808191814C01AA249A
:10D9C00097FCA094BA2CB7FE0AC0B094A09490948F
:10D9D0008094811C911CA11CB11C8DE289A70AE0D6
:10D9E0006FC01F3411F01F3631F41F3411F491E071
:10D9F000F92A08E064C0103779F4F201A2E0B0E03F
:10DA00004A0E5B1E808191814C01AA24BB2400E157
:10DA1000B0E4FB2A18E753C01337C1F5F20122E046
:10DA200030E0420E531E608071806114710489F4ED
:10DA30003E010894611C711C88E289838EE6F30123
:10DA4000818385E78B838CE68C838D8389E28E834B
:10DA50001F82E7FC13C08E2D992787FD9095AC019E
:10DA600060E070E0C3010E941171009729F0382E28
:10DA70003618E3140CF0C3C03E2CC1C0F301019072
:10DA80000020E9F731973E2E3618B9C0153511F050
:10DA9000153731F4153511F4F1E0FF2A0AE00FC013
:10DAA000183519F0183709F0A0C000E1F3FE07C0DF
:10DAB00081149104A104B10411F020E4F22A19A602
:10DAC000EDA6E7FC02C03FEDF32229E2622E712CA5
:10DAD0006C0E7D1E81149104A104B10421F44DA5A6
:10DAE000442309F47BC0802F9927AA27BB278EA740
:10DAF0009FA7A8ABB9AB202E332490E0891690E005
:10DB0000990691E0A90690E0B90648F0C501B40174
:10DB10002EA53FA548A959A90E94077317C0AFEFCA
:10DB20008A169104A104B10449F040F0C401B10186
:10DB30000E94E0729B014427552708C0882D602F62
:10DB40000E94D472282F3327442755272AAB3BAB9A
:10DB50004CAB5DAB0A3059F48AA9880F880F880F47
:10DB60009AA9990F890F382D381B832F10C00031C7
:10DB700039F48AA98295807F482D481B842F07C0DD
:10DB80008AA9880F880F880F582D581B852F90E081
:10DB90002EA53FA548A959A982169306A406B50645
:10DBA00008F091E08AA89BA8ACA8BDA88A3010F420
:10DBB000805D04C0895A183509F48F7DD3018E9396
:10DBC0003D01992309F099CF083041F4F3FE06C0D6
:10DBD000803321F080E3FD0182933F01CE01019665
:10DBE000382E3618F8E23F0E0BC0112309F46CC032
:10DBF0003E010894611C711C198391E0392E19A60D
:10DC0000032D2DA4231827FC222489A5882311F095
:10DC10000F5F02C0F6FC0E5F020DEF2CFF24C70160
:10DC200080739070892B49F48CA5801B682F2C96EB
:10DC30008EAD9FAD2C970E94A56B89A5882331F0EE
:10DC400041E050E0BE01675D7F4F0AC0E6FE0EC0B6
:10DC500080E38AA71BA742E050E0BE01665D7F4FCC
:10DC60002C968EAD9FAD2C970E94766BC70180736A
:10DC70009070809749F48CA5801B682F2C968EADF0
:10DC80009FAD2C970E94B66B622D2C968EAD9FADEA
:10DC90002C970E94B66B832D992787FD9095AC0138
:10DCA000B3012C968EAD9FAD2C970E94766BE4FE4F
:10DCB00089CD2CA5201B2CA7622F2C968EAD9FAD55
:10DCC0002C970E94A56B7ECDE2E1CB5C0C94607337
:10DCD0002FB740E0F894E0E0F0E081E28093570055
:10DCE0009491E2E0F0E0809357003491E4E0F0E0BA
:10DCF0008093570084912FBF9E3199F4363941F4B7
:10DD0000893011F441E00DC08A3059F442E009C075
:10DD1000373939F4863011F443E003C0853009F413
:10DD200044E0842F992708959FB7F8948091C90003
:10DD3000877F8093C9008091C9008F7E8093C9003E
:10DD40008091C9008F778093C9008091C9008F7B33
:10DD50008093C9008091C9008F7D8093C9009FBFC7
:10DD600008951F93CF93DF93182F80917C0388230E
:10DD700009F4A0C08091AC01181709F49BC08091F0
:10DD80007B03882321F40E94686E80937B0382EDDD
:10DD900091E090933E0180933D018AE699E09F9344
:10DDA0008F93CBE9D2E1DF93CF93E0919503F0918C
:10DDB000960309950F900F900F900F90812F992740
:10DDC00084309105F1F0853091051CF4892B51F0D8
:10DDD0000CC086309105D9F086309105ACF00997DA
:10DDE00041F12AC086E699E002C08DE599E09F9353
:10DDF0008F93DF93CF93E0919503F091960309956C
:10DE000027C088E599E0F3CF80E599E0F0CF88E47A
:10DE100099E09F938F93DF93CF93E0919503F091D7
:10DE20009603099588ED91E090933E0180933D0122
:10DE30000FC083E499E0DBCF87E799E09F938F934E
:10DE4000DF93CF93E0919503F0919603099510E04D
:10DE50000F900F900F900F9080917B03843011F002
:10DE6000823099F40E94946E812F8150833018F48F
:10DE70000E94C1651DC0143019F40E94566A18C072
:10DE80001930B1F40E94B86913C0112389F08DE8EC
:10DE900099E09F938F938BE992E19F938F93E09109
:10DEA0009503F091960309950F900F900F900F90A6
:10DEB0001093AC01DF91CF911F9108950F931F93A1
:10DEC000082F81E080937C034091AB01E3EFF8E001
:10DED00020E030E05FE4849199272F5F3F4F829FDD
:10DEE000B001839F700D929F700D112446275150F1
:10DEF000319657FFF0CF4093AB01EBECF8E020E018
:10DF000030E057E2849199272F5F3F4F829FB00105
:10DF1000839F700D929F700D1124462751503196AA
:10DF200057FFF0CF4093AB0180917B03882321F40E
:10DF30000E94686E80937B0387EC9BE69093960328
:10DF4000809395038091AB01833459F088E190E090
:10DF500029E20FB6F894A895809360000FBE209335
:10DF60006000073091F088EA99E09F938F938BE9E6
:10DF700092E19F938F93E0919503F0919603099519
:10DF80000F900F900F900F90EECF0E94460583E602
:10DF900090E09F938F938AE090E09F938F9382E02D
:10DFA00090E09F938F93809103016AE00E94D47266
:10DFB000892F99279F938F93809103010E94D47298
:10DFC00099279F938F9385EC99E09F938F930BE90B
:10DFD00012E11F930F93E0919503F0919603099539
:10DFE00083EF98E09F938F931F930F93E091950396
:10DFF000F091960309958BEC98E09F938F931F9374
:10E000000F93E0919503F091960309950E944605C0
:10E0100083EC8093810080916F00806280936F0019
:10E020008DB79EB746968DBF1F910F910895809131
:10E030009D068D3338F080915B0987FD03C08CE32A
:10E0400080939D0680914B06882331F0805585365C
:10E0500018F08FE780934B06089580917C03882306
:10E0600009F482C0809192038150809392038823A7
:10E0700009F069C089E18093920380919D068E33F7
:10E0800038F080915B0987FD03C08DE380939D0686
:10E09000809193028238A0F5809161029091620292
:10E0A000805D974020F08091E609843620F410923C
:10E0B00094031092930320919303309194032115BC
:10E0C0003105B1F1C90101979093940380939303B3
:10E0D000419798F180915B0984FF2FC080915F0286
:10E0E000846080935F028091690987FF26C08091D8
:10E0F0007A03882311F130939403209393031DC076
:10E1000080919302853BC8F090919D0684E1989F91
:10E11000C001112440962091930330919403281755
:10E12000390730F42F5F3F4F3093940320939303CC
:10E1300080915F028B7F80935F028091AB0183347B
:10E1400011F010927C038091AF01882321F081505F
:10E150008093AF0108958BE48093AF018091AC016F
:10E16000843011F40E94C36A08951F920F920FB673
:10E170000F9211242F933F934F935F936F937F934D
:10E180008F939F93AF93BF93EF93FF932091CE0014
:10E190008091BC018823B1F02093C6008091BC011E
:10E1A000823029F52F3F19F58FEF94E3ACE0B0E012
:10E1B000C297A109B109B7FFFBCF8091D403809327
:10E1C000CE0015C09091AC01892F8150833020F48E
:10E1D000822F0E9418660BC0943021F4822F0E9477
:10E1E000B66A05C0993019F4822F0E94B969FF916F
:10E1F000EF91BF91AF919F918F917F916F915F91BF
:10E200004F913F912F910F900FBE0F901F90189537
:10E21000FB01DC0102C005900D9241505040D8F73F
:10E220000895FC014150504030F001900616D1F79E
:10E230003197CF010895882799270895A0E0B0E08D
:10E24000E4E2F1E70C944C736C017B01EA015901A3
:10E2500021978FEFCF3FD80789F086010894C11C22
:10E26000D11CC7010894E11CF11CF5010995F801C6
:10E2700080832197FFEFCF3FDF0779F7EAE0CDB743
:10E28000DEB70C946873CF92DF92EF92FF920F93F8
:10E290001F937C016B01FB010995082FC7010196B3
:10E2A000F6010995182FC8011F910F91FF90EF906B
:10E2B000DF90CF900895A0E0B0E0E1E6F1E70C94A4
:10E2C0004E738C017B01EA01690121978FEFCF3FEB
:10E2D000D80771F0F70121917F01C8010F5F1F4F2F
:10E2E000622FF60109952197FFEFCF3FDF0791F7E6
:10E2F000E8E0CDB7DEB70C946A73CF92DF92EF926D
:10E30000FF920F931F936C018B017A01FA0109951B
:10E31000812F9927682FC6010196F70109951F9152
:10E320000F91FF90EF90DF90CF9008955058BB274A
:10E33000AA270ED0E0C0D1D030F0D6D020F031F4F2
:10E340009F3F11F41EF4C6C00EF4E095E7FBBCC07D
:10E35000E92FE2D080F3BA176207730784079507A5
:10E3600018F071F49EF5FAC00EF4E0950B2EBA2F5A
:10E37000A02D0B01B90190010C01CA01A0011124CB
:10E38000FF27591B99F0593F50F4503E68F11A1677
:10E39000F040A22F232F342F4427585FF3CF469508
:10E3A00037952795A795F0405395C9F77EF41F162A
:10E3B000BA0B620B730B840BBAF09150A1F0FF0FF4
:10E3C000BB1F661F771F881FC2F70EC0BA0F621FE0
:10E3D000731F841F48F4879577956795B795F795D0
:10E3E0009E3F08F0B3CF9395880F08F09927EE0F62
:10E3F00097958795089598D088F09F5790F0B92FFA
:10E400009927B751A0F0D1F0660F771F881F991F89
:10E410001AF0BA95C9F712C0B13081F09FD0B1E0BF
:10E4200008959CC0672F782F8827B85F39F0B93FCF
:10E43000CCF3869577956795B395D9F73EF490958B
:10E440008095709561957F4F8F4F9F4F0895E89409
:10E4500009C097FB3EF490958095709561957F4F2C
:10E460008F4F9F4F9923A9F0F92F96E9BB279395DA
:10E47000F695879577956795B795F111F8CFFAF4EA
:10E48000BB0F11F460FF1BC06F5F7F4F8F4F9F4F1B
:10E4900016C0882311F096E911C0772321F09EE879
:10E4A000872F762F05C0662371F096E8862F70E0DF
:10E4B00060E02AF09A95660F771F881FDAF7880FB9
:10E4C0009695879597F9089597F99F6780E870E08A
:10E4D00060E008959FEF80EC089500240A941616DA
:10E4E000170618060906089500240A941216130642
:10E4F000140605060895092E0394000C11F48823D0
:10E5000052F0BB0F40F4BF2B11F460FF04C06F5FEB
:10E510007F4F8F4F9F4F089557FD9058440F551FC1
:10E5200059F05F3F71F04795880F97FB991F61F095
:10E530009F3F79F087950895121613061406551F0C
:10E54000F2CF4695F1DF08C0161617061806991F78
:10E55000F1CF86957105610508940895E894BB276D
:10E5600066277727CB0197F90895629FD001739FA3
:10E57000F001829FE00DF11D649FE00DF11D929F5F
:10E58000F00D839FF00D749FF00D659FF00D99279E
:10E59000729FB00DE11DF91F639FB00DE11DF91FC2
:10E5A000BD01CF0111240895991B79E004C0991F82
:10E5B000961708F0961B881F7A95C9F780950895DD
:10E5C000AA1BBB1B51E107C0AA1FBB1FA617B70799
:10E5D00010F0A61BB70B881F991F5A95A9F78095B5
:10E5E0009095BC01CD01089597FB092E07260AD00E
:10E5F00077FD04D0E5DF06D000201AF47095619510
:10E600007F4F0895F6F7909581959F4F0895A1E269
:10E610001A2EAA1BBB1BFD010DC0AA1FBB1FEE1F9C
:10E62000FF1FA217B307E407F50720F0A21BB30BE7
:10E63000E40BF50B661F771F881F991F1A9469F763
:10E6400060957095809590959B01AC01BD01CF01BF
:10E65000089597FB092E05260ED057FD04D0D7DF6D
:10E660000AD0001C38F450954095309521953F4FC5
:10E670004F4F5F4F0895F6F790958095709561958F
:10E680007F4F8F4F9F4F08952F923F924F925F92EF
:10E690006F927F928F929F92AF92BF92CF92DF92B2
:10E6A000EF92FF920F931F93CF93DF93CDB7DEB717
:10E6B000CA1BDB0B0FB6F894DEBF0FBECDBF0994AB
:10E6C0002A88398848885F846E847D848C849B8402
:10E6D000AA84B984C884DF80EE80FD800C811B8110
:10E6E000AA81B981CE0FD11D0FB6F894DEBF0FBE3F
:10E6F000CDBFED010895EE0FFF1F0590F491E02DC1
:04E700000994FFCFAA
:10E7040004035E0A010164FF010020FFFFC01FC073
:10E714001F0101F40101737373FF03007D0000C442
:10E7240009C4099600134167696C650051756164F9
:10E73400726F0000000000000064000C09D20101A7
:10E74400200B050000000204060708080807060459
:10E754000200FEFCFAF9F8F8F8F9FAFCFE000204EB
:10E76400060708086440415A4655326464640A0244
:10E77400969696960864403A1030380132FF037F2B
:10E784000090D0030090D0030032002064FFFFFF0C
:10E79400FF64200B0A13100B0C100B0A100B111042
:10E7A400FA2068010101FFF7FFFCFF70FF010F640D
:00000001FF
